:10800000B0120020ED6A0100F76A0100F96A010070
:10801000FB6A0100FD6A0100FF6A01000000000028
:10802000000000000000000000000000016B0100E3
:108030000000000000000000216F0100E595000035
:10804000076B0100096B01000B6B01000D6B010058
:108050000F6B0100116B0100136B0100156B010028
:10806000176B0100196B01001B6B01001D6B0100F8
:108070001F6B010061930000236B0100256B010061
:10808000276B0100296B01002B6B01002D6B010098
:108090002F6B0100316B0100336B0100356B010068
:1080A000A9820000396B01003B6B01003D6B0100B0
:1080B0003F6B0100416B0100436B0100456B010008
:10820000000000000000000000000000000000006E
:108210004A2D4C696E6B204F422D43616C6C696F27
:1082200070652D6D696E6920636F6D70696C656432
:10823000204F637420203520323032302030383ADD
:1082400035363A333400436F707972696768742049
:10825000323031372D323031372053454747455280
:108260003A207777772E7365676765722E636F6D37
:1082700000000000000000000000000000000000FE
:1082800080B500F047F804480BF048FF0348044964
:10829000044A0CF005F980BD486A0100998001008C
:0882A000794501006145010070
:1082A80010B572B60D4C2078401C20706078401CC8
:1082B80060700B480068002800D080476078401E36
:1082C800607060682178012903D1002801D00EF080
:1082D8008DFE2078401E207062B610BD500E002022
:0482E800FCF1FF1F87
:1082EC0006490A68C02313433F2293430B60044999
:1082FC0008600120000603490860704718E400E09C
:08830C00FCF1FF1F00E100E09D
:108314000120800403490A6802430A600A6B02438D
:088324000A6370470480044065
:10832C00F0B58BB0049203910646EFF310800290E7
:10833C00012181F3108881204002224A11680191A9
:10834C000840112189024118116005214903401888
:10835C001060002B0FD0B0050DD10498401E801278
:10836C00441C08D0184D3746384600F031F8E8194F
:10837C00471C641EF8D1049C601007900696039D60
:10838C00059505A800F02CF80E480199016002989B
:10839C0080F310883046294622460DF029FF00282C
:1083AC000ED00A4C0025284605F03CFE204600F075
:1083BC001FF8284605F048FE204600F019F8F1E7B2
:1083CC000BB0F0BD0C3000F0FF03000020A1070043
:1083DC0008B4024B9C4608BC6047C046910E002076
:1083EC0008B4024B9C4608BC6047C046CD0E00202A
:1083FC0008B4024B9C4608BC6047C0466D10002078
:10840C0070B5EFF31084012181F3108881214902AA
:10841C00084D2E683140112292028A182A600522DA
:10842C0052038918296000F007F82E6084F3108835
:10843C0070BDC0460C3000F008B4024B9C4608BC22
:08844C006047C046910E0020BC
:1084540070B53B20C40201208502044E2046FFF77C
:10846400D3FF76196419002EF8D170BD00E0FFFF28
:10847400F0B5C7B007208002564908601020C443F5
:1084840055490C60554E336C6025AB4333643368F7
:108494000225AB4333600122019212021346543386
:1084A4004F4D2B606B604F4D2B604F4D2B603067F1
:1084B4000B6803430B603B20C10207AD28460292C0
:1084C4000DF044FE284620300FF074FC0646284682
:1084D40024300FF06FFC0746303528460FF06AFC55
:1084E40003903740791C01D1401C01D00FF04CFAA5
:1084F4003F20C50207AE30462946029A0DF026FEFB
:1085040030460FF057FC0390411C08D037490FF058
:1085140082FC06460390583E701E864100E0002609
:1085240007A8001D0FF046FC0390401C00D0019EDC
:1085340027460D3707A8C01914300FF03BFC0390F1
:10854400401C03D13F1D0B2FF4D900E001260D344C
:1085540007A8001924300FF02DFC0390401C04D10F
:10856400241D7B2CF4D9002E02D02846FFF74CFFA3
:1085740007A82946029C22460DF0E8FD0798401CF6
:1085840006D000F061FE05200DF026FD47B0F0BDD9
:108594001049886A0490486A0590086A069004A8FD
:1085A4000C21002205F07CFC0390104903AD2A46FF
:1085B40010F026FC0E4803990818039007AE042215
:1085C400304629460DF0C2FD304621460FF0F8F939
:1085D40000F010F838800440D4F00F4054F00F40FD
:1085E40014B0044010C0044004A0044080969800D5
:0485F40000BC733420
:1085F800012181F3108801F06FF8024802490160F7
:0C860800FEE7C0460CED00E00400FA059F
:0886140000487047E40C00006F
:10861C00024800684006C00F7047C04690F00F40FB
:10862C00024800688006C00F7047C04690F00F40AB
:10863C000548016860229143016055208000034980
:10864C00086048607047C04694F00F4014B0044076
:10865C00054840210160C2680A43C2605520800071
:10866C00024908607047C04688F00F4018B00440BB
:10867C0005484021016002690A43026155208000CF
:10868C00024908607047C04684F00F4018B004409F
:10869C00054820210160C2680A43C2605520800051
:1086AC00024908607047C04688F00F4014B004407F
:1086BC0005482021016002690A43026155208000AF
:1086CC00024908607047C04684F00F4014B0044063
:1086DC0010B508482021416002690A430261552205
:1086EC009200054B1A60016004690C4304611A6026
:0C86FC0010BDC04684F00F4014B00440D4
:0C870800014800687047C046C00B00200C
:1087140010B50C460146054A00201060012902D11B
:10872400204600F0EBFD02490C6010BDC40B002094
:04873400C00B002056
:1087380080B506490978012902D100F0D5FD80BD30
:10874800302181800249016080BDC046330E00207F
:04875800006CDC02D3
:08875C000048704710270000DF
:108764000C2803D880000349085870470020C043F0
:088774007047C0469862010045
:0C877C000148012101707047B50C00207D
:0C8788000148002101707047B50C002072
:1087940080B510480078012805D1104801780029D7
:1087A40005D0491E0DE00C48102181600AE00A49F9
:1087B4000A68D20602D410224A6001E010228A60BC
:1087C400FA21017006480078012801D100F070F800
:1087D40080BDC046B50C0020C0F00F40BD0C002089
:0487E400BE0C0020A7
:0887E80000487047FF2F00203C
:1087F000F8B52A4D2868002809D02949096A081ABD
:1088000028490C78052806DB0020286003E026486C
:1088100000688007C40F002C10D0224800788442E2
:1088200005D02248002101601D48006A28601D48CB
:1088300004701F480078012828D02AE01C4E3078A8
:10884000002801D10FF038FC164F387800280BD0E3
:108850001348016A29603178002915D10021397047
:10886000006A1249086014E0307800280CD10F48E3
:1088700000680B49096A081A7D2149018842D6DB44
:1088800000F08CF80120307000203870204600F095
:1088900007FB01F057FC0020F8BDC046C80B0020C4
:1088A000500E0020BF0C002050F00F40CC0B0020D9
:0488B000BE0C0020DA
:1088B400F8B53248007800285CD12F4800780028A9
:1088C40058D12F490878002801D0401E51E02D4C82
:1088D400211D05252846009106F062FF0726710335
:1088E400304606F05DFF2846214606F059FF264F24
:1088F4003046394606F054FF244801782448405C49
:108904000A224A432349891800263546324603463B
:10891400D340DB0708D04B7810249C4025430B78C8
:108924003C4610349C402643891C521C052AEED137
:1089340005273846134906F033FF072420463146FD
:1089440006F02EFF3846009906F02AFF20462946F5
:1089540006F026FF00243846214606F097FF0B4A0E
:108964001078401CC1B2042900D8044614700420B5
:1089740003490870F8BDC046C30C0020C50C002094
:10898400C10C002008050050F01F0000C20C00209C
:08899400D69501000C940100CE
:10899C00F0B597B0EB4800240470EB480470EB483A
:1089AC0001250570EA480570EA480470EA49284632
:1089BC0006F032FE07F0FCF8002800D0BFE1049569
:1089CC0006940220214606F0E7FE0420E34906F057
:1089DC00E3FE0524E249204605940D4606F0DCFE34
:1089EC000726E049304606F0D7FE29460C312046D2
:1089FC0006F0D2FEDC49304606F0CEFE2946E439BC
:108A0C00204606F0C9FED949304606F0C5FE06AC34
:108A1C003046214606F036FFD54D2F6A0598D049D1
:108A2C0006F0BAFE3046214606F02CFF072006ACB5
:108A3C00214606F027FFE078800703D4286AC01B84
:108A4C006528F3DB0524CB4D2046294606F0A4FE11
:108A5C0007260021304606F09FFE049FB9072046EA
:108A6C0006F09AFE3046394606F096FE2046294618
:108A7C0006F092FE0CA9304606F004FF07240CA960
:108A8C00204606F0FFFE0C980028F7D0052630464D
:108A9C00294606F081FE00210391204606F07CFE5B
:108AAC00B54D291D3046029106F076FE670320462F
:108ABC00394606F071FE3046294606F06DFEAF4988
:108ACC00204606F069FEAC4D10353046294606F0BE
:108ADC0063FE20460597394606F05EFE3046294671
:108AEC0006F05AFE2046A54906F056FE0CA9304663
:108AFC0006F0C8FEA0491431304606F04DFE0320A6
:108B0C000104204606F048FE9D4D291D304606F016
:108B1C0043FE2046039F394606F03EFE304629466A
:108B2C0006F03AFE2046394606F036FE3046394607
:108B3C0006F0A8FE029E052528468F4906F02CFE5D
:108B4C0007273846059906F027FE2846314606F0D9
:108B5C0023FE3846894906F01FFE0024284621468C
:108B6C0006F090FE874800F015F92846314606F0CD
:108B7C0013FE3846059906F00FFE28467E4906F08E
:108B8C000BFE38467D4906F007FE28460394214625
:108B9C0006F078FE0498C00705D07A4800F0FAF881
:108BAC0000200490C7E77D208000774908F092FFF1
:108BBC00764908600028634F00D1BAE00F20C50247
:108BCC000CA8083001904020059020210CAE2846BE
:108BDC00324600F09BFA3078002800D19BE0E52863
:108BEC0000D198E00CA8418B002900D193E0139997
:108BFC000029674E00D18EE0C07A3F2101400F2939
:108C0C0000D188E01E21084000D084E0029507A81E
:108C1C000025C5700CA90A7A202A2B4600D01346D1
:108C2C0003704A7A202A2B4600D013464370897A67
:108C3C0020292A4600D00A468270A800315807A87D
:108C4C000FF0BFF8002805D00120002D0546F4D008
:108C5C00029D60E003981828029D59D84B48006883
:108C6C00049000250CA8405D202805D014A9485577
:108C7C006D1C082DF6D1082514A846190322304680
:108C8C0001990DF05FFA0027F7702E1D039800284C
:108C9C0017D0009600252F4604984419264608360E
:108CAC0014A8314610F034F900280CD414357F1C6C
:108CBC000398B842F0D104984419224F029D009EAB
:108CCC001BE0049C14E0142003994843421B2046EB
:108CDC00143021460DF074FA14A93046009E324629
:108CEC000DF030FA0CA8408B049948511398606031
:108CFC00029D03988742134F0AD12046083014A9CD
:108D0C0032460DF01FFA0CA8408B2060139860605F
:108D1C000398401C03900598401E2035002800D075
:108D2C0052E70398192801D9192005E00398002867
:108D3C0003D100F0DFF9002003900398387017B0CE
:108D4C00F0BDC046C50C00201F0E0020200E0020D8
:108D5C00210E0020220E002000093D0002000023FD
:108D6C00F0ED00E003005FA0010000010400FA0533
:108D7C00500E00200001004008050050F01F0000BC
:108D8C004007005020A107002A970100D00B0020BB
:108D9C00CC62010008B4024B9C4608BC6047C0463C
:048DAC006D10002026
:108DB000F0B583B001242849204606F033FC06F0C4
:108DC000FDFE002846D100270197019E0296022051
:108DD000314606F0E7FC0420214906F0E3FC0520BB
:108DE000204906F0DFFC07252846214606F0DAFC7C
:108DF0002846314606F04CFD029602A9284606F0A8
:108E000047FD02982040384324D1144E3146F031BA
:108E10000525284606F0C6FC07273846214606F0F9
:108E2000C1FC2846314606F0BDFC38460E4906F026
:108E3000B9FC06F081FC06F07FFC06F07DFC06F034
:108E40007BFC2046044906F0EDFB06F0B7FE002847
:108E50002746BAD003B0F0BD00093D000CED00E09C
:0C8E600002000023440500400400FA0555
:108E6C0080B50120064906F0D7FBFFF711FCFFF790
:108E7C00EFFB4B20800000F005F8FFF7F9FB80BDFD
:108E8C0000093D0008B4024B9C4608BC6047C04634
:048E9C006D10002035
:108EA000F0B589B00446844E3078002C05D10028F6
:108EB00003D08248012101700DE0002C0BD0002866
:108EC00009D17E480078002805D0FFF771FFFFF731
:108ED000CDFFFFF791FB7A4D2878002800D1E7E01D
:108EE000009478490831052006F05CFC072707ACA0
:108EF0003846214606F0CCFC3846214606F0C8FC30
:108F00000798C103CC0F8003C60F6F4800788642D4
:108F10000BD005200DF062F8002E06D06B480178CA
:108F2000002900D12978491E0170019702966848EE
:108F3000007884420ED005200DF050F8002C09D0A6
:108F40002878421E614801788A4201D0491C00E01D
:108F5000002101705D48039400780590594F391D38
:108F600006910524204606F01DFC019D6903284654
:108F700006F018FC20460494394606F013FC554EC2
:108F80002846314606F00EFC2046394606F00AFC1B
:108F90000598400050490A5C0A2353434F4AD218AF
:108FA0000592081840784400105D10368640284627
:108FB000314606F0F7FB049F3846069906F0F2FBAF
:108FC00005980019039C407810218140284606F03E
:108FD000E9FB00263846314606F05AFC029908465D
:108FE00020435FD139480078142141433C48006850
:108FF0004258069208924018456800F081F801270F
:109000007C023849204608F06BFD0590002841D0CD
:1090100035480770354836490160364F0699C80310
:10902000049006950498C019214635462646059CAD
:10903000224600F071F8204634462E46069D314601
:10904000224607F0D7FF601C854219D336193F1915
:1090500029482D18002FE4D10C20089F4743F80819
:10906000019909034018022108AA00F055F80420CC
:1090700038400899C1402148014008911D4FCEE772
:1090800008F00CFA08F036FA002017490870059825
:1090900008F03AFDFFF78CFEFFF7E8FEFFF7ACFAA9
:1090A000039C02990A48047007480170009C024E14
:1090B000347009B0F0BDC046220E0020230E0020FF
:1090C000C50C002008050050200E00201F0E0020B7
:1090D000210E0020F01F00003E9401000C940100BE
:1090E000D00B002036970100C30C0020840C002018
:1090F000386301000080FFFF00FEFFFFFF0F00004C
:1091000010B5044C2068002803D008F0FDFC0020B6
:08911000206010BDD00B00200F
:10911800F8B515460C460A4F04267E606946C870A5
:10912800020A8A70000C487003200870084631460D
:109138000DF080FD284621460DF090FD3E60F8BDFB
:0491480084F00F4060
:10914C00F0B585B002920C460646FFF711FB002CD9
:10915C0031D0012000020090194D04276F600620C9
:10916C00049004A801210DF063FD2F6000F02AF893
:10917C006F6003A8C670310A8170310C41700221F6
:10918C000170019739460DF053FD00988442254635
:10919C0000D3009D029F384629460DF049FD0198E9
:1091AC00074908607F190297AE19641B00F00AF892
:1091BC00002C034DD1D1FFF7E1FA05B0F0BDC0464C
:0491CC0084F00F40DC
:1091D00070B582B0094D04266E600520019001A88B
:1091E00001210DF02BFD01AC012120460DF03AFDCF
:1091F0002078C007F7D12E6002B070BD84F00F4018
:10920000F0B583B00C460646FFF7B8FA0E4F0425BA
:109210007D600620029002A801210DF00FFD3D6047
:10922000FFF7D6FF7D6001A8C670310A8170310C4E
:109230004170047029460DF001FD3D60FFF7C8FF45
:0C924000FFF7A2FA03B0F0BD84F00F406D
:10924C000720800220490A6802430A601F4A1368FB
:10925C001F480340052189015B1813601D4A1368E0
:10926C0003405B181360536803405B1853609369A9
:10927C0003405B189361184A136803405B18136032
:10928C00536803405818506014480121016002696A
:10929C000A43026104210164026D0A430265022142
:1092AC000164026D0A4302650D4920220A600B69B4
:1092BC0013430B6140220A600B6913430B61016D70
:1092CC0080229143016570473880044000A004401F
:1092DC00BFF8FFFF04B0044014C0044044F00F403A
:0492EC00C4F00F407B
:1092F00018218180014901607047C046006CDC0282
:1093000080B50621414307480CF0DEFE042801DB4E
:10931000001F01E00020C0430349086000F008F886
:10932000024880BD006CDC02C40B0020D462010046
:1093300010B5094801684022914301605521890018
:10934000064A516003460C3B20241C6003682343FB
:1093500003601160002010BD94F00F4014B0044071
:10936000B0B582B0154C6578207901A90870A906BE
:1093700002D513490968884768061DD5207840063C
:109380001AD51048016801A88847002812D0207813
:10939000BF21014021700C480168102291430160F7
:1093A0000320000209490A688243012000021018C4
:1093B000086001E00198207102B0B0BD03B0064022
:1093C000D40B0020D80B002094F00F4010B00440C4
:1093D0000D218901084A13680B43136007490A6885
:1093E000102313430B6006494A780871087840221D
:1093F00002430A707047C04610B0044094F00F401A
:0494000003B006406F
:10940400F0B587B005930692039039480078012897
:1094140001D100F087F80C9804900127F80201901C
:1094240034498A6A02438A621022D543324A136855
:109434002B40136008200290C34314681C4014603E
:109444003E02304657302D4C206060601068284042
:1094540010600320000265688543AD1965601568D6
:109464001D4015602268024322600868244A0240B5
:109474000A60486A019A10434862224C0425A57088
:109484000020E070A071207260711F48039A82422C
:1094940000D30246D0001D49401811010CF012FE01
:1094A400C104C90E21706070E07802990843E0702D
:1094B400E0782843E070E07820210143E170FF2048
:1094C400000213490A688243B8031018086011485F
:1094D40005990160104804990160104806990160DB
:1094E4000348077078030E49086007B0F0BDC04612
:1094F400240E00201080044094F00F400CB004406F
:10950400AFFFFDFF00B0064040420F0000366E0181
:109514000CE400E0D40B0020DC0B0020D80B00206E
:0495240000E100E082
:1095280070B517490868102290430860154A5368B7
:10953800154C2340012005025B1953600B6808266F
:10954800B3430B6011682140491911600F490A683B
:109558000F4B13400B60C0024A6A02434A620D482F
:109568000178DF220A4002700178F7220A4002706F
:109578000178FB220A40027007480021017070BD83
:1095880094F00F400CB00440FFFCFFFF1080044033
:0C959800AFFFFDFF03B00640240E0020D2
:1095A40010B50C480078012813D10B4C2078401CCE
:1095B40020700A480068804772B6606821780129E3
:1095C40003D1002801D00DF013FD2078401E207037
:1095D40062B610BD240E0020500E0020DC0B0020CB
:1095E40010B50C4C2078401C2070FFF7D1F801F026
:1095F40033FF0CF071FC72B660682178012903D145
:10960400002801D00DF0F4FC2078401E207062B6D2
:0896140010BDC046500E0020FD
:10961C00F0B585B01D486C4621460CC80CC12CC851
:10962C002CC172B61A4D6878401C687000F0A8F80E
:10963C007D20C100174E30680CF040FD401E164ACC
:10964C0050601648036816490B400327BF07DB1907
:10965C00036000239360072313600246183A114BF2
:10966C00136002680A400121C90751180160306873
:10967C00009020460CF0B6FC6878401E6870687844
:10968C00002800D162B605B0F0BDC04624630100CD
:10969C00500E00204C0E002010E000E020ED00E009
:0896AC00FFFFFF000080000039
:0C96B400014800687047C04618E000E064
:1096C00001208106014800680840704704ED00E071
:1096D0000120C003014908600020704708ED00E048
:0C96E000014900200860704708ED00E020
:1096EC0070B520480023036001214A021E48446BD8
:1096FC00144344631D4A02641D4A14681D4D2C40DA
:10970C00146054682C4054601B4A55784024254002
:10971C0024355570194D80262E709A251570D578E4
:10972C001F262E40D6700325157153719379DB06D5
:10973C00FCD495790C231D40082DFAD154719479E1
:10974C001C40082CFBD194796406FCD51A241470A7
:10975C0094791C400C2CFBD1090402680A4302606A
:10976C0070BDC0460081044004800440000001101C
:10977C0048900440FFF8FFFE0040064000500640B1
:10978C00B0B5324C20783F2810D86079400618D4F8
:10979C002078400727D420788006400F2C49C14000
:1097AC0060788006800F20D049091EE02178C02007
:1097BC000140402911D16078C00723D10120C0039A
:1097CC003BE020791F252840411C21480CF076FCF9
:1097DC0001466079284018302EE02178014080291C
:1097EC0033D11B4829E00120C103E0784009C04671
:1097FC007844007940008744030B0E1114181C1E8A
:10980C00052009E0207A0007410F1248C84014E0F7
:10981C000520000210E00F20C0010DE005204002E1
:10982C000AE00520C0015C3006E005200002B830DB
:10983C0002E00A4800E00848484309490968090F52
:10984C00491C0CF03BFC07490860B0BD00400640C9
:10985C000024F40000093D00710B00009508000085
:08986C00448004404C0E002072
:10987400F0B5A1B00C920D46074600F025FA002879
:1098840000D5F7E07F48816A0DA800F073FB044619
:10989400002D00D1F3E0002C00D5F0E02A46794CED
:1098A40065686B423B40BB420A92099370D176488B
:1098B400874207D97648381829460CF003FCA1687A
:1098C400081803E0384629460CF0FCFB072603463B
:1098D4003340C1102268515CD940C90756D0029068
:1098E400206A0690606A0590A06A0490E06A01907C
:1098F400A06903903D46E76815A80024302208902B
:10990400214607920FF074FA1C941B942B461A9567
:10991400012519951894179420965C481F9059486E
:10992400C06916900398C0190499002901D00199BF
:109934004018059941181591069940180146283197
:109944001D9150498A6AC96A002A1F4600D04942BB
:1099540009181E9107992246089B05F051FD3028ED
:1099640000D089E0474EB16A08466840B06211A849
:1099740000F000FB0446306802992A460FF0A0FA72
:10998400002C7CD475680A9A344600E00A9A099B34
:10999400E068A1690E18A06A00280B9701D0E06A5C
:1099A4003618206A0890606A37180B98181A2D1810
:1099B400954200DB154600243846294622460C9B76
:1099C40005F01EFDA84259D10898361815A8302272
:1099D4000890214607920FF00BFA1597304628306D
:1099E4001D901C941B941A9419950B9F1897179407
:1099F4000620209025481F90224AD0691690916A2B
:109A0400D06A002900D04042089B079980191E9013
:109A14003046224605F0F4FC30282DD1194CA06ABA
:109A240001214140A1621848099A824207D9184885
:109A3400101861680CF046FBA168091804E061681D
:109A440010460CF03FFB0146206801220FF00AFA91
:109A540020460A9C641B816A0DA800F08BFA2246FA
:109A64000446002A0BD00C9840190C90EF19002CD6
:109A740005D414E7044602E0064C00E0E443204623
:109A840021B0F0BDC8F1FF1FFF0F0010FEFFFF7FE4
:089A940000F0FFEFFAFEFFFFF6
:109A9C00F0B597B000F014F900284BD400F064F83E
:109AAC002E4F386A0490786A0390B86A0290F86A6C
:109ABC000190FE68BC690BA800253022069029464F
:109ACC0005920FF091F91295119510950F950E9531
:109ADC000D950720169022481590A019029900297F
:109AEC0001D001994018039941180B91F9690C9117
:109AFC0004994018014628311391BA6AF96A002A70
:109B0C0000D049420918149105992A46069B05F084
:109B1C0073FC302818D1B96A01204840B86207A8F4
:109B2C0000F024FA04463868B9684A1C00210FF08A
:109B3C00C3F90AE00949086889684A1C00242146CF
:109B4C000FF0BAF9E44306E0064C3868B9684A1CD1
:109B5C0000210FF0B1F9204617B0F0BDC8F1FF1F7E
:089B6C00FEFFFF7FFAFEFFFF80
:109B7400B0B584B000F0A8F800280BD4064DA96A4B
:109B84006C46204600F0F6F9A86A012141402046BF
:0C9B940000F0F0F904B0B0BDC8F1FF1FF4
:109BA00010B50E4C2068002808D0012181F31088E0
:109BB000206807F0A9FF002181F310883020205C85
:109BC000002802D0002005F09DFBFEF7DDFD0348D4
:109BD000002134220FF00EF910BDC046C8F1FF1F5E
:109BE00080B505F0EBFF002811D10220002105F01F
:109BF000D9FD04200C4905F0D5FD05200B4905F0E1
:109C0000D1FD0720012105F0CDFD05F095FD0DF0FA
:109C1000F8FF0EF004F84B20800000F009F80EF079
:109C200028F8002080BDC046020000234405004003
:109C300008B4024B9C4608BC6047C0466D1000202B
:109C400010B5081D0EF0B8F80146C007064809D047
:109C50000B46083B054C0022A34200D81046491C85
:109C600000D1104610BDC046F6FEFFFFF7FF0F0003
:109C700010B502280FD8441E012C0CD85918000129
:109C8000084C2018C468A14205D8816810461A46BD
:109C90000CF05EFA10BD002110461A460FF0AAF82B
:089CA00010BDC0465463010031
:109CA80080B5022906D80901054A511810220CF07E
:109CB8004BFA80BD002110220FF098F880BDC046F5
:049CC80054630100E0
:109CCC00F0B599B030279B48C05D002803D0002622
:109CDC00304619B0F0BDFEF74BFD012496492046E5
:109CEC0005F09AFC954804700FF044F805F060FFFD
:109CFC00079009AD00264022284631460FF074F833
:109D0C000694AC808E4809903046294605F016FB27
:109D1C00304605F0A9FA0169C069036C0846314662
:109D2C003246984787498E1C07990029D0D10028C4
:109D3C00CED4049705F0D2FB8348089083480427BF
:109D4C00002508AC39462A46234605F055FB8048C9
:109D5C0008907E480C30079039462A46234605F079
:109D6C004BFB7C480890794B1846E43805903946F3
:109D7C002A461D46234605F03FFB069847067648C3
:109D8C00046A0A340421002208AB284605F004FBBF
:109D9C000898384203D17048006A8442F2DA0424ED
:109DAC002846002508AB21462A4605F0F5FA6148FD
:109DBC00031D6A4821462A4605F0EEFA6748001D45
:109DCC005C4A13460833214614462A4605F0E4FA49
:109DDC006068401C022800D27AE7A068411C022966
:109DEC0000D275E72168002914D10830C010089002
:109DFC00012181F31088089807F02CFE20600021C7
:109E0C0081F310882068002845D0A1684A1C0021E5
:109E1C000FF052F800F0DEF8002800D588E0E0687A
:109E2C007D21CD002C46B03400224D4B214605F04F
:109E3C00E3FA00F0E9F800287AD400F02DF90028B4
:109E4C0076D4019402200890464C042103910026FC
:109E5C0008AB02932046324605F0CEFA06980890DD
:109E6C000834204603993246029B05F0C5FA3A485D
:109E7C00006A44190125002208AE3B4829463346A6
:109E8C0005F08AFA3078C00708D13348006A84425A
:109E9C00F0DA2C4E1CE72B48461C19E72A48089090
:109EAC0004210691002608AC28483246234605F0CA
:109EBC00A3FA27480890079806993246234605F0DE
:109ECC009BFA24480890059806993246234605F0DB
:109EDC0093FA2148046A0A340421002208AB1B4877
:109EEC0005F05AFA0898384203D11B48006A84429C
:109EFC00F2DA0421002208AB144805F04DFA00F008
:109F0C0069F8002814D40B48C0680024144B01993C
:109F1C00224605F071FA00F077F8002808D400F01A
:109F2C00BBF8002804D4049802490D542646CFE609
:109F3C000646CDE6C8F1FF1F00093D00330E002098
:109F4C00FF000006FEFEFFFF03005FA0F0ED00E047
:109F5C00010000010400FA05500E00201000001052
:0C9F6C004697010004E5014000E40140BC
:109F7800F8B5044614488269C3689A18036AD51864
:109F88002835002901D0C06A2D187D20C0000F494E
:109F9800096A0F181021002628463246234605F084
:109FA800FDF910280CD1206801210143094881429C
:109FB80007D10648006A8742ECDA0548861C00E0AB
:109FC800034E3046F8BDC046C8F1FF1F500E0020B2
:089FD800F9FEFFFFFFFFFF7F10
:109FE00070B50B4938220020B323DB000124A50300
:109FF00064078726F600CC600D614B6124338B61CA
:10A00000CE6108624A6288623836CE6270BDC04650
:04A01000C8F1FF1F75
:10A01400F0B58DB0204FF8687969BA6912183B6AB7
:10A02400D21800920818042100246B46224605F039
:10A03400E7F901AD30262846214632460EF0D8FE17
:10A044000B940C940098314622462B4605F0D8F91F
:10A05400124D30281DD1F86A00994018302100248F
:10A0640001AB224605F0CCF9302812D101200106BB
:10A0740010200EF049FEF868796909180D200EF0D9
:10A0840043FEF868811C0F200EF03EFE05F04CFAEA
:10A09400254628460DB0F0BDC8F1FF1FFAFEFFFFAC
:10A0A400F0B597B0234F386A0490786A0390BE6A7B
:10A0B400FC6AF8680290B86901900BA80025302268
:10A0C4000690294605920EF093FE1295119510956F
:10A0D4000F950E950D950820169017481590002E93
:10A0E40000D13446029801990818039909180919EE
:10A0F4000B91F9690C910499401800190146283113
:10A104001391BA6AF96A002A00D04942411814919D
:10A1140005992A46069B05F073F9302807D1B96AD8
:10A1240001204840B86207A8FFF724FF00E0034875
:10A1340017B0F0BDC8F1FF1FFEFFFF7FFAFEFFFF5F
:10A1440080B50848007801280AD107480068074903
:10A15400096A081A0649884202DB012000F00AF85D
:10A1640080BDC046250E0020E00B0020500E0020CC
:04A17400E9030000FB
:10A17800F8B500900D48066807270D4D0D4C30883E
:10A188002968081801214902B21CFEF7DBFF3619BD
:10A198007F1EF4D10848002404700098002804D0D9
:10A1A800024D286807F0ACFC2C60F8BDE40B0020D9
:0CA1B800E80B002002020000250E002031
:10A1C40010B58CB06C460021302220460EF010FEF3
:10A1D40001204102218205490B91C00303900448E8
:10A1E4000090204608F0C6F90CB010BDA46301002D
:04A1F400846301007F
:10A1F800F0B58BB0EA48002404701F20C0430590D6
:10A208001F30E8490860FF204600B51C284607F0C3
:10A2180023FC074640210494204601913A46FEF764
:10A2280077FF3C46163420460DF0BDFD0721090393
:10A2380003910F21C902029102281BD1387C022800
:10A2480018D1384611300DF0AEFD402812D1787B78
:10A2580040280FD138460B300DF0A5FDB11C8842BF
:10A2680008D1384613300DF09EFD0121C9038842FC
:10A2780000D1C8E038462430069007940024099499
:10A2880020460CF088FF384621462A460EF0AEFDDF
:10A29800E9203870F81CC44908220BF055FF3846ED
:10A2A8000B300121089149020EF088FD019C7C7356
:10A2B80038460E3038210EF081FD0A9602263E748B
:10A2C8003846113021460EF079FD3846133008998A
:10A2D800C9030EF073FDF820089078750798314689
:10A2E8000EF06CFD38461830FF2107910EF066FD20
:10A2F80038461A303F2100900EF060FD292006995B
:10A3080088708020087038462730A8490EF05AFD1A
:10A3180038462B30A6490B220BF016FF384636304C
:10A32800A4490A220BF010FF55200A99785478188E
:10A33800AA214170099C204629463A46FEF702FFA9
:10A34800384621462A460EF051FD37242E4630461F
:10A3580029463A46FEF7F6FE7619641EF7D1059CA3
:10A368001E34039E0997099F0798B870787008985B
:10A3780038700A98851C304629463A46FEF7E2FEB0
:10A388000021384606912A460EF030FD76193046EF
:10A3980029463A46FEF7D6FE7619641CE4D3099F8F
:10A3A8003846069C21462A460EF020FD80490B229D
:10A3B80038460BF0C9FE3C82FC817C73FC61282086
:10A3C800F8723846143021460EF0F8FC0098214601
:10A3D8000EF0F4FC784838837C82FC820298294687
:10A3E8003A46FEF7AFFE384621462A460EF0FEFCF6
:10A3F8003D2046020324304629463A46FEF7A2FE8F
:10A408007619641EF7D1384607F07AFB0124260333
:10A418006A49304607F060FBA5020A94E402002866
:10A428000894079556D007460398069631463A464B
:10A43800FEF76EFE09973F193C46203C049B1846E0
:10A448001D463978002901D0E52906D15B1E203444
:10A458006D1C2037402DF4D126E05F29F6D1F97A1A
:10A468003F260A4632400F2AF0D012221140022914
:10A47800ECD1798B0029E9D00998049300F08CF984
:10A48800049BE5213970002D0A98DFD01846224632
:10A49800D37A33400F2B04D11170059BD218401C7E
:10A4A800F6D30A98049BD1E70028079D099E0DD092
:10A4B800701931462A460BF047FE039C20460CF0E3
:10A4C8006FFE204606993246FEF73CFE304607F0FE
:10A4D80017FB089C61204001394907F0FDFA002864
:10A4E8002CD00646039829463246FEF711FE0A96F6
:10A4F8007619029821463246FEF70AFE0996203E52
:10A50800019C35462020305C2036E52811D00028F3
:10A5180011D0F07A1221014012290AD13F27384080
:10A528000F2806D00822304626490BF063FE002883
:10A5380006D0641EE5D10A9807F0E2FA0BB0F0BD28
:10A54800688F0028F7D0698F002902D00A9800F098
:10A55800F9F8E5203070E97A39400F29059B08D1D0
:10A5680028705919CA7A3A400B315D1815350F2AE7
:10A57800F6D0039D28460CF013FE2846079C21467A
:10A588000A9D2A46FEF7DEFD1D20800221462A4646
:10A59800FEF7D8FD02980899099AFEF7D3FDCAE795
:10A5A800260E0020EC0B0020E0950100DEBC9A0886
:10A5B800629C010087920100724500007E940100B0
:08A5C800E9950100FE95010078
:10A5D000F8B51C4615460E460A480078012802D1F7
:10A5E0000020FFF7C9FD76020120470230463946B8
:10A5F0002A46FEF791FDED19F619641EF6D10020EA
:08A60000F8BDC046250E002044
:10A60800F0B585B015464A023F29049206D842485B
:10A6180000210170C8433F49086014E008464038EB
:10A628008009801C3B4A1368834202D13A4801786A
:10A6380006E010603F200140481E81413648017005
:10A648000029049A4AD0364E164036480078012828
:10A6580013D135480068B0420BD13448006807214F
:10A66800334A049C0388F318A3424CD08018491E2F
:10A67800F8D10020FFF77CFD049A2C4C2768002FA6
:10A6880008D12C482C4907F027FA049A074620607D
:10A69800002831D003950120019044020825029634
:10A6A800B2420BD00720400230403880BA1C3046F6
:10A6B8002146FEF72DFD049A1D483F1836196D1ED8
:10A6C800EED11949029808601649019B0B7015468E
:10A6D8000CF066FD28462146039A0BE00F4810400F
:10A6E800824203D110460CF056FD049A0120410223
:10A6F80010462A46FEF726FD1048006A10490860F1
:10A70800002005B0F0BD801C01214A0229460BF04B
:10A718001BFDF1E7EC0B0020260E00200080FFFF58
:10A7280000F0FFFF250E0020E80B0020E40B0020BE
:10A73800020200000E0E00006E9C0100500E002068
:04A74800E00B002002
:10A74C00F8B50322920200908518CF03104C3819EB
:10A75C00403020212A46FEF7D9FC2878E52813D072
:10A76C00002813D0E87A3F2101400F290CD06E8BC2
:10A77C00002E09D0C00603D500983146FFF7E0FF44
:10A78C000098314600F006F82034E0D1F8BDC04600
:04A79C000080FFFF3B
:10A7A000F8B50D4600900C246C43E00800990E1893
:10A7B00030460DF0FCFA05460427274030460DF0E0
:10A7C000F6FA074C08342146B940884381B2304636
:10A7D0000EF0F8FAFD40254001488542E3D9F8BD66
:04A7E000F70F00006F
:10A7E40002480068106001207047C046F00B00204A
:10A7F40002480068106001207047C046F00B00203A
:10A80400F0B58DB0544805F051FF402005F054FFD9
:10A81400022005F057FF514805F01EFF504805F08F
:10A8240021FF092081014F4C20680291401800212A
:10A8340060220D460EF0DCFA3320000121680A582C
:10A84400002A05D5501C6ED0FF20C04382426ADD29
:10A854002C4615204001049008186C222F462946E6
:10A864000EF0C6FA2E46019506A83146FFF71AFAED
:10A8740006984049884205D03F4988422AD000289A
:10A884003BD13FE0059407980EF0A6FA07461D2831
:10A8940000D31D27242403956C43324D28680019E6
:10A8A4000499401807993A460BF050FC2868039D18
:10A8B4000119049A89180022CA55059C2301C0185D
:10A8C400029BC150C01842600E6209998160641CE9
:10A8D4006D1C12E0059407980EF07EFA07460B28CB
:10A8E40000D30B2707990AAC20463A460BF02EFCFE
:10A8F4000020E05501200190059C052C02DC761C0B
:10A90400032DB1DB0198002801D00AA800E01B4800
:10A914000DF0F3F91348006802994018214605F038
:10A92400A7FE0DB0F0BD029809180F4808600F4B40
:10A934001C685868944202D008330028F8D10028D3
:10A9440000D10B4848600EF047FA4921CA00054976
:10A954000968885001247CE74555000085A900005A
:10A96400B9A90000F00B00200C960100B4630100AB
:10A97400B49401000177755303777553A0940100D3
:10A98400B0B51446024615204001094D2D6828181B
:10A994001B680325834204D06D1E2430002DF9D199
:10A9A40003E0006A2346FFF761F90020B0BDC0460A
:04A9B400F00B002084
:10A9B800F0B585B00E460546CD20800036490C68B6
:10A9C80021580027002963D10396002E03D02118AF
:10A9D800097C00295CD001900292002B25D01968CF
:10A9E8000A78002A2846039B2B4E26D0083104AF4C
:10A9F800032238460BF0A8FB0020F87004A9095C74
:10AA0800202902D104A900220A54401C0328F5D1A8
:10AA18000027224EF05904A90DF0D5F9002808D0D6
:10AA28003F1D242FF6D1002732E02846039B1A4EFB
:10AA380003E0194E34682846039B0D21890101253E
:10AA48006550174A174911601946029A06F0CEFA5E
:10AA5800CB218900144A126A33685A5059180027C2
:10AA68004F61002804D4087E0D76474247410FE025
:10AA780006F036FD3168019A8918002801D00D606A
:10AA880002E00868002803D0087C002800D10D7473
:10AA9800384605B0F0BDC046F00B00204464010004
:0CAAA800840C002038630100500E0020D8
:10AAB4000146064A136850688B4202D008320028C7
:10AAC400F8D1002800D102487047C046B4630100A1
:04AAD400B494010035
:10AAD800F8B5264D2868002846D0CF21890040586F
:10AAE800002841D009F0D0FB0321014002293BD1C5
:10AAF8000DF0DFF96720C600286882596521C90072
:10AB080040181B49096A002A01D101610A468B1ABB
:10AB18000A2B29DB037F002B26D08369002B23D146
:10AB28004368CB1A7D24E400A3421DDB521A036854
:10AB3800D218026001610068002815DC06F0AAFC42
:10AB48003320070106F0CCFC2968C85109F062FCE3
:10AB580006F0CCFC00F00EF820460BF03BFA08F0AB
:10AB68002DFF286800218151F8BDC046F00B002058
:04AB7800500E00205B
:10AB7C0080B56520C0000549096864220A50081890
:10AB8C0000210177C16006F07FF880BDF00B00203A
:10AB9C00F0B593B06520C6003546203522492846CD
:10ABAC0006F098FF00283DD0044605960026314655
:10ABBC002A460BF025FB1D480460402002900090B3
:10ABCC00012702210391384604973246334608F098
:10ABDC0033FE12AD2870029800907F02E3193046C4
:10ABEC000399324608F028FE6870284607F042FCAC
:10ABFC0006F04AF806AD3022284631460EF0F4F83D
:10AC0C002F820B4811900B4809900B480690284650
:10AC1C0007F0ACFCFFF7D0FA64200599605060187F
:10AC2C000499416113B0F0BDA6940100F00B002013
:0CAC3C0034640100455500001464010060
:10AC480070B50C4605461C267543FFF793FF05486B
:10AC580000684019C32189004018214632460BF08C
:08AC680073FA70BDF00B00202F
:10AC70001C224243054800688018C5229200825871
:10AC80000A606322D200805A88807047F00B00204F
:10AC900010B50846012181F310886521C900064BD3
:10ACA0001B6864245C50002181F31088114605F074
:0CACB00011FDC00F10BDC046F00B0020CD
:10ACBC0010B50846012181F310886521C900064BA7
:10ACCC001B6864245C50002181F31088114605F048
:0CACDC00A1FEC00F10BDC046F00B002010
:10ACE800F0B5A3B0029315460F46064603A81449CB
:10ACF80080220BF029FAB46C002D04D0029880470A
:10AD080040190190FFE7306C811C3164215AC80654
:10AD1800400E03AA12583046904700280DD1002F44
:10AD280002D07F1E01D107E00027002DEBD002984A
:10AD380080470199081AE6D5002023B0F0BDC04627
:04AD48006C64010036
:10AD4C0010B5044688081C220240E06B8218E263AE
:10AD5C000A0607D4490A226D8A4213D98A00A16CCB
:10AD6C00E36C09E0226C911C216401218A43A16CE3
:10AD7C008A5AD200064B1B689A58081890472060D4
:10AD8C00002010BD206C801E2064022010BDC04627
:04AD9C004868010002
:10ADA00080B502480EF026FA80BDC046F0FFFF1FB6
:10ADB00080B502480BF01EF880BDC046F0FFFF1FB3
:10ADC00080B502480AF084FC80BDC046880B002094
:10ADD00010B584B00A480AF0D9FF0A480224214677
:10ADE0000AF05CFC02941920800101900649009150
:10ADF000081806490322064B0BF0A0F804B010BD5A
:10AE0000F0FFFF1F880B002000F3FF1FC992010015
:04AE100015AE00007B
:10AE14000F4C20460AF0ECFF01F048FE064600F015
:10AE24001BF807460DF0ACFFFFF754FEFDF7DEFC00
:10AE3400054620460EF0DCF9002EEAD0002FE8D0BB
:10AE4400002DE6D0012103480AF066FCE1E7C04684
:08AE5400F0FFFF1F880B002036
:10AE5C00F0B589B009F016FA03210140012402294A
:10AE6C0070D13A48006800286CD039480068411C01
:10AE7C0068D038490B68384A156AEB1A834261DB93
:10AE8C00126A121A0A6035490A78012A03D1002283
:10AE9C000A70002804D03248007801280AD051E00A
:10AEAC003048016830480068002204F0F5FE2C4858
:10AEBC00012101702D4E31680024E543002906D193
:10AECC002B4805F0CFF80146306000280FD0284FF2
:10AEDC003A68284800682B4607F016F8002806D474
:10AEEC003460386824490A681018086001E0224868
:10AEFC00006800280AD01F48006807F013F80646BF
:10AF0C001D4F3868801B05F097F83E6005F088F8F7
:10AF1C000246202800DB2022002A13D0154E306870
:10AF2C0001A92B4606F0E4FF01280BDB014601A822
:10AF3C0004F0D0FF05F074F80246202800DB202234
:10AF4C00002AECD1204609B0F0BDC046F40B00201D
:10AF5C00F80B0020FC0B0020500E0020B40C00203D
:10AF6C00B80C0020040C0020000C0020080C002061
:0CAF7C000C0C0020100C0020140C002015
:10AF8800F0B585B004A8012103F02AF903A804212B
:10AF980003F026F90398083006F05EFD0446022007
:10AFA800C6430399002C17D0204603F019F904A8CA
:10AFB80000780025042848D8784400794000874460
:10AFC80002122E343B0020460CF0F2FE0146201DF2
:10AFD80004F082FF064638E0084603F0F5F9761CCF
:10AFE800002501AC31E020460CF0E2FE0746204681
:10AFF80006F086FD00970837384606F02DFD01ACAF
:10B00800002837D007460830009904F0D7FF0546D6
:10B018001A48006A1A49086000263C4615E020468E
:10B028000CF0C6FE04F048FF04E020460CF0C0FE19
:10B0380011490860002507E020460CF0B9FE0025FC
:10B0480029462A4604F02AFE2E46204631460DF0AF
:10B05800B9FE201D29460DF0B5FE083520462946C3
:10B0680003F0DAF801A8844202D0204606F048FD31
:10B0780005B0F0BD761CE8E7F80B0020500E002064
:04B08800FC0B00209D
:10B08C00F0B587B00DF010F8012141402C4C216037
:10B09C0051D007F0EDF8206800284CD058202949F1
:10B0AC0006F018FD002846D004464C3005900025CB
:10B0BC000C26294632460BF0A3F82046403004906B
:10B0CC00294632460BF09CF840200290009001205B
:10B0DC000390022631462A462B4608F0ADFB06AFFC
:10B0EC00387002980090284631462A46234608F0CC
:10B0FC00A3FB787000950321082203982B4608F0D7
:10B10C009BFBB870384606F017FF0F4C20600F49B8
:10B11C0006F0DEFE20680E4906F0E2FE78780D4C53
:10B12C00049922462B4609F011F8387805992246E5
:10B13C002B4609F00BF808480021016007B0F0BD60
:10B14C00F40B0020FA940100100C002069B10000EF
:0CB15C00DF72010005820100F80B0020EA
:10B168000168084A1160084901220A7041798A1E5B
:10B1780050425041012901D0000200E0034804492F
:10B1880008607047000C0020B40C0020000101008A
:04B19800040C002083
:10B19C00F0B5B1B0044620AD0221284603F01EF8EC
:10B1AC00298810A803F01AF82888042804D310A8BA
:10B1BC000CF0FCFD074600E0104F21AE00254022AC
:10B1CC00304629460DF010FE35730121B1800C4834
:10B1DC00289068462590219700F0D6F80948201849
:10B1EC00643800788000084909583046884725980B
:10B1FC00294600F0C9F831B0F0BDC046FF0000038D
:0CB20C00EC640100C29C010050650100D0
:10B21800F0B58DB007460020C643702A01D23046EB
:10B22800A1E014460D4678690390B869069000219C
:10B238007022284604910DF0D9FD39684B48002941
:10B24800024600D00A464A494A4B8A42194600D06B
:10B2580049490594824200D00B462C465434387B29
:10B268000290787B010601920DD5012161760905CE
:10B27800C2030A40079307235B0500051840079B94
:10B2880080184840E865B87B411E1F2901D28640D6
:10B29800F343069E042E079311D3039E30460CF009
:10B2A80087FD0146A865371D6F6038460CF040FBE6
:10B2B800A86DC1007818069A511A0E1F00E003986D
:10B2C800029A042E01D8314600E0711F1206069238
:10B2D80000290CD0042E00D9401D0CF069FD01276F
:10B2E800074002D0254908400690049E01E0049ECC
:10B2F80037460120049000020CF09DFD0521617085
:10B3080020701F481F49079A2A66069A6A661E4ACD
:10B31800E9602946103145C1EE6127760D20020209
:10B32800002F1146304600D13946A182002F01D0A6
:10B33800103200E01022E282AD60059C703C12D011
:10B348007021284606F0ECFB08AE00211422304696
:10B358000DF04CFD04980A9001980990304602F0CF
:10B3680057FA286020460DB0F0BDC046FF00000324
:10B37800FF00000EFF0F0000FF03000000F0FFFFBA
:0CB3880065D60000E1D50000D9D6000019
:10B3940070B582B00468A66C002913D0F16A204607
:10B3A4008847B16920468847104800681049884298
:10B3B4001AD2B368012501AA204629469847019A62
:10B3C400AA430CE009480068094988420CD2B368D2
:10B3D400012501AA204629469847019A2A43019249
:10B3E400336920462946984702B070BD6C0C002092
:04B3F400A6AE000001
:10B3F8007F2909DD8039112915D8012088400C4A98
:10B4080010420AD00B487047084802290CD3042977
:10B4180007D0082907D126307047002903D11F20FB
:10B4280070470120704700207047C0461100008017
:08B4380034FC0300012F008029
:10B4400000200A21044A535A002B00D0401C24310A
:0CB450009A29F8D17047C04684080020FB
:10B45C00F8B53E4C2068401C20600A2873D13C484B
:10B46C000168491C01600127384602F02BFD0026BB
:10B47C00266039480078002808D036480078002823
:10B48C0004D13648006A3649884201DC0BF079FE5B
:10B49C00344D2C68012C23DB09D1344A1068411C33
:10B4AC001160622803DC002002F0CEFD06E00025CE
:10B4BC00284602F0B7FD2D4805602A4D2C488442E1
:10B4CC0000D02746781C28602A498F4219DB64215A
:10B4DC000DF0BCFC002811D0002002F0A3FD10E000
:10B4EC00002C0ED5002002F0AFFD2868401E28600D
:10B4FC001D49884205D1FDF779F802E0002002F0E1
:10B50C00A3FDFDF781F81C490A681C4B98420BD32C
:10B51C001B48824230460EDC002A02D14868401C8F
:10B52C0048600A32104606E0002A304603D04868CC
:10B53C00401C48603046086012480168491C0A29C2
:10B54C0000D00E46066002F053FDF8BD180C00202A
:10B55C007C0C0020340E0020350E0020500E0020F4
:10B56C00BFD40100780C00200CFEFFFF200C002043
:10B57C00FFFFFF7FB2020000680B00204C040000AC
:08B58C00FF5B26051C0C0020EA
:10B5940070B50446194D2878002806D01D2C15D303
:10B5A40060085C2811D80BF09AFE2046C738122890
:10B5B4001ED8012631468140114A114211D0124849
:10B5C4000078124904F02CF82E706334E0B2800045
:10B5D4000F490858804702F0A7FF0E4800F01CF8F6
:10B5E40070BD084A114205D1122801D10026EBE7AB
:10B5F400052CD3D101202870D0E7C046360E002098
:10B60400C0C1000001000200330E002040420F00C0
:08B6140078650100C027090060
:10B61C0010B50C4C0A340C490A6A00212388002B03
:10B62C0004D00223E358D31A834204DA2434491C8D
:10B63C000429F3D110BD084603F05EFE00202080E3
:0CB64C0010BDC04684080020500E0020F5
:10B65800F8B5184D1C350821C94300244A00AB5AD7
:10B66800834206D02435641C042CF7D108310C46DB
:10B678001DE00026AE5288004719386A002803D01A
:10B68800203706F03DFA3E602868002802D006F010
:10B6980037FA2E60204603F031FEFFF7CDFE002872
:10B6A80005D1FCF7C7FF0448067002F049FF2046A1
:0CB6B800F8BDC04684080020360E0020BB
:10B6C40080B504200DF006FA03480DF003FA0120BA
:0CB6D400C0020DF0FFF980BDE32E000065
:10B6E00010B582B001AC0221204602F07DFD218818
:10B6F0000648814202D101A8002101807D20C000BE
:10B70000484303F0C5FF02B010BDC046FFFF000074
:10B71000F0B59FB00BAD01242846214602F064FD30
:10B7200009A80426314602F05FFD08A8314602F060
:10B730005BFD07A8214602F057FD06A8214602F04E
:10B7400053FD0AA8022102F04FFD2878652810D089
:10B7500064285ED10AA8008800280FD08F21C94331
:10B76000434A53189A241C5B84424ED02431F8D1AA
:10B770004FE00AA80088FFF76FFF4AE001943E48B7
:10B7800007883B4E7F1C0A21725ABBB29A42F9D0FD
:10B7900024319A29F8D10AA90F80078007A80278D6
:10B7A00006A80078039009980290089B002504954C
:10B7B0000095284634186189002911D024306D1C69
:10B7C0009028F7D12D4814461D46FFF727FF2B463A
:10B7D00022460498002801980490009DE9D018E0C2
:10B7E0000299315067810398607222726360214828
:10B7F000006AE0600CA80CF001F90C980D9920612A
:10B800006161284601F086F903E01A48006A9C212C
:10B8100058500CA805900AA8018805AC20460CF0E9
:10B82000B4FA0425204629460CF0AFFA1021204630
:10B830000CF0ABFA204629460CF0A7FA0024059834
:10B840000B4D291910220AF083FC05981030059041
:10B850002434902CF5D1FCF7DDFE014605A80CF050
:10B860009BFA0CA84C2102F0DBFC1FB0F0BDC046D7
:10B8700084080020500E0020B60C00201027000085
:10B8800080B5054801210170044802F0B9FD044863
:10B890000CF0CDF880BDC046270E00206C0C0020B7
:04B8A0001047040049
:10B8A400B0B584B06846102102F09CFC0121C84365
:10B8B400009A7F2A0BD81346083B032B59D30B2A33
:10B8C40036D0052A3BD101980DF024F950E0D30974
:10B8D400022B0CD881235B009A4235D0FF2302331C
:10B8E4009A4242D009028A4243D127483EE00321CA
:10B8F400CC01214680318A423BD2611C8A4212D15A
:10B904001E490A316A46138900220D889D4204D0DB
:10B914002431521C042AF8D1421C0199104601F02A
:10B9240011F90020009AA11C8A4222D114481DE07A
:10B93400019A012A1DD115480170084619E00199A0
:10B9440010460BF027FC14E00C4A0A3269460B89B6
:10B95400002114889C4204D02432491C0429F8D1C3
:10B96400411C084601F0FCF802E006480199016018
:10B9740000200CF05AF804B0B0BDC0468408002082
:10B98400240C0020740C0020700C0020BC0C00203F
:10B99400F0B599B001277D032549284606F09EF8A5
:10B9A40004460020C643002C27D0009600262046DB
:10B9B40031462A460DF03CF83F022046394602F053
:10B9C40011FC18A8042102F00DFC16A8082102F0AD
:10B9D40009FC20463946324602F062FA1899884238
:10B9E40006D1144816A908220CF004FA00280ED037
:10B9F400009D204606F086F804E00C35284602F047
:10BA0400E5FC354628460CF010F819B0F0BD01A845
:10BA14000CF0AEFC204629460DF032F8054600280D
:10BA240000DA009D044801780229E2D00670E0E7BC
:0CBA340018950100E29C0100320E002079
:10BA400070B584B0012004021A49204606F048F877
:10BA5000002824D00546214602F0C6FB03A8042195
:10BA600002F0C2FB01A8082102F0BEFB0026284616
:10BA70002146324602F016FAF643039988420CD169
:10BA80000D4801A908220CF0B7F9002805D1284675
:10BA900021460CF089FC002807DA304605E00C341A
:10BAA000204602F095FC0020C0430BF0C0FF04B01C
:0CBAB00070BDC046D0920100E29C010075
:10BABC00F0B5D9B058AC01252046294602F08EFBD2
:10BACC0057A802F097FC2478032C17D8A00001A1EA
:10BADC0008588746F1BA000015BB0000F1BA000007
:10BAEC0085BB000002AE08273046394602F076FBD3
:10BAFC002802002C019072D0044671E0579800285F
:10BB0C0000D1ADE00C30ACE0579908460C306A031C
:10BB1C00914200D09FE07E4905F0DCFF002800D167
:10BB2C00A9E0044657990C3102F058FB57990025AF
:10BB3C0020462A4602F0B0F90746579820180CF018
:10BB4C0035F9EE43874215D157982018011D6F48DF
:10BB5C0008220CF04BF900280CD102A80CF004FCC4
:10BB6C00579920460CF088FF06466A48017802294E
:10BB7C0000D0057030462EE0579908460C302A024A
:10BB8C00914268D1604905F0A5FF04460020C543E9
:10BB9C0057990C31002C00D1AFE0204602F01EFB6F
:10BBAC0057990022204602F077F90646579820183C
:10BBBC000CF0FCF886420DD157982018011D534803
:10BBCC0008220CF013F9002804D1579920460CF0E8
:10BBDC00E5FB054628460BF024FF204638E06C03B5
:10BBEC004A4831463A460CF001F9002835D148490B
:10BBFC00204605F06FFF064620460BF012FF002E84
:10BC0C00019F00D0274617AD002E00D035460026E8
:10BC1C000197A74200D3274658A80078002805D0E2
:10BC2C00284631463A460BF0B0FE04E02846314631
:10BC3C003A460CF0F9FE2846394602F0EBFAE41BC2
:10BC4C00BE19002C019FE4D117A8854211D02846BB
:10BC5C0005F054FF0DE002F0B5FB0020C04306E0F8
:10BC6C000820579002F0AEFB0020C043401E0BF0A2
:10BC7C00D8FE59B0F0BD02A80CF076FB0BF080FE9C
:10BC8C00280201900024579E25460198864200D335
:10BC9C00019E17AF3846314602F0A0FA38463146BD
:10BCAC00224602F0F9F8044638462946324602F09C
:10BCBC003BF95798801B5790751900280646E4D11C
:10BCCC0017AD0C21284602F089FA28460CF06EF8C4
:10BCDC00A04207D117A8011D0C4808220CF086F8C9
:10BCEC0000280FD00BF04CFE0020C04309490A7805
:10BCFC00022ABCD000220A70B9E7084602F062FBA7
:10BD0C002846B4E70020F1E75A960100E29C0100B6
:08BD1C0041960100320E0020E7
:10BD240010B582B00020C04300F0F2FE01AC032144
:10BD3400204602F057FA2078242141430348401852
:10BD4400617800F0A3FF02B010BDC0468408002053
:10BD5400F0B583B002AD01242846214602F042FA30
:10BD64002878062800D986E0784400794000874482
:10BD740003078282821C520005200BF056FE7AE0F3
:10BD840005F0EAFD0BF043FE05F0ECFD0BF03FFE81
:10BD940005F034FE01200CF03BFB0BF038FE0020D4
:10BDA4000CF036FB05F032FE65E0374F38680028AA
:10BDB40006D132483249016005F06EFB05F098FB6C
:10BDC40001A802F01BFB64023049204605F086FE00
:10BDD400019E002834D00546A64200D326462846B4
:10BDE400314602F0FFF927480068002808D1396875
:10BDF4002846324605F0FCF8002801D521490860A0
:10BE04003868801938600198861B0196E4D1284669
:10BE140005F078FE2FE019481949016005F03CFB54
:10BE240005F060FB044605F063FB164E30680028FD
:10BE340000D4204600280ED400200BF0F6FD16E0B6
:10BE4400304602F0C3FA0F480168002913D10021DB
:10BE5400C94301600FE0FEF72BFE04460CF0BCFF63
:10BE640005460BF0E2FD2046294602F0D7F90020F2
:10BE740030600549086003B0F0BDC046840C002062
:10BE8400386301002C0C0020280C00202A950100A6
:10BE9400F0B5A3B002A8042102F0A4F90298002886
:10BEA40045D026490978019100242646C10738D097
:10BEB4000D2E01D0304600E00220FCF751FC05466F
:10BEC400401C27D01C2E27D801273846B0401C49D7
:10BED400084221D00D2E13D01A48007802280FD022
:10BEE400002806D18021042217480CF0A1FD154832
:10BEF400077015480068002802D4400040102D1A2D
:10BF04000198002808D17D20C10028460BF088FF45
:10BF1400054601E00020C543A00003A90D50641CA0
:10BF2400029840080290761C0028BFD100E000244B
:10BF3400A10003A802F072F923B0F0BDBC0C0020EC
:0CBF44001C200018320E0020680C0020A9
:10BF500070B5A2B001A8042102F046F901990020B1
:10BF6000002914D00D4A0346CC0709D0032B01D871
:10BF7000146801E00024E443850002AE7451401CC3
:10BF8000121D49085B1C0029EED10021019181009E
:10BF900002A802F045F922B070BDC046680B00202F
:10BFA000F0B583B002A8012102F01EF901A8042413
:10BFB000214602F019F96846214602F015F90028D9
:10BFC00040D40198009C20433CD005F029FD8442D8
:10BFD00002D905F025FD04461C49204605F080FDE8
:10BFE000002831D00546AA2122460CF003FF009F0D
:10BFF000A7423E4600D3264602A8007864280CD00B
:10C00000652821D102F026FA0028FBD1019828608A
:10C010002846314602F0B0F905E02846314602F0E4
:10C02000E3F800280BD4BF1BE2D102A800786528F2
:10C0300001D10CF05BFD0198401E0190D7D128463C
:10C0400005F062FD03B0F0BD0BF04BF93C9501002B
:10C0500080B582B06846012102F0C6F80190002840
:10C0600011D168460078FE2803D0FF2804D10220B1
:10C0700004E00648007801E001F01CFF019001A8EF
:10C08000042102F0CDF802B080BDC046330E00207E
:10C0900080B50448042102F0C3F80020014601F0F5
:08C0A00017FF80BD04670100D9
:10C0A80010B582B001A80124214602F099F868462B
:10C0B800214602F095F8022002F086F9002813D1F3
:10C0C8006846007801990902081880B2FF210231F8
:10C0D800884205D00549884202D00549884200D1E6
:10C0E800044C20460BF09FFC02B010BD0106000076
:08C0F80001030000FF05000038
:10C1000010B582B001AC0421204602F06DF86088C1
:10C1100040BAFF210231884205D00649884202D048
:10C120000549884203D101A80078FFF737F802B02B
:0CC1300010BDC046010600000103000025
:10C13C00B0B588B06C460021202520462A460CF06C
:10C14C0053FE0A4920460CF03BFEA12020726220CF
:10C15C00E0719120A0717C2060711C202071204620
:10C16C00294602F057F808B0B0BDC046335A6AB839
:10C17C00F0B583B002AC0321204602F02FF82778EB
:10C18C006078A17809020D186C1C2F49204605F027
:10C19C00A1FC0190002819D00F20384001218140CA
:10C1AC004E083806000F1BD0019F3846294602F076
:10C1BC0015F8002E03D06E43304600F047F80020EF
:10C1CC0078553846214602F025F838E0284602F02A
:10C1DC00F9F828460BF020FC06200CF06DFC31E041
:10C1EC000198294602F006F8002402F00BF8291AEF
:10C1FC000F1B002801D0FF2FF7DDFF2F01DC394684
:10C20C0002E03F2239469143002800D00F46002E11
:10C21C0004D030467843800A09F0DAFE0198001900
:10C22C003C19AC4203D0394602F0A0F8DDE70021FE
:10C23C00C155791C02F09AF80CF052FC019F38465B
:10C24C0005F05CFC03B0F0BD6F96010008B4024B26
:0CC25C009C4608BC6047C04671100020E2
:10C26800F0B5C5B044A802F0C7F843A802F0C4F876
:10C2780043981B490B68591C02292CD3449E01463C
:10C28800314303220A4026D1012109020091009975
:10C298008842044600D3009C001B439003AF0194DE
:10C2A800029330460BF084FD05460299414038461A
:10C2B8000CF088FD0B484540241F361D3F1D002CFF
:10C2C8002B46EDD103A8019901F0A6FF4398002859
:10C2D8002B46DCD101E00BF0A1FB45B0F0BDC04618
:08C2E800240C0020A5A5A5A56A
:10C2F000F0B589B0054607A800240470E04301901A
:10C3000000F008FC0595CD2D07D108AD0221284687
:10C3100001F06AFF2878012106E008AD03212846D4
:10C3200001F062FF6878022108AA51180978090211
:10C330000818C61DF7087D00681C484905F0D0FBA9
:10C340000028029064D0C119054606910846394676
:10C3500001F04AFF2846394601F052FF0720B0435A
:10C36000049001F055FF391A0E1B002801D0FF2E52
:10C37000F7DDFF2E01DC314602E03F2231469143DA
:10C38000002800D00E46F500002801D104982D1A8F
:10C3900007A80078002807D006980019E91DCA10E0
:10C3A00000210CF027FD17E02D480078012810D15E
:10C3B00001982C49086003F05BF90298001906996E
:10C3C0000919294A1268526803920A462B46039DAE
:10C3D000A84707A800210170059DD52D14D0CF2DA9
:10C3E00031460DD13019B842314609D11F48007885
:10C3F0000028314604D00698001907998155711C10
:10C400000698001901F0B8FF3419BC42A9D10CE01C
:10C41000284601F0DDFF38460BF004FB07A8062193
:10C420000170012101F0FCFE059D114801780029F1
:10C4300001D107990170D52D0BD00CF057FBCF2DF2
:10C4400007D10A480078002803D107A800780CF02B
:10C4500039FB029805F058FB09B0F0BDDF920100EE
:10C46000330E0020600C002084100020270E0020D6
:04C47000280E002072
:10C47400F0B58DB004460BA8082101F0B3FE0020EE
:10C484000994074620630B9C0C98079085B205F02D
:10C49400C5FA85422E4600D3064601200003864293
:10C4A40002D9FF20000206403749304605F016FB4A
:10C4B400F943089000284ED03A46002D5AD00391F3
:10C4C4003248079901400791029528460496B042E4
:10C4D4000690074600D337460898394601F08EFE89
:10C4E400002505940A942E4601F090FE391A4C1B3F
:10C4F400002803D0402CF7D33F208443002E16D1CC
:10C50400089842190998C1698E6800920A992246CE
:10C51400079BB047A04201D0064600E000260A98D7
:10C5240020180A9003D30999086B401C0863651905
:10C53400BD42D9D1002E3A46069800D0039AC01BBA
:10C54400002A0BD4002E09D1059C14190028049E3E
:10C55400BDD1029A0BE028460A4602E0002A00D424
:10C56400039A002803D0144601F030FF22460898AD
:10C57400002804D00898144605F0C4FA2246104650
:10C584000BF053FA0DB0F0BD059301000000FFFF5E
:10C59400F0B597B005460BA8082101F023FE002052
:10C5A40028630C990B9F07918EB2112E09D3341D69
:10C5B40005F034FA844200D30446204605F04EFACE
:10C5C400231F002800D110230121069189028B42E8
:10C5D40001D8059302E033491940059130490DAA69
:10C5E400002800D0024607980840079003960A9254
:10C5F40004932D48129000201690149013920698DC
:10C6040040021590E869446812A8009201909E4285
:10C61400059A00D83246284639460992079BA04716
:10C62400044601281EDB3146311BE719089702D363
:10C63400286B401C28632F461698251A0E4600299D
:10C644000A9919D00818294601F094FE0CF04CFA06
:10C654000A9A099884423D46089F049BC9D00398CE
:10C66400841B02E01698361A02D030460BF0D8F933
:10C6740020460BF0DAF90BE0081903990CF0A4FB3F
:10C6840016980A990818291D01F074FE0CF02CFA6A
:10C694000A980DA9884201D005F034FA17B0F0BD0C
:0CC6A4000000FFFF00FEFFFF55740100C6
:10C6B00070B5044600290DD0094D286A4618206936
:10C6C000E169096A8847002808D1286A8642F6DAB3
:10C6D000002070BD2069E169096A884770BDC046C5
:04C6E000500E0020D8
:10C6E400F0B587B003930F460546848C0C9BDC4061
:10C6F400069219D0296A9442164600D82646059611
:10C704009E40384602913246049309F01FFD059875
:10C71400241A0BD00298811904988440286A22466E
:10C7240009F014FD049B03E0144606E0049B9C40BE
:10C73400AC84069A0598141ABF191648006A03991E
:10C7440040180290002C1DD02869E969896C059174
:10C7540003990091019300213A4604972F461D4600
:10C76400069B059EB0472B463D46049F069AC1177B
:10C774008843241A98403F180648006A0299814267
:10C78400E0DC00E00024342001212954EB84101B58
:08C7940007B0F0BD500E0020BB
:10C79C0070B586B0054604AE0821304601F01EFD8A
:10C7AC00F08831888900884200D80846001D05F0C1
:10C7BC0051F9F188002819D00446002902D02046EE
:10C7CC0001F00CFD04A8407901281AD000282CD1C6
:10C7DC0004A84388028802200090211D2846FFF7F8
:10C7EC007BFF014603908000051D21E0084601F007
:10C7FC00E9FD1548401E039003A8042101F00AFD31
:10C80C0020E0022129852869EA69956C04AA13881D
:10C81C00D688528800920191B108C91A8900621811
:10C82C000121A8470146039001E007490391042523
:10C83C0020460CF0C5FA2046294601F0EBFC2046B8
:0CC84C0005F05CF906B070BDFAFEFFFFBD
:10C85800B0B5002901D02D4900E00121002851D0B0
:10C868004368002B01D0022319438368002B01D0B1
:10C8780004231943C368002B01D008242143046909
:10C88800002C01D0102421434469002C01D020241D
:10C8980021438469002C01D040242143C469002C21
:10C8A80001D0802421430124056A002D01D02502EE
:10C8B8002943456A002D01D065022943856A002D68
:10C8C80001D0A5022943C56B002D01D025032943BA
:10C8D800002B01D063031943436D002B01D0A3043F
:10C8E8001943836D002B01D0E3041943836C002B9B
:10C8F80002D00923DB021943436C002B02D01046F7
:10C908009847014608460BF08EF8B0BD010000407C
:10C91800F0B595B005A80021402200910CF066FA08
:10C9280004A80124214601F05BFC03AD28462146FA
:10C9380001F056FC287800284DD005AD281D01903F
:10C948006F1D083502AC0121204601F049FC207812
:10C95800C01F03280CD8C04678440079400087449B
:10C96800010C101E03A8017805A801F04FFD0DE089
:10C9780003A8007801F028FD08E003A801780198D1
:10C9880002E003A80178384601F02AFC03AC012133
:10C99800204601F025FC20780028D3D11BE003AE07
:10C9A8003478082C00D308242846214601F018FCC6
:10C9B8003078061BEAD03046114905F08DF80A9008
:10C9C800002804D0314601F00BFC0B96DEE703A8E3
:10C9D8000078001BCEE704AC207805A902F0B0FC73
:10C9E800207802F043FC04460069002806D16069FB
:10C9F800002803D005F084F80098606115B0F0BDF8
:04CA0800F2920100A5
:10CA0C00F8B56D460221284601F0E8FB287803288A
:10CA1C0008D881011F4A5418E169002902D06E78A8
:10CA2C00142E02D901F00CFCF8BD25461C3524222D
:10CA3C00424319488018194A126AC2602069274675
:10CA4C00103700280CD1A069002802D0606900289A
:10CA5C0002D0204602F012FC38680028E4D0296885
:10CA6C0034220123A354CA6C002A0CD00121904714
:10CA7C00B0000B4909582046884738682968CA6CA9
:10CA8C0000219047F8BDB000054909582046884759
:10CA9C00F8BDC046C406002084080020500E0020BB
:04CAAC000867010016
:10CAB000F8B501200090134D0C26134A134F144C67
:10CAC0002869002818D03420285C002814D035208C
:10CAD000285C002810D19059C019216A88420BDDCA
:10CAE000E869016D002907D01446284688470028C8
:10CAF00000D100902246064C243640359C2EDFD1D2
:10CB00000098F8BDC406002084080020102700000B
:04CB1000500E0020A3
:10CB1400421C114600D30421824200D2002082012B
:10CB2400074B9A1834321346243B1B68002B01D060
:10CB3400002313704032401C8842F4DB7047C04627
:04CB4400C406002003
:10CB4800002807D48001044A10180269002A01D07D
:0CCB5800352281547047C046C4060020FE
:10CB640010B5800107490C18E069026E002A08D04C
:10CB7400206903219047002803D00146103420681F
:08CB8400884710BDC406002023
:10CB8C0010B582B004466846082101F027FB0098D6
:10CB9C00012805D1012001990143E162002000E048
:10CBAC0002480AF03EFF02B010BDC046FAFEFFFF7D
:10CBBC00F0B585B00191039003A804F0AFF9039987
:10CBCC000A78002A55D000200290C04300902C4EC9
:10CBDC00DF205F2A03D00240413A192A4BD8491C66
:10CBEC00029D4C5D2346303B224602406D1C5F2C5F
:10CBFC00F7D0413A0A2BF4D31A2AF2D30027F419AE
:10CC0C006068A84206D1F05903992A460BF0EEF859
:10CC1C00002805D00C37542FF1D1F419002700E06F
:10CC2C00012703984019039003A83D210AF07CFCCE
:10CC3C00002820D403A804A904F082F9002F05D001
:10CC4C00A268002A02D004980199904703A804F026
:10CC5C0065F903980078002500280DD003A83B2126
:10CC6C000AF062FC002806D403990A78002AAFD196
:10CC7C0002E0002500E0009D284605B0F0BDC0464E
:04CC8C005C670100E0
:10CC900080B5012903D88900014A5158884780BDD1
:04CCA000B067010078
:10CCA400F0B587B0044600260696C069002802D075
:10CCB40004F028FFE66105A8042101F093FA04F0CA
:10CCC400ADFE07462D4904F009FF054605998F423C
:10CCD40005D2084601F07AFBF04306903FE0029447
:10CCE400284601F07FFA03AC002107222046019177
:10CCF4000CF07EF828462146FFF75EFF00282AD470
:10CD04001F48381827D4092044012846019F394672
:10CD140022460CF06DF82846214604F003FF029CDD
:10CD2400E5615422284639460CF062F828465C3006
:10CD34006864686513480078002802D0072800D08A
:10CD4400114FAF6503A9012809D14879002806D1FC
:10CD540002F032FF03E00020C0430690029C002D45
:10CD640006D00698002803D5284604F0CBFEE661D9
:10CD740006A8042101F052FA07B0F0BD0A9D010093
:0CCD8400E0FEFFFF330E0020CC67010032
:10CD9000F0B58DB005460CA8042101F025FA04F089
:10CDA0003FFE514946181C243046214609F08CF9B3
:10CDB000002E00D501200C99884200D801460F466C
:10CDC0004C434A49204604F08BFE0646142002904C
:10CDD00000200190C0430590E869002869D07442A2
:10CDE0007441002E67D0856D002D64D002993C46B9
:10CDF000794371180391E96A099088470C98049661
:10CE00000895A04200D3204604460299414330468B
:10CE100001F0EAF901F01EFB0028FBD1002C3CD008
:10CE2000039F049E019806940790357CB07C0028EF
:10CE30001DD02F48046A707C002802D00898C3686F
:10CE400001E0089883680AAA0998294698470028AB
:10CE50001AD47168B2680A9B0B40934214D02448DC
:10CE6000006A001BF1688842E5DB05980CE0707CE5
:10CE7000002803D032680898436902E032680898B5
:10CE800003690998294698470A9903C70798401CDF
:10CE900000371436069CA042C6D3E100039801F087
:10CEA0006BFA0C98001B0C90049EAAD10BF01EFE8E
:10CEB00014E0744274410C990298484301F088FAD6
:10CEC00000200B9005980A900AA8082101F0A8F903
:10CED0000C98401E0C90F7D1002C02D1304604F083
:10CEE00013FE0DB0F0BDC04600FEFFFF35930100FC
:04CEF000500E0020C0
:10CEF400F8B5009105460068846C0A4928460BF091
:10CF040075FC064663682868032100229847074693
:10CF14003743636828680121009A98473843C0174B
:08CF2400F8BDC046F0ED00E08D
:10CF2C00F0B504466C34550325D46578002D01D03A
:10CF3C00C56D1CE003252D05466E9E4217D1866DEE
:10CF4C00002E0BD04568F7007D19083D2F688F42E5
:10CF5C000CD9083D761EF9D1154608E00168496BDD
:10CF6C000D4EB14203D10F210D0500E06D6801217A
:10CF7C0049070A402A43059D01684A60426E9A425D
:10CF8C0001D1006E00E005488860CB600120487438
:10CF9C000D6020780874F0BDFF00010EFF03000047
:10CFAC00F0B585B00668B46C019000F043F80290BF
:10CFBC0063680025304629462A469847074603945D
:10CFCC00636804AA30462946984702990F430743E1
:10CFDC0013D5019800F02EF80290039C636830463C
:10CFEC0029462A4698470746636804AA30462946CC
:10CFFC00984702990F43074318D4039C04980103E4
:10D00C0010D5636900250A4A30462946984763685B
:10D01C00304629462A469847636804AA3046294672
:10D02C00984704988003C00F05B0F0BDE843FBE7B8
:04D03C0003005FA0EE
:10D04000F0B587B06A21415A02910568AE6C436E13
:10D05000059300210691009101214A071049FFF72D
:10D0600065FFB06B03900496022428460C492246C3
:10D07000069B039FB84706900598029A02433369BE
:10D08000284621461446984706460498416A284691
:10D090008847AC6106980643F01707B0F0BDC0465C
:04D0A000F0ED00E0CF
:10D0A400F0B585B004460668B56C17490BF09EFBD5
:10D0B4006E200490205CC0001449471803956B69E6
:10D0C4000321029630463A469847204600F022F85B
:10D0D40002460498205C6E34002810D00C480740A7
:10D0E400039D6B6903210191029E304604923A46E6
:10D0F40098476B680022304601999847049A0020AB
:10D104002070104605B0F0BDF0ED00E003005FA014
:04D11400F3075FA01E
:10D11800F0B583B00568AE6C736803210022284619
:10D12800019298470C4F386A841C7368032102AA3D
:10D1380028469847002808D402A88078800707D492
:10D14800386AA042F1DD019803E00198C04300E08D
:0CD15800012003B0F0BDC046500E0020C6
:10D16400F0B583B00F4605460668B46C00F05CF871
:10D17400002846D4012007400097244928460BF094
:10D1840035FB636903271F223046394698472846F2
:10D19400FFF754FF6368002130460A4698476368E6
:10D1A40002AA304639469847636801AA3046394690
:10D1B40098470099C800164A871802980007C00FBC
:10D1C400814205D06369002130463A469847104AA7
:10D1D400901D07406369002130463A469847A16A8A
:10D1E400304688470B480068002801D000F014F846
:10D1F40028460BF00FFB0028009A04D46E216A54D1
:10D2040001E00020C04303B0F0BDC04630ED00E0B3
:10D2140003005FA0700C002008B4024B9C4608BCBD
:08D224006047C0466D100020B8
:10D22C0070B505460068406B0C49884210D12E46FB
:10D23C00083630460AF094FA002400280AD4304606
:10D24C000AF087FA0649284622460AF07CF902E0E1
:10D25C00002400E0E443204670BDC046FF00010EF0
:04D26C0050EF00E09F
:10D27000F8B504460568AE6CFFF7D8FF00281ED449
:10D28000114920460BF0B4FA7369104A0C32032797
:10D2900028463946984773690C4A0A322846394667
:10D2A00098472046FFF738FF314606464B69284627
:10D2B0003946064A984720460BF0AEFA01E00020B6
:10D2C000C6433046F8BDC046F0ED00E003005FA065
:10D2D000F0B589B01C4615460E460768B96C079133
:10D2E000FFF7AEFE0021C94300283DD4019104950B
:10D2F00005943D461E4F069503963278079C636958
:10D300000121284698476368002128460A46984725
:10D310003E6AC83620464368002408AD0698214678
:10D320002A469847A878C00704D1386AB0420798BF
:10D33000F1DD17E0079E736802210291069D2846E1
:10D3400022469847736828460299049E32469847B9
:10D350000598401E361D0496039E761C05900028F5
:10D36000CAD102E0019C00E00C46204609B0F0BDA5
:04D37000500E00203B
:10D37400F0B587B01C461746039101680491896C87
:10D384000591FFF75BFE0021C943002835D40091C5
:10D39400029401200504039E01973A68059C636981
:10D3A4000221049F38469847039632782A436369DA
:10D3B4000121384698476368002138460A46984751
:10D3C400104F3E6AC83605984368002406AA04989C
:10D3D400214698470698284203D1386AB042F2DDC4
:10D3E40009E00298401E019F3F1D039E761C029097
:10D3F4000028D1D102E0009C00E00C46204607B092
:08D40400F0BDC046500E0020EF
:10D40C00F0B589B00892079105460F210E9C26466F
:10D41C000E40201601402F68BA6C069215D00022DF
:10D42C00082939D3009207210840610B18220A40C1
:10D43C008018059303062846079D29462246FFF7C8
:10D44C006FFD0698046B03201EE005936B6E0F9A1C
:10D45C00786B134988420DD103920493A000089A6B
:10D46C0000D50122B2402846083007990BF04CFA3F
:10D47C00049B039A00922846079D29462246FFF7F3
:10D48C004FFD0698046B0020009601903846294603
:10D49C00089A059BA04700E0D04309B0F0BDC046F8
:04D4AC00FF00010E6E
:10D4B000F0B587B0069104460F210C9D2E460E4014
:10D4C0002816014027680397BF6C0497059317D06F
:10D4D0000292002308293FD3009307210840690BDB
:10D4E00018230B40C01803062046069C21462A46F6
:10D4F000FFF71CFD0498456B0320009601903AE06D
:10D50000636E012A2AD134490698884226D1022E18
:10D5100024D105980D460AF04FFC06902668B76C9A
:10D52000204629460BF064F90021CD43002828D17C
:10D530007B6907213046069A9847002824D4B96AA7
:10D54000304688470698400722D43B6803210022D2
:10D5500030469847012514E0DD4312E0002700978C
:10D5600002922046069C21462A46FFF7DFFC0498DB
:10D57000456B0096019703982146029A059BA847A0
:10D580000546284607B0F0BDF96930468847F8E7F8
:10D59000396A30468847022008F020FD3C460F4893
:10D5A000076A236803210022304698470125002896
:10D5B000E7D54B2000013F180848006AB842E0DC7C
:10D5C000642008F00BFD23680321002230469847B1
:10D5D0000028F1D4D5E7C0460CED00E0500E002045
:10D5E000F0B583B00A4606460568686B1B49884259
:10D5F00030D100270297AC6C1948011D30460192CA
:10D600003A4609F0A6FF304615490BF0F1F8636879
:10D610000326284631463A469847636802AA2846B8
:10D6200031469847019C267101252560029F3E40A6
:10D630001020B0400AF003FCE0713801400C401C9F
:10D640000AF0FDFB6071F804800D401C0AF0F7FB46
:10D650002574A071002003B0F0BDC046FF00010E8C
:04D6600080ED00E079
:10D66400F0B583B00468616B184A91422AD1A56C65
:10D67400174964310BF0BAF86B680327002620467B
:10D6840039463246984701956B6802AD20463946C3
:10D694002A4698472878800715D5019E7369012189
:10D6A40020460B4A984773680325002220462946E2
:10D6B4009847736802AA2046294698470298C003EF
:10D6C400C60F00E00026304603B0F0BDFF00010E97
:04D6D40014ED00E071
:10D6D800B0B50468646B094DAC420DD1049CA4003C
:10D6E8000919CC79A24089792024611A8B40134307
:10D6F80003491A4609F029FF0020B0BDFF00010EBA
:04D7080074EF00E0DA
:10D70C00002901D00020704700487047558901005E
:10D71C00F0B582B0009201910124012B03D0022BB1
:10D72C0003D1002209E0E20707E0436B124DAB4244
:10D73C0002D021231A0600E02206E30645682F01D9
:10D74C003B40A607A902314011431943A2063A40B7
:10D75C000A4363063B4013437340290305D5407CC1
:10D76C00002802D103208006834300980001019910
:0CD77C000843184302B0F0BDFF00010E8E
:10D78800F8B50C46054620202958CEB2FF2E04D005
:10D79800FF229143EA68914208D0001D3028F3D156
:10D7A800287C002804D0DF20000102E000202AE0C5
:10D7B800F020EA680243A86C0369022128469847CA
:10D7C80000200090A86CC36803266A4628463146A4
:10D7D80098470F214B03009A134001200704BB42CE
:10D7E80006D10A40511E042902D88900074A565812
:10D7F80020216A5CFF2A03D0091D3029F9D102E0F3
:10D80800EA6832436A502660F8BDC046B86701002E
:10D81800F8B50446264F3D68002D09D02946303119
:10D82800142220460AF0E4FA00283CD0ED6CF3E715
:10D8380004F0F2F80546C008222801D809F04DFD89
:10D848001C49284604F048F9002815D0064623202C
:10D85800C2003546002130460BF0C8FA2020FF21CF
:10D868002950001D3028FAD1A068072801D00028C7
:10D8780006D109F032FD09E009F02FFD002515E079
:10D888000D48A8645421284604F04AF93036142279
:10D898003046214608F058FCA86CC16A28468847DB
:10D8A8003868E8643D60286D401C28652846F8BD46
:0CD8B800300C00207C960100CC670100C1
:10D8C400B0B5016D491E016500D0B0BD0A490B68B1
:10D8D40000242246002B05D01D46543598421C4690
:10D8E4002B46F6D1002A01D04C321146C26C0A6094
:0CD8F40004F008F9B0BDC046300C002064
:10D90000F0B58BB008930691002A07D00546079220
:10D91000109E0127012E03D00A9703E000247FE028
:10D9200041480A90002E01D140480A901198029077
:10D93000002438462146324608F0F0FB09906A6818
:10D9400078070590E0430090079F019504920394A7
:10D95000AC682846069D29463246029B0AF096FF8F
:10D96000AC43F440611C8F42079700D30F460599E2
:10D97000049A0A4200D0079F00284ED4022E089C29
:10D980003D460FD10320089C20403D460AD1012F7F
:10D99000089C3D4606D90898394601F0E5FF002865
:10D9A00019D53AE02178002E0AD06078000241189B
:10D9B000012E05D0A07800044018E178090641182E
:10D9C0000A984143072001F0EDFE002805D409988C
:10D9D00024186D1EE6D1002501E001F0D1FE01F012
:10D9E000ABFE0320002101F053FF781B17D4039CEA
:10D9F0000419002D14D13846B040019D6A6805997C
:10DA00000A4202D10699091806910799CF1B089975
:10DA100009180891002F99D102E0009C00E004460B
:10DA200020460BB0F0BDC04601000100010101011C
:10DA3000F0B58DB01D4614460E46074609F055FF59
:10DA40003C20385C00280A9500D18AE0002008902C
:10DA50003A4637462646864D0A990D401398099056
:10DA6000129BF807079221D0002E1FD01069D169B0
:10DA70000C6B059500950999019101223946069391
:10DA8000A047002800D5F1E0341A012800D0DBE0DF
:10DA900004967E1C069B5B1CBE42079A03D2106B49
:10DAA000401C10630026059D0A9902E00496344646
:10DAB0003E46480000D5AEE00227022C059528D34B
:10DAC0003046384025D002971069D169096B03911F
:10DAD0000122154300950999019131461546069397
:10DAE000039FB847002800D5C0E04100641A012810
:10DAF00000D0A8E0B01C0390069B9B1CE843864224
:10DB0000079A02D3106B401C1063059D0A99029F6F
:10DB1000039E002953D4042C51D31069D169324695
:10DB20003E460F6B2E43009609990191A608039279
:10DB3000114632460693B847002800D596E081008A
:10DB4000671AB0427ED10320844303980619069BCE
:10DB50001B198642079A02D2106B401C1063059D68
:10DB60002EE00BA80021082208910BF043F90C9538
:10DB700038690B90B96B096800293A463746264642
:10DB800007D00BA8144688472246002800D062E739
:10DB90001069D169C969154688472A460128344663
:10DBA00056D1906B416801200890002900D152E7BE
:10DBB0000BA888472A460028344649D44BE7274615
:10DBC000022F27D31469D169086B0A9038460127C0
:10DBD00002973D4307460095099901914208204666
:10DBE00003963146164606930A9CA04700283DD46A
:10DBF00041007C1AB04226D1029887430398C61987
:10DC0000069BDB198642079A02D2106B401C1063F8
:10DC1000059D00E03C46002C11D01069D1690F6BC6
:10DC200000950999019131462246B84700281DD434
:10DC3000241A08980028049E079A09D115E00024A8
:10DC4000049E02E03C46049E079A089800280CD0E7
:10DC5000906B8168002903D00BA8154688472A4697
:10DC60001069D1694A6900219047301B0DB0F0BDA1
:04DC70000000FF3F72
:10DC7400F0B58BB01F4608920E46054609F033FEF8
:10DC84003C20285C002827D000200790834A3A4093
:10DC9400109BF0071ED0089800281BD00597286910
:10DCA400E9694C6B06920092012231461F46A04757
:10DCB400002800D5EDE008990C1A012800D0D8E01E
:10DCC400701C3B467B1CB0422CD2286B401C286342
:10DCD400002628E0089C28E009A800240822214600
:10DCE4000BF086F80A9728690990A96B096800293E
:10DCF40005D0079409A888470028C7D12869E9698D
:10DD0400C96988470128089C00D0B5E0A86B416820
:10DD1400012000290790B9D009A888470028089C49
:10DD2400B4D5A9E00646069A059F780000D592E08E
:10DD34000221022C069229D33046084026D00291B3
:10DD440005970127114639432869EA69526B039202
:10DD54000091314601973A460493039FB84700283F
:10DD640000D596E04100641A012800D081E0B01C7F
:10DD74000390049B9B1C0198C043864202D3286BEA
:10DD8400401C2863069A059F0299039E002F3AD4EB
:10DD9400042C38D30396002A16D1E869866B002E2A
:10DDA40012D00291286900210091A208039F3946EC
:10DDB4000493B04700286CD48000049B1B18C71937
:10DDC4000397241A069A0299A6081ED011432869BB
:10DDD4000A46E9694F6B0092039932460493B847A7
:10DDE400002856D48100671AB04254D103208443DA
:10DDF40003980619049B1B19864202D2286B401C07
:10DE04002863069A03E0274601E02746039E022F73
:10DE140020D301201146039001432869EA69546B19
:10DE240000917A080596314616460493A0470028C7
:10DE34002FD441007C1AB0421BD103988743059824
:10DE4400C619049BDB19864202D2286B401C286346
:10DE5400069A00E03C46002C0AD02869E9694F6B19
:10DE6400009231462246B847002812D4241A00E012
:10DE74000024079800280AD0A86B8168002901D0E3
:10DE840009A888472869E9694A69002190470898E0
:10DE9400001B0BB0F0BD3C46EBE7C0460000FF3F63
:10DEA40080B5024B09F047FD80BDC0462083B8ED24
:10DEB40070B50446034E3578034901F0B1FB347064
:0CDEC400284670BD330E002040420F00C5
:10DED000002803D0012803D1034800E00148016075
:0CDEE0007047C04600F0FF1F04F0FF1F59
:10DEEC0080B50A480021016001200AF0E5FD64209C
:10DEFC0008F06EF872B6064806490160064841788B
:10DF0C00491C4170FAF772FB80BDC046780C0020AA
:0CDF1C0000F0FF1F21433412500E0020C3
:0CDF2800014810307047C0460082000025
:10DF3400F0B5C3B01446FF22D5432A46FF32002869
:10DF44004ED0002C4ED016464A0B01964CD10746B3
:10DF54006018274B5B1C984246D8012000020290AF
:10DF6400FF2923D800953D4602980F46461AA6423B
:10DF740000D3264603A801902946324608F0E6F865
:10DF84003B20C00238180023019932460193FAF766
:10DF9400CBF93946F119A41BAD190298814201D27B
:10DFA400002CE1D12F46002C009D1DD04D19029864
:10DFB4008442264600D3029E03A801903946324685
:10DFC40008F0C4F80B48281800230199324601933D
:10DFD400FAF7AAF97519A41BBF19002CE7D103E0BD
:10DFE400019201E000200190019843B0F0BDC046C9
:08DFF400FF1F000000D901002D
:10DFFC00B0B50B4CA088002810D0451E0DD1A078D0
:10E00C0001214140A170002802D02046083000E0D8
:10E01C00A01D0588002000F03DF8A580B0BDC046CD
:04E02C00F60C0020CE
:10E0300010B5002800DD10BD0A214143044A5318E1
:10E0400001245C70515C0029F5D109F0A1F810BDE4
:04E05000F60C0020AA
:10E0540010B5002800DD10BD0A214143044A5318BD
:10E0640000245C70515C0029F5D109F090F810BDD2
:04E07400F60C002086
:10E07800B0B5002800DDB0BD0A214143054A531858
:10E088005C78012565405D70515C0029F3D100F092
:08E0980003F8B0BDF60C0020F6
:10E0A00080B50A214143084A535C5118002B01D026
:10E0B000891C00E0491C0978002902D009F068F8A1
:0CE0C00080BD09F066F880BDF60C002061
:10E0CC00B0B5002800DDB0BD0A2242430B88114CCC
:10E0DC00A354A2188D88D580CC881481002C07D02D
:10E0EC00002D09D0151D4988002908D0298001E090
:10E0FC0000219180012104E00021918001E02C801D
:10E10C0000219170002B01D100219180FFF7C2FFFB
:08E11C00B0BDC046F60C002066
:10E1240082B02B48C41D07208443FAF75BFB001B15
:10E13400411C204603F054FDFAF79AF90AF01AFC40
:10E1440009F059FC00242046FFF770FFFAF774FA2F
:10E15400FAF75EFA0125284609F0C0F800F080F9C4
:10E1640009F0C2F8FCF732FE1A4E1D4F0AF0C0FC4B
:10E17400002807D12046FFF77DFF3470322007F0D6
:10E184002BFFF3E71448057000263046FFF74EFFD7
:10E1940012480078002810D13D6001A800F086F9EB
:10E1A4000028F5D4F0433860FCF700FE01A800789D
:10E1B400FDF7EEF9FCF7F2FDEAE7FCF7F7FD00F0F6
:10E1C40067F9FCF7EBFD034806700646CEE7C04648
:10E1D400B0120020360E0020340E0020370E00202E
:04E1E400780C002093
:10E1E80080B5002904D0034A12689268904780BD20
:08E1F800002080BD380C00205E
:10E2000080B5024A1268D268904780BD380C002061
:10E2100080B5024800680068804780BD380C002047
:10E2200080B500280CD000290AD0064A1268002ABE
:10E2300002D000F011F880BD034A1268526990477D
:0CE2400080BDC046340C0020380C0020CB
:0CE24C000148012101707047370E0020CE
:10E25800F8B50C4605462348006800283AD0224FF6
:10E26800396800291ED0214A1268521AA24226464D
:10E2780000D81646002E15D040182946324607F019
:10E2880063FF386881193960A41BAD191748006805
:10E29800814207D113480068154A1268D26990472D
:10E2A80000203860002C14D01048006846422640F0
:10E2B80008D00F480068C269284631469047A41B19
:10E2C80007D0AD19074800682946224607F03CFFE9
:10E2D8003C60F8BD06480068C26928462146904758
:10E2E800F8BDC0463C0C0020400C0020440C002027
:04E2F800380C0020BE
:10E2FC0010B5084C2068002800D010BD06480068F6
:10E30C00406A804705490860054903F0E3FB20603B
:10E31C0010BDC0463C0C0020380C0020440C0020E2
:04E32C008D960100C9
:10E33000F0B589B00446C9B201A820252A460AF0E2
:10E3400059FD0B4F202C264600D32E463868002856
:10E3500004D001A83146FFF77FFF05E005480068BB
:10E36000426901A831469047A41BEBD109B0F0BD2A
:08E37000340C0020380C0020E1
:10E3780080B5064A1268002A02D0FFF769FF80BDFF
:10E38800034A12689269904780BDC046340C002049
:04E39800380C00201D
:10E39C0010B5094802680A480068002808D0074CE4
:10E3AC002168002904D0526990470020206010BDDC
:10E3BC00106A804710BDC046380C0020400C00206D
:04E3CC003C0C0020E5
:10E3D00070B588B00446094E202C254600D3202570
:10E3E000002D06D03068826868462946904700288C
:10E3F00002D1641BF0D1002008B070BD380C0020A1
:10E4000080B5034909688A680421904780BDC046E9
:04E41000380C0020A4
:10E4140070B582B0044600220192002913461546C5
:10E42400164610460CD009480068826801AD28469B
:10E4340090472E78E9780A06A9780B0469780D02CA
:10E4440035431D431543256002B070BD380C0020D0
:10E4540080B5024800684068804780BD380C0020C1
:10E4640080B5044807F002F900F078F8024803493F
:10E47400016080BD940B0020380C00200868010066
:10E4840080B5024807F022F980BDC046940B0020F5
:10E4940080B5044800210170034800680069804782
:0CE4A40080BDC046370E0020380C002060
:10E4B00070B582B00446184D09F0E8FA002803D080
:10E4C00009F0DFFA00280FDC09F0E0FA002806D096
:10E4D00001A80026314609F0C3FA002810D4022111
:10E4E000284607F01BF9E7E7074808490160084894
:10E4F000006A084A10608A6801212046904700E0BF
:10E50000F04302B070BDC046380C0020086801001E
:0CE51000500E0020640C0020940B002032
:10E51C0080B502490860FFF7EBFE80BD340C00208B
:10E52C0080B505480168002902D0491E016000D061
:0CE53C0080BDFFF72DFF80BD340C0020D7
:10E5480010B5044C2068002803D003F0D9FA002045
:08E55800206010BD3C0C002006
:10E56000F0B585B000F07AF805F0E8F9FCF78EFD1B
:10E5700000240094012002254026294632462346E5
:10E5800005F060F904AF387000962C4B2046294600
:10E59000324605F057F97870384603F043FC2849B5
:10E5A000204603F067FC27482749224605F0BCFDBA
:10E5B00026484088800602D5002003F045FCFCF781
:10E5C000EDFA502503AE0122304629460AF032FA10
:10E5D0003078002805D0FF2803D06D1C702DF1D1B4
:10E5E00024E02E46503E1A4806421FD019480AF031
:10E5F000F5FB029040194E38174903F071FA0028D4
:10E6000014D007461349029A07F0A2FD5F20029931
:10E61000785478180290401C502132460AF00AFAC9
:10E62000029840194F38047008488760074805F081
:10E630003DFF05F0C7F905B0F0BDC046830D0020D1
:10E64000FD8A0100A00B0020C9E600005C1000203C
:0CE65000DFFFFF7F569501002A9D0100AE
:10E65C0070B584B009F028FD054601AC01212046B7
:10E66C000A460AF0E1F9124E002D00D1361D207831
:10E67C00022806D0012802A80021042209F085F9FD
:10E68C0004E002A8082104220AF0CEF902980B2417
:10E69C00084D0A2103AA0AF0AFFB03993031295522
:10E6AC00641E611CF5D30448468004B070BDC0469E
:0CE6BC0021100000881000205C100020DD
:10E6C80010B50C4603200840022801D0FFF7D6FEFB
:10E6D800600702D501480121017010BD350E0020E8
:10E6E80010B582B00C46014606480068009000202C
:10E6F8002246034603F098FAA04201D009F0A5F992
:08E7080002B010BD80100020DA
:10E71000B0B582B0074D2868009000240123204640
:10E720002146224603F084FA2968204603F0AEFB16
:08E7300002B0B0BD8010002012
:10E7380010B50C460146054803680020224603F040
:10E7480065FAA04201D009F080F910BD80100020C0
:10E7580070B582B00C4605460B4801680026304665
:10E7680003F09CFB002801D009F06FF9F0430090FA
:10E77800304629462246334603F056FA002801D58A
:0CE7880009F063F902B070BD80100020A1
:10E7940010B50C460146064803680020224603F0E3
:10E7A40077FAA04201D009F052F9002010BDC0460A
:04E7B40080100020B1
:10E7B800F0B587B014460F4624214143454A511805
:10E7C8008D690521CE43002D08D02968424A91421F
:10E7D80006D1A968DB2966D9361D78E0761C76E073
:10E7E8000496039300200290019406AA284639460D
:10E7F80000F010FB04998E1C002868D400240594AE
:10E80800022205AB28460097394600F047FB00284E
:10E818005DD405980399884253D1304F5822384621
:10E8280021460AF0E3FA64202D49F9643865029B11
:10E83800002B00D02C69069838642959F9632819E7
:10E84800B8646A6952187A65002B049A1AD0091FAD
:10E85800F96340180599002911D09200019BD4183A
:10E868001434890061580AF0ADFAF86B001FF86398
:10E878000599491E0591BA6C10180029F1D1042197
:10E888000AF0A0FA072205AB2846009900F006FB1B
:10E89800012818D107F02EF8104808F024FB064686
:10E8A80007F030F813E004960393A9690122029255
:10E8B800002999D029462A4600F024FA002893D541
:10E8C80004E0049E03E0054808F00DFB06463046C8
:10E8D80007B0F0BD8408002050435632E0090020FC
:04E8E8004C68010077
:10E8EC00B0B59EB001AC01212046FFF777FC207833
:10E8FC00112800D9D0E0C046784400794000874404
:10E90C00080A10CBCB121C1ECB364B6165696B769B
:10E91C008C90664801E008F0FBFA009009F081F851
:10E92C00BAE002207AE0052000F042F9002800D578
:10E93C00B2E05D4800F05AF9AEE0062047E002A8CC
:10E94C000821FFF74BFC0299039A544C544B204678
:10E95C00FCF7C4F90B904C200A900AAD28460830FD
:10E96C004822214607F0EEFB5021284692E002ACEB
:10E97C000C212046FFF732FC201D0421FFF74AFC36
:10E98C00464A906C002878D0029B0399CC18526DA3
:10E99C00944273D8C0187DE002A80C21FFF71EFC2E
:10E9AC003E4A906C00286DD0029B0399CD1802ACA6
:10E9BC00526D954267D8241DC018FFF70FFC042137
:10E9CC00204667E00B2000F0F3F865E00C2000F027
:10E9DC0067F961E00D2021E068460421FFF7FEFB9A
:10E9EC0000991F292FD802A8FFF7F8FB31E00AA8DD
:10E9FC000821FFF7F3FB24200A99414329484018CA
:10EA0C00806942690B9991422FD202698358801810
:10EA1C00C018FFF7E3FB0B9813E0102000F048F848
:10EA2C003AE00AA80C21FFF7D9FB24200A994143AC
:10EA3C001C48401880690B9940180C99FFF7CEFBC5
:10EA4C000C98C01716E00846FFF7BCFC02A8002182
:10EA5C00017002A800F0CAF80A901048C16B006C53
:10EA6C000B900C910AA80C2114E00846FFF7AAFCA5
:10EA7C000020C043029002A80BE00399084608F05E
:10EA8C00CBFF09E003990846FFF79CFC002000909F
:10EA9C0068460421FFF7BEFB1EB0B0BDE0090020A4
:10EAAC0001ED0000840800209E960100E63F000066
:10EABC0070B5A4B005461AA800240C2221460AF011
:10EACC0093F9102D11D00D2D1FD11DAE08213046FC
:10EADC00FFF784FB10A8047030781D901E99202934
:10EAEC0021D810A8FFF77AFB20E01AAE0C21304693
:10EAFC00FFF774FB10A8047030781A901B9920292A
:10EB0C0016D810A8FFF76AFB15E018A919AA284611
:10EB1C0000F028FB2420199E7043224908181899EC
:10EB2C00816121491DE00846FFF74CFC1D9E10E059
:10EB3C000846FFF747FC1C98810001221202904204
:10EB4C0003D86846FFF74AFB02E00846FFF73AFC99
:10EB5C001A9E19962420704312490818806918903F
:10EB6C0010A91C9B6A463046FFF720FE1F900F48E9
:10EB7C0003463C330ECB2092006821AA0BC2022D17
:10EB8C000AD12420704307490D18A869002803D026
:10EB9C00183502F0B3FF2C601FA81421FFF73AFBC5
:10EBAC0024B070BD840800209E960100E00900206E
:10EBBC0010B584B0694603AA00F0D4FA002400987A
:10EBCC00002806D02421039A4A43074989188861F2
:10EBDC0000E0E44302940420019001A80821FFF70F
:0CEBEC0019FB204604B010BD8408002076
:10EBF800F0B583B00646274884690420C743002C33
:10EC080008D020682449884206D1A068DB2832D978
:10EC1800FD1C2DE03D462BE00020019002AA204675
:10EC2800314600F0F7F8002821D41C4E0025582260
:10EC3800304629460AF0DAF864201949F16430654B
:10EC4800019B002B284600D0206902993164215885
:10EC5800F1632018B064626952187265002B07D0FE
:10EC6800091FF163401804210AF0ACF800E07D1C8C
:10EC7800284603B0F0BDA069012100280191CDD03C
:10EC880000202146224600F03DF80028C6D505465A
:10EC9800EEE7C0468408002050435632E0090020C1
:04ECA8004C680100B3
:10ECAC0070B584B000250C28284605D103AC04218E
:10ECBC002046FFF793FA20780390242460430C4EEF
:10ECCC003018202145548069002806D002F016FF28
:10ECDC0003984443301900218161002002900420E4
:10ECEC00019001A80821FFF795FA04B070BDC04649
:04ECFC008408002068
:0CED00000148006A7047C046500E002019
:10ED0C00F0B58BB01546242242433F48841820208E
:10ED1C00225C0020002A75D1EA68D300CF18203776
:10ED2C00002A099505900691049424D000263446B7
:10ED3C0038460AF04DF8411C0A917A5C0A928819FF
:10ED4C007918002A0CD04B780A93CA1895780A9532
:10ED5C00C018801C911C002DF5D1D71C099D00E01A
:10ED6C004F1C641C461CE8688442E1D30320064017
:10ED7C0001D0B81B071DA86900283BD0C00039186A
:10ED8C0000242246039102940892D0000790385830
:10ED9C000E1804251D48415930460AF0B9F80028D0
:10EDAC0006D001200004241808351C2DF2D127E0D0
:10EDBC00099D286906990818079979184968411816
:10EDCC0001910AA807900426324607F0BBF970207F
:10EDDC000A9901400C43832020430A90019807991B
:10EDEC00324607F0AFF9089A521CA869824203997F
:10EDFC00029CC9D30499203101200870059801E0C8
:10EE0C000720C0430BB0F0BD84080020306801001F
:10EE1C00F0B583B015460A46064600681C49884280
:10EE2C001ED1F0680024E1430291012824DB0095F7
:10EE3C00C0003018203001903746243702988000EB
:10EE4C00385801990818154611460AF061F800283F
:10EE5C0013D00837641CF06884422A46EEDB0FE0BE
:10EE6C000C4910460AF054F80290002802D00020F9
:10EE7C00C0430290042004E003E0386800210291B2
:10EE8C00009D002D00D02860029803B0F0BDC04654
:08EE9C00504356329E9601001E
:10EEA400F0B585B00491064600682B4988421AD112
:10EEB4000292019337462037F068C1007918002484
:10EEC4000128039413DB002438680D4608180499BC
:10EED4000AF022F8002808D0F068641C083784423D
:10EEE4002946F1DB03E0002004E0F068294684426F
:10EEF40002D1039805B0F0BD0D46049809F06CFFEB
:10EF0400F168491E8C4204D13A68A9183369F31890
:10EF140002E03968BB680A46C4431B195B1A8018AF
:10EF24004019401C029D002BE3D00478002CE0D053
:10EF34002106DED442781106DBD4811CAC4205D014
:10EF4400981E831A8818002BEDD1D2E7019807F098
:0CEF5400FDF80120CEE7C04650435632C5
:10EF6000B0B534C8036888180C194A1902490968F1
:0CEF70004D682146A847B0BD8410002069
:08EF7C0000487047FAFEFFFF98
:0CEF84000148006A7047C046500E002093
:10EF900010B500780021CC43062806D8800004492B
:10EFA00008588047FF2800D00446204610BDC046C0
:04EFB000DC69010017
:10EFB40080B50168CA1F0B2A40D841687A44127987
:10EFC40052009744050A10151A1F243B3B3B3B296A
:10EFD400012041401A48017030E07D20C0004843C0
:10EFE40000F054FB2AE000291AD008F024FE25E0A2
:10EFF400002918D008F042FE20E0002916D008F0BD
:10F0040028FE1BE0002914D008F031FE16E0002988
:10F0140012D008F025FE11E0012008F0BBF80DE045
:10F0240008F0D8FD0AE008F0FFFD07E008F0E7FD6E
:10F0340004E008F0F2FD01E008F0E8FD002080BDE6
:04F04400310E002069
:10F0480080B50168CA1F00200F2A10D87A441279A7
:10F058005200974407141B1E2124272F2F2F2F2FD0
:10F068002F2F2F2A164801780120484080BD2129DA
:10F078001ED022291ED11048806C008880BD09F05E
:10F088004DFE7D21C90007F01BF880BD09F05AFE2E
:10F0980080BD09F05BFE80BD09F048FE80BD09F027
:10F0A8004DFE80BD09F046FE80BD0448007880BD55
:10F0B800F9F7ACFA80BDC046E0090020330E002005
:04F0C800310E0020E5
:10F0CC0070B582B00D4606686C46002107222046BA
:10F0DC0009F08AFEA8192146FDF76AFDA0790121E5
:10F0EC000140074801706079002805D10548007877
:10F0FC00012801D100F05CFD002002B070BDC046BB
:08F10C00300E0020330E00203C
:08F1140000487047FAFEFFFFFE
:10F11C0080B5074B1B78012B07D1002901D00421A6
:10F12C000843114600F038FB80BD0120C04380BD70
:04F13C00330E00206E
:10F1400010B51446094A1278012A0BD1002905D0BE
:10F1500004210843002100F09BFB0320214600F01E
:10F1600097FB10BD0120C04310BDC046330E0020E8
:10F17000F0B58DB00192009100240C940B2802D1BF
:10F180000CA8FFF73DF90BA8FFF73AF924260C98D5
:10F190007043264908182027C4550B9D214603AC0F
:10F1A000204602913A4609F025FE202D00D33D4627
:10F1B00020462946FFF718F81D48039C844201D1D8
:10F1C000089902911949844200D1049C0CA8007846
:10F1D0000C907043081880690B9F002807D002F03C
:10F1E00093FC0C984643114880190021816138191D
:10F1F00002994018603002F033FC00280CD006461B
:10F2000003A92A4606F0A4FF70190B99491BFEF7C3
:10F21000EBFF0098066003E00B98401BFFF7D8F85F
:10F220000C98019908600DB0F0BDC046840800201C
:04F2300050435632BF
:10F234000246032043020A489A4205DCFF230233B4
:10F244009A4208D0094B03E0064B9A4203D0064B7E
:10F254009A4200D00020002901D000220A607047A1
:10F26400EC64010001060000010E0000010300002F
:10F27400042801DB00207047800101490818704709
:04F28400C40600209C
:10F2880070B5044602F0C8FB01214A02904201DC35
:10F29800002501E0164A851809225202904200DD35
:10F2A8000D03002D22D01349284602F015FC002832
:10F2B8001CD00646E069C36A204631462A4698476C
:10F2C800002810D4291A304602F02AFC0020A08415
:10F2D80026612062E0690068002807D0064902F02C
:10F2E800FBFB206270BD304602F00AFC70BDC046D0
:0CF2F80000FEFFFF5E9D01006A93010014
:10F30400B0B580010E490C182069002817D0E169B6
:10F31400C96D002900D08847206A002803D0204600
:10F32400203002F04BFC254610356069002803D0DC
:10F334001434204602F042FC284602F03FFCB0BDE3
:04F34400C4060020DB
:10F34800F8B5032824DC0D4604460F790E68FFF74C
:10F35800D5FF300E0026FF28314600D00102C8191B
:10F368003146FFF763FFE861A0010A490F18402200
:10F378003846294606F0E8FE200107490C181022F5
:10F388002046314609F032FDBC633846FFF778FF66
:0CF39800F8BDC046C40600208C0A00200E
:10F3A400F0B585B01C46134604910646134FF86920
:10F3B400C26C002A16D03869012103939047F8697A
:10F3C4004068029000250094019538463146049A1D
:10F3D400039B029CA04704463869F969CA6C294614
:10F3E400904708E0456800200094019003483146A6
:10F3F400049AA8470446204605B0F0BDC406002080
:10F40400F0B583B01C46134602910646104FF869C6
:10F41400C26C002A12D03869012101939047F8691F
:10F424008568009438463146029A019BA8470446F1
:10F434003869F969CA6C0021904706E08568009430
:10F4440003483146029AA8470446204603B0F0BD5B
:04F45400C4060020CA
:10F45800F8B513460D4606460F4FF969CA6C002ADF
:10F4680011D038690121009390473869F9690C690E
:10F4780031462A46009BA04704463869F969CA6C98
:10F488000021904705E038690C6931462A46A047B3
:0CF4980004462046F8BDC046C406002013
:10F4A400B0B50F4DE969CA6C002A0DD02869012155
:10F4B40090472869E969096A884704462869E9691F
:10F4C400CA6C0021904703E02869096A884704460A
:10F4D400601E414241413C2029542046B0BDC046F3
:04F4E400C40600203A
:10F4E800B0B50F4DE969CA6C002A0DD02869012111
:10F4F80090472869E969C969884704462869E9691C
:10F50800CA6C0021904703E02869C9698847044606
:10F51800601E414241413C2029542046B0BDC046AE
:04F52800C4060020F5
:10F52C00B0B5104DE969CA6C002A0FD028690124C6
:10F53C00214690472869E9694A6921469047044663
:10F54C002869E969CA6C0021904704E028694A6976
:10F55C00012190470446002C02D13C200021295463
:08F56C002046B0BDC4060020DA
:10F57400F8B5009315460E46074608480168084C3E
:10F5840021600022026008698047206804683846C8
:10F5940031462A46009BA047F8BDC046800C002097
:04F5A40084100020AF
:10F5A800F8B5009315460E46074608480168084C0A
:10F5B8002160002202600869804720684468384654
:10F5C80031462A46009BA047F8BDC046800C002063
:04F5D800841000207B
:10F5DC0010B506480168064C2160002202600869DB
:10F5EC00804720688068804710BDC046800C002092
:04F5FC008410002057
:10F6000010B506480168064C2160002202600869B6
:10F6100080472068C068804710BDC046800C00202D
:04F620008410002032
:10F62400B0B5F9F775F80D4900240C60002801D035
:10F63400014600E00A490B4A1160002800D1E44366
:10F6440089692E25002905D000208847002801D08B
:10F6540080470546044805602046B0BD800C002064
:0CF66400F869010084100020480C002010
:10F6700080B505490868002805D000220A600349C2
:10F6800008600069804780BD800C00208410002045
:10F6900080B5014602480078FFF7C4FF002080BD16
:04F6A000330E002005
:10F6A400B0B50C4C2168002900D0B0BD0A490968E6
:10F6B400C140C807F9D0094D2868C168002901D0A4
:10F6C4008847286820604069002800D104482860E1
:10F6D400B0BDC046800C0020480C002084100020DF
:04F6E400146A0100A3
:10F6E800034801680029FCD00020C0437047C04689
:04F6F8004C0C002096
:10F6FC00034801680029FCD00020C0437047C04675
:04F70C004C0C002081
:10F71000034801680029FCD00020C0437047C04660
:04F720004C0C00206D
:10F72400034801680029FCD00020C0437047C0464C
:04F734004C0C002059
:10F7380010B584B002A9FF20087001A80022027049
:10F74800034A1268546803AA0823A04704B010BDEE
:04F7580084100020F9
:10F75C0010B582B0044800684468044804496A46FD
:10F76C003023A04702B010BD841000206495010026
:04F77C00A3100020B6
:10F7800010B582B0044800684468044804496A46D9
:10F790003023A04702B010BD841000206A950100FC
:04F7A000A310002092
:10F7A400F0B591B002AA0023009353702D4B185C5E
:10F7B40010700591080C4840010A4140080948406E
:10F7C400810841404808484001210191084005A9A9
:10F7D40008712548066A6436254C24480068456843
:10F7E40002A803AF0D2321463A46A847797807209B
:10F7F4000840022804D11C48006A8642EDDA17E06A
:10F80400012818D0042820D00098012825DC1C48A1
:10F814000078002821D11548006845682120C300DC
:10F8240007AA18481849A8470098401C0090D4E734
:10F834000198C04314E00D480068446805A80F49C6
:10F8440003AA2123A04700200AE00848006844686E
:10F854000848094907AA3023A0470198C043401C1F
:10F8640011B0F0BD729D0100500E002084100020E4
:10F874009510002064950100A3100020781000204A
:0CF88400300E0020A3960100C496010085
:10F89000F0B591B0019105A900220A7103A9029265
:10F8A0004A70284A105C08702748076A6437274C5A
:10F8B0002068456803A804AE0D2325493246A847B1
:10F8C000767807203040022804D11F48006A87421A
:10F8D000EEDA15E0042816D001281FD0029E012E72
:10F8E00018DC1E480078002814D1206845682120C3
:10F8F000C30007AA1A481B49A847761C0296D7E7F7
:10F900000120C0431CE0206844681248124907AA3D
:10F910003023A0470120C043401C11E02068446808
:10F920000B48811C05A804AA2123A0470020019BA5
:10F93000002B05D004998900F206920F89181960EE
:10F9400011B0F0BD7A9D0100500E002084100020FF
:10F950009C10002064950100A3100020300E0020B0
:08F96000A3960100C49601000A
:10F96800F0B589B00E46054600F050F80190002821
:10F9780047D403A8012102914171FF210171C1708F
:10F9880081704170017002CD07A8029C44710A0C75
:10F998004A40130A53401A095A40930853405A08D8
:10F9A8005A402240763202710791174909684C681B
:10F9B80003A905AF2E233A46A04778790E210140C6
:10F9C800022904D000F022F80190002819D4761EEC
:10F9D800012ED8D82968080C4840020A424010096C
:10F9E800504082084240530853400298034007A8F9
:10F9F80003710791044909684C6803A905AA2123E2
:0CFA0800A047019809B0F0BD8410002058
:10FA1400F0B58FB004A800224270BB21017003A886
:10FA240000924270FF2101700120C04301901E48E2
:10FA3400046A64341D4D2868466804A803A902AF0B
:10FA44000D233A46B047797807200840022804D1AC
:10FA54001548006A8442EEDA16E0012816D004281C
:10FA640016D0009801281ADC13480078002816D113
:10FA7400286846682120C30005AA10481049B047E9
:10FA84000098401C0090D6E701980AE0002008E0A6
:10FA9400286844680648074905AA3023A047019806
:10FAA400401C0FB0F0BDC046500E00208410002052
:10FAB40064950100A3100020300E0020A3960100DD
:04FAC400C4960100E3
:10FAC800F0B587B016460F460546072000242146A4
:10FAD800FFF7DAFEE143002801D00C4660E0039608
:10FAE800022F1CD3032028407F1E00282DD00E464D
:10FAF800072004A9FFF7C8FE002848D104982870F9
:10FB0800010EE970010CA970000A687004210398BD
:10FB180009F026F92D1D7F1EEAD1029600E0029118
:10FB2800032004A9FFF7B0FE06460499284609F009
:10FB380049F9002E34D01C48006844681B481C4909
:10FB480005AA3023A047029C2AE002910399019458
:10FB580000293E4606D08868C968081A87423E468A
:10FB680000D30646002407202946FFF78DFE00280B
:10FB7800E1D1641C2D1DB442F5D3039C20463146C7
:10FB880009F0EEF82146BF1B019CE1D1C8E7064801
:10FB9800006844680548064905AA3023A04734464A
:10FBA800204607B0F0BDC046841000206A950100C9
:04FBB800A310002076
:10FBBC00F0B58BB0334F386845682120C40032480B
:10FBCC00324901AA2346A847002569462846FFF773
:10FBDC0059FE002812D508F0C1FE322006F0F8F9C3
:10FBEC00386845682848294901AA2346A8470020B7
:10FBFC006946FFF747FE00283AD4012501246E46DA
:10FC0C0020463146FFF73EFE3078B22108420FD035
:10FC1C00386846681E481F4901AA3023B0476E4613
:10FC2C0020463146FFF72EFE3078A021084225D120
:10FC3C000520010700910120FFF7AEFD0446002DC1
:10FC4C000CD0002C0AD008F08DFE322006F0C0F942
:10FC5C0000990120FFF7A0FD044606E0002D04D01A
:10FC6C0008F080FE322006F0B3F9601E844105E0F6
:10FC7C0008F078FE322006F0ABF9012420460BB0D8
:10FC8C00F0BDC04684100020A3960100C49601006C
:08FC9C0064950100A310002093
:10FCA400F0B583B0029101902A4C207801270028F6
:10FCB40014D1294800210170FF2602362749304615
:10FCC40001F00CFF26490E61086081262549304663
:10FCD40001F004FF24490E6108602770234E306848
:10FCE400002808D0224801780029FCD121488068E6
:10FCF4008047002030601F4DA86980471E4C20704B
:10FD0400174A116851609160D160174A13685360B3
:10FD14009360002B12D0002910D03068002801D045
:10FD2400401E3060154800906D68154A154B0198C7
:10FD34000299A8473068401C30602078124900229C
:10FD44000A6012490A60124908701248077003B029
:10FD5400F0BDC046290E00202A0E00207D9301002C
:10FD64002C0B002088930100400B0020500C002035
:10FD74002B0E0020F06201002C0E00206DFE00000E
:10FD84009DFD0000F1FD0000580C0020540C0020E3
:08FD94002D0E00202E0E0020B0
:10FD9C0010B504460D48006A0D4908600D480078FE
:10FDAC00002804D00C48806A8047002808D10B48F2
:10FDBC000122214607F06AFF002801D0002010BD67
:10FDCC00074800210170012010BDC046500E0020D4
:10FDDC00540C00202D0E0020F0620100400B00207E
:04FDEC002B0E0020BA
:10FDF00010B51749096A174A116017494A688B6894
:10FE0000DC43121901D50C691219002A0CD05C1CB4
:10FE10008C601870FF2302330868C3188C689C42FA
:10FE200000D18860501E00E000200C4909780029AC
:10FE30000DD00B490978002909D1012807DC0948B0
:10FE40000068002803D10848016A0120884710BDD6
:10FE5000500E0020580C00202C0B00202D0E0020EE
:0CFE60002A0E00205C0C0020F062010063
:10FE6C0080B508480078002803D00748007800289F
:10FE7C0000D080BD054800780028FAD100F00CF9BC
:10FE8C0080BDC0462D0E00202B0E00202F0E002012
:10FE9C0080B506480168002902D0491E016000D0D7
:10FEAC0080BD03488068804780BDC046500C002050
:04FEBC00F0620100EF
:10FEC000012181F310880449086004480121017070
:10FED000002181F3108870475C0C00202A0E00205E
:10FEE000F8B505461A48006800282DD0194B586807
:10FEF0009E68F2438718186900D53F188F4200DBCF
:10FF00000F461449096800970818801B87423C4631
:10FF100000DB044630462946224606F019F932191C
:10FF20000C49086909680B189A420E4600D016461B
:10FF30003F1B2D19002FE7D106488660009C012C3D
:10FF400003DB00F009F800E000242046F8BDC046BD
:08FF5000500C0020400B0020C2
:10FF5800F8B5154C012525701448007800281FD1E4
:10FF68001348017801290ED100260670114F387800
:10FF780002280ED01048806A8047012808D13E70B8
:10FF88000D48406A80470B480078002801D105E0F9
:10FF98003D700948806A8047002801D100F07EF84A
:10FFA80000202070F8BDC0462F0E00202B0E002028
:0CFFB8002E0E00202D0E0020F062010033
:10FFC40070B50A460146124800680024002804D08F
:10FFD40010484368C068984201D0204670BD0D485F
:10FFE40007F058FE04460C4800780028F5D0002C91
:0CFFF400F3D00B4800780028EFD1084E35
:020000021000EC
:1000000030680028EBD00848016A00252846884758
:100010003560E4E7500C00202C0B00202D0E002052
:0C0020005C0C00202A0E0020F0620100A1
:10002C00044948688A68D243801801D50969401888
:08003C007047C046400B002094
:10004400B0B508490B6914C9D51822180839AA4251
:1000540000D3D21A4A60002803D00348016A002062
:0C0064008847B0BD2C0B0020F0620100AA
:1000700070B50B4A9368D1681569146866198B428C
:10008000344600D31C46631A04D0B44200D3641B28
:10009000D46000E00021002800D00360084670BD55
:0400A0002C0B002005
:1000A400B0B582B00C4D002028600C4908600C48A3
:1000B40001A90124224607F0EDFD012809D10948D0
:1000C400006A28600848047001A800780749096894
:1000D400884702B0B0BDC046540C0020580C002024
:1000E400400B0020500E00202B0E0020F062010077
:1000F400F8B56821304F785C002800D0F8BD009135
:100104003868002801D12D483860397B002901D195
:10011400402139737D68002D01D102257D600222C2
:100124000124EB43C018831E484218403C627A62A3
:10013400B86205F0A9FFF8622149884201DA0C216E
:1001440000E010213C640022FA6339634843401EF6
:10015400C117090D40180013811C7964401C786391
:100164004000401CB8644019F86400F0DDFD786D6F
:10017400002801D001F0C6FC786B4002114901F05F
:10018400ADFC7865796B4A020025294608F030FEFB
:100194000720C043C61D396B32468A40811A28465F
:1001A40000F0D8FD386B8640F143204600F0D2FDC4
:1001B40000983C54F8BDC046140900204555000081
:0801C400F50F0000E5960100B3
:1001CC00F0B5A5B00746002B01D0002018600293B3
:1001DC00109203920020C5432C463A5C2E2A02D082
:1001EC00002A01D102E00446401CF6E7621C0246DC
:1001FC0000D02246861AB818002E00D0401C002EC3
:10020C0000D0761E082300240F94109C1C401094E0
:10021C0030D10124002A24D00D94082A20DC032E8E
:10022C001EDC0E930890099604913C460A921646E1
:10023C00207800F04BFE002815D1761E641C002E91
:10024C00F6D1099E002E00D1F9E1089C207800F02F
:10025C003DFE002807D1761E641C002EF6D104E06A
:10026C000D9C0F9406E00D980F900499099E089828
:10027C000A9A0E9B402A00DD6EE1402E00DD6BE1F8
:10028C0008900029049109960A9210D00E93ED481B
:10029C00C46A002611A9304600F08EFD1198002882
:1002AC0008D0761CA642F5DB0024019409E000205E
:1002BC00019024E0B44201D0019601E000200190AD
:1002CC00A41BE04E307B410204984018401E05F000
:1002DC00F5FE844200DA3FE10090F06A461E23A945
:1002EC00304600F069FD2398002802D0761EF6D126
:1002FC0003E00098301A401C0190099E0E9B0F9849
:10030C00002803D0002E17D0022016E00E9320A850
:10031C0020210B26324608F067FD1098002800D1EA
:10032C001EE10A9B0B2B1A4600DB324620A83946ED
:10033C0008F026FD039F2CE101200A99711808187A
:10034C00079040001A2124AA0D9108F055FD24991C
:10035C00002900D0401C0F900F200C9040010E90F3
:10036C00B84840684002400910901BD000260B96FC
:10037C0034462009B4490840002100F05BFD0028F8
:10038C0012D031460E9A1140405CE52804D000286A
:10039C000AD00B98401C0B902036641C1098A0427D
:1003AC00E7D101E000200B9010980B99401A0F999F
:1003BC00884200DCD0E020A820210B2208F014FD9C
:1003CC000A9B002B079E3046099C07D0062B1A4629
:1003DC0000DB062220A8394608F0D2FC20A97E2298
:1003EC000A54081831214170002C09D0032C2246E4
:1003FC0000DB032220A808300899234608F0C0FC33
:10040C0020A807F081FC0020034620A9095CDA0132
:10041C00DBB25B08D2188B18401C0B28F5D10B9360
:10042C00B819461919A96818401E099008461630C3
:10043C00089011A802461C3206920A310A91411CFE
:10044C0005910E3007900F98109011A800242022CF
:10045C00214608F0C9FC19A8FF210D9F3A4608F067
:10046C00C3FC24992494002900D00F460999C9197A
:10047C0032784C700A7076196918491EBF1EF7D174
:10048C0019A90A22059805F05DFE0C2207980A9915
:10049C0005F058FE04220698089905F053FE11A8A1
:1004AC000B9941730C99C1720F99109A8A4201D021
:1004BC00114601E040211143017000F09DFC0746FC
:1004CC00000961490840012100F0B4FC002807D064
:1004DC0079010E9A1140401811A9202205F032FE24
:1004EC001098401EB0D111AF20223846214608F09A
:1004FC007BFC3846083020AE31460831032205F02B
:10050C0021FE08223846314605F01CFE3C82FC8157
:10051C007C730398F8720498189038461430019E36
:10052C00310C08F049FC38461A30B1B2049E08F080
:10053C0043FC464838837C82FC8200F05DFC044618
:10054C00000941490840012100F074FC002853D0F7
:10055C0061010E9A11404AE02C46204625B0F0BDB0
:10056C000A9B082B1A4600DB0E9A20A8394608F085
:10057C0007FC099B002B039F08D0032B1A4600DBBA
:10058C00032220A80830089908F0FAFB20A807F0ED
:10059C00BBFB11AC002620222046314608F024FC7F
:1005AC0020A90B22204605F0CDFD2682E68166733C
:1005BC00E7720498189020461430019F390C08F00B
:1005CC00FBFB20461A30B9B208F0F6FB1F4820831B
:1005DC006682E682049E00F00FFC04464001400A4D
:1005EC00012100F027FC002806D02107C90D401876
:1005FC0011A9202205F0A6FD0024002EADD00198F3
:10060C00009A10180F49C96A884212DC0120871A17
:10061C000198461C002F01D0314604E00949096BB2
:10062C002A468A40D14300F091FB7F1C012F3046B3
:10063C00EFD10298002890D0019901608DE70499C0
:10064C0015E6C04614090020FFFF7F00724500002C
:0C065C00014988617047C0461409002065
:0C0668000149C8617047C0461409002019
:1006740070B50C460546FFF73BFD0B4884634561A6
:10068400012C0FDB2E68002E08D0A9682B460C33F2
:1006940021223046FFF798FD002803D4641E10354C
:0C06A400002CEFD170BDC04614090020EE
:0C06B000014908607047C0461409002092
:0C06BC00014908737047C0461409002073
:0C06C800014948607047C046140900203A
:1006D400F0B58DB00C4607467E48C16C0026B94281
:1006E400304605DC781A7B49097B05F0CDFC801C7B
:1006F4000690009609A908AA334600F0F7F8FF20EF
:1007040040000790851C204631462A4608F070FBBD
:10071400704E316CB94228D925462435E920207021
:10072400E01C6D49082205F011FD20460B30012123
:10073400490208F045FB307B6073318C20460E3053
:1007440008F03EFB02202074B188204611300905D0
:10075400090C08F035FB31686048814220DC2046F2
:10076400133089B208F02CFB1EE00495B06CB8423B
:100774004AD9781A0C90756B0CAA294608F040FBEC
:100784000C9840020C906902884206D2716D0918D7
:100794000798821C204605F0D9FC00F0AFFB30E03E
:1007A4002046203008F010FBF82060754948818EFF
:1007B4002046163008F004FB20461830FF2108F0CC
:1007C400FFFA20461A303F2108F0FAFA2920A870CF
:1007D4008020287020462730414908F0F5FA204649
:1007E4002B3040490B2205F0B1FC204636303E49FF
:1007F4000A2205F0ABFC5520079960546018AA2121
:10080400417000200DB0F0BD71680918B9420CD9CF
:10081400381A002100F012FB00282CD0014607985A
:10082400821C204605F092FCEBE70397029409A88A
:10083400007808A9097801430699E2D02548846B19
:10084400012CDEDB2348027B05924669F768781E9B
:1008540088420BD2B568E817C00D281840120599D4
:1008640005F012FC0699C01988420BD2641E10369A
:10087400002CEBD1C5E70798821C0021204605F027
:10088400C3FCBEE7B81E07DB059941431148C06CA1
:1008940008180399091A00E0039949028D42B0D956
:1008A4007068002808D043186A1A0498824200D35A
:1008B400024602981946B5E7064A9469002CF2D01C
:1008C4006A1A0798801C824200D302460298334673
:1008D400A04796E714090020F2960100FFFF0000EC
:0C08E40067452301829D010093930100F1
:1008F000F0B587B01F4616460D4604900024092225
:100900000846214605F082FC04223046214605F0C7
:100910007DFC39460C9F002900D00C60002F00D0D0
:100920003C600498022850DB3C4840680001059078
:1009300040D0009100242046214600F081FA002892
:1009400039D00196029703952107C90D4618F07A10
:100950003F2101400F2920D0307800281DD0E52804
:100960001BD0708B002818D0054606A900F02AFA83
:1009700000270698002808D0F943284A126B9140B6
:1009800002468A43C9438A42EED104988542039DB8
:1009900003DB708B0499884219DD641C059884423E
:1009A0000CD06001400A002100F04AFA0028CBD1A7
:1009B000029F00E003E00020287000E0029F002F6B
:1009C00003D02878002800D03E6007B0F0BD009921
:1009D000002900D0086008222846314605F0B8FBFF
:1009E000314608310322019805F0B2FBE85D20286A
:1009F00003D07F1C082FF9D101E00020E85500202A
:100A0000029F0199095C202903D0401C0328F8D1DA
:100A1000D5E70021019A1154D1E7C04614090020FE
:100A2000F0B58FB007910546984FF86CA8421FDCCF
:100A3000281A397B05F02AFB002819D4064609A894
:100A40000090B01C0CAC0BAA0AAB2146FFF750FF7C
:100A50002178E52900D115E10998002800D1A9E005
:100A6000C269002A00D0A6E0002009900A90A2E006
:100A7000386CA8421CD8796B0A18AA4218D9281ACF
:100A80000C900CAA08F0BEF90C9840020C90796BFF
:100A90004902884206D2796D081801214A02079955
:100AA00005F056FB64200121395400F029FAE9E0F1
:100AB000B86CA84200D9E5E079680A18AA4200D8C3
:100AC000E0E02C1A8C4200D3DCE0012120460491A6
:100AD00000F0B6F902906E4820400027394600F039
:100AE000AFF905900028079E1AD1304608300690CD
:100AF0001024F07A3F2101400F290FD00CAD0822BD
:100B00002846314605F024FB0BAE032230460699F9
:100B100005F01EFB00202872F070079E641EE8D1CD
:100B20000498400206900598C519F4192022284619
:100B3000214605F063FB002830D02878E52801D055
:100B4000002801D1049800E00020E17A3F220A4009
:100B50000F2A23D0002810D10CA803900822294680
:100B600005F0F6FA08350BAE03223046294605F0AB
:100B7000EFFA002003990872F0700CAD08222846A5
:100B8000214605F0E5FA08340BAE03223046214633
:100B900005F0DEFA00202872F070079E20370698D4
:100BA000B842C0D1029800286CD00799069A05F087
:100BB000CFFA67E00020BA6D002A03D03A6E521CCB
:100BC000AA425FD1002906D00A99002903D0022940
:100BD0000CDA00210FE0F96C691AFB6D3A7B541EA8
:100BE0000C4205930CD0002B14D11AE03A7B891EDD
:100BF0005143FA6C8918691A4C026142614114E050
:100C0000012306930024059B002B0FD03B6E5B1C39
:100C1000AB420BD13B6E5B1CAB4202D10599691A0A
:100C200001E07243891A4C0200210691FE69002EF0
:100C300028D0002811D008AE00210422304605F04B
:100C4000E5FA09980890F869059001204202079892
:100C500021463346059CA04705E0012042020023BF
:100C600007982146B047002809D40699002900D0EA
:100C7000FD653D66012805D10120B86502E0002030
:100C8000F865386600200FB0F0BDC046140900209A
:040C9000FFFF7F00E3
:100C9400F0B587B0234D686D002801D000F032FF15
:100CA40000F042F800276C222846394608F0A0F8E4
:100CB400F9F7A6FDFFF71CFA64200121295468689E
:100CC400000102903C466001400A0025294600F0DC
:100CD400B5F8002823D00F2149013940425C002A8D
:100CE40018D0E52A16D04618F07A3F2101400F2982
:100CF40010D004A801900822314605F027FA0836DE
:100D040003A800900322314605F020FA01980572E9
:100D14000098C5702037641C0298A042D3D10020EB
:080D240007B0F0BD1409002026
:100D2C0070B5094CA068002809D0206D00254668D4
:100D3C0000F0E4FE6D1CA06885423046F7D300201D
:0C0D4C00A060206570BDC04614090020A6
:100D5800F8B50091184A136B5843072405462540F7
:100D6800526D0026F7431F2B03DC3E469E40B143DD
:100D78000091002D09D0A9400091AF40C610965DA2
:100D8800BE430E430096E91801E00E461946C31803
:100D9800234008D00C18E410145DDC408C40344328
:100DA8000094C91A0831C0101018C91DCA10694624
:0C0DB80005F0CAF9F8BDC046140900207F
:100DC40070B582B00C4605460C48066B7543E910B5
:100DD400406D4118F01DC21001A805F0B7F90020BC
:100DE400C043202E01DAB040C04307210D400199D1
:100DF400E9400140216002B070BDC04614090020E2
:100E040070B50D484068400245090026344660012B
:100E1400400A002100F012F800280BD00F214901EC
:100E24003140405C002805D0E52803D02036641CFE
:0C0E3400AC42ECD3204670BD1409002035
:100E4000F0B583B00546224B5A680020AA423CD92F
:100E50009A6800292ED0AA422CD80190184650300A
:100E60004121C9000291002634460768002F19D19C
:100E70000298184900F034FE002818D007460021D7
:100E8000029A05F0C3F9384608303860002E02D0C7
:100E9000301D0F4902E00E4908465030076088684F
:100EA000401C8860641C381DAC423E46DDD9084BAE
:100EB0009A680198AA4208D9196D002D02D06D1EBA
:100EC0004968FCD1002900D0086803B0F0BDC046D5
:080ED0001409002070950100D7
:100ED80001460246203A01201F2A05D801239340E3
:100EE800044A134200D070475C29FCD07C29FAD010
:080EF80000207047058400D4BE
:100F0000F8B56425074E705D00280AD0F76A002402
:100F100069462046FFF756FF641CA742F8D100201F
:080F20007055F8BD1409002012
:100F280010B50168064A0B78093B172B05D8012430
:100F38009C40144201D0491CF5E7016010BDC04631
:040F48001300800012
:100F4C00F0B583B00F460568264C29780A46093A55
:100F5C00172A05D801239340234201D06D1CF4E7D6
:100F6C002B2900D16D1C2E782D2E00D16D1C2B78C9
:100F7C00302B16D1697820220A43782A18D1029096
:100F8C00A87806F0D0FE0024002829D40197AF1CC5
:100F9C0021010C1878787F1C06F0C5FE0028F7D5C7
:100FAC0014E019463039092902D90020C04315E054
:100FBC000290019700240A2161435C18303C6F1C9D
:100FCC006B78194630390A293D46F4D302980760EC
:100FDC002D2E00D1644201980460002003B0F0BDB6
:080FEC00E043FBE71300800065
:100FF400F0B58DB0E34FBE69002E00D043E20A90F5
:10100400387F0026002800D03DE215467C68002C7D
:1010140005D07869884207D000F03EFA33E200290F
:1010240002D0D948461E2EE2012670020990787F2C
:10103400002815D13868002810D1012181F31088C7
:1010440009981230D14900F049FD3860002181F33C
:1010540010883868002801D10120B8610120787710
:10106400002C089632D10A9800780021796153281F
:1010740003D03A2803D1032027E0022025E02846A4
:101084000A9C214600F006FCBF494E1C002800D5EE
:10109400F9E120460830BE49102206F0ABFE0C9060
:1010A40020463230BB49082206F0A4FE07950546C7
:1010B4000C9805435434B8490522204606F09AFE9C
:1010C4002843079D089800D1DDE17860BE69002DB2
:1010D40000D1D4E1002E00D0D1E1387F002800D027
:1010E400CDE10898C0430290EA4BBA6809981146CA
:1010F400841A1234AC4200DB2C46002C13D038681E
:1011040040180A9E3146224605F020F8B8680119B5
:10111400B9602D1B36190A96B869002802D0002040
:10112400B86063E1DB4B78680328089E00D1A9E02E
:10113400022800D050E138680B900C46002C00D1F6
:1011440072E100270B98C05D01460939172907D8B9
:1011540032468A401A4203D07F1CBC42F2D14AE193
:101164000795E11B032900D86AE1532800D06CE1FC
:101174000C940B98C6197578B41C0691022120466C
:1011840000F0D4F942000699091F914200D262E1AD
:10119400294630390A290799BE4B00D346E1342D3C
:1011A40000D143E1069204950396311D0191002676
:1011B400059005460221204600F0B8F986196D1EF7
:1011C400A41C002DF6D1FF24B4430B9806994018B3
:1011D400C019861C0221304600F0A8F98442079DFC
:1011E40000D041E1049833280B9615D032280C9A8C
:1011F40022D03128089E32D10421019800F096F9BA
:10120400014603980830059CE21E00F0B9F90298E3
:1012140044430C98001926E00821019800F086F94F
:10122400014603980C30059C621F00F0A9F902984E
:1012340044430C9800190EE006210198164600F06C
:1012440075F9014603980A30059C221F00F098F9AD
:10125400029844433019C01B811E089E05E0029881
:10126400059941435018C01B811E8A4B874FB869AA
:101274008C1E00D1C2E00B99891C0B91002800D16F
:101284005CE7BBE0079538680B900D46002D00D154
:10129400AEE00C9500240B9D285D01460939172901
:1012A40008D832468A401A4204D0641C0C98A042E2
:1012B400F2D19DE00C99091B0491082900D8C1E0E2
:1012C4003A2800D0B8E028190690451C0221039161
:1012D400284600F02BF905900698C01C042100F064
:1012E40025F901900698C01D039900F01FF90246E4
:1012F40004990939059840000490801C814200D269
:10130400AEE0052A1CD803920598071D0026022189
:10131400284600F00BF986197F1EAD1C002FF6D16C
:101324000B980499401800190930022100F0FEF8C6
:101334007142C9B28142554F089E039A00D097E08A
:101344000E2A069800D995E00930C0467A441279ED
:10135400520097440771112723278F8F8F8F8F8F08
:101364008F8F2700FA683969019BC91812048918FC
:10137400059A00F005F915E0049900F0D7F800018A
:1013840038610FE0D0FFFF1FF5FEFFFF88950100D5
:10139400FB9601000C97010082950100049900F06E
:1013A400C5F8F8600298059941430C9842180C92CC
:1013B4000B3AB869A242374B09D0151B0B9A049912
:1013C400521812190B320B92002800D15EE70C99C7
:1013D4000C1B0B3C079D11E03A68786900242346F6
:1013E40000F004F9002800D5B861BC60294B12E074
:1013F4000024079D01E00024244FB86900280AD185
:10140400002C07D0B868011B38684118224604F044
:10141400DBFE204BBC60BE69002D30D0002E2ED1E7
:10142400387F00282BD160E60024E6E71848C01C6A
:10143400164FB8610D46EEE700F02EF8002410E0D8
:101444000C4606E0079D049CD7E700F025F8114BF5
:1014540000240E4FCDE70D4F079D0E4B0C9CCCE79F
:101464000C9C079D0B4BC8E7084F0948B861BDE7C2
:10147400074801E00648C01CB861079DB6E77869D3
:1014840009994018786130460DB0F0BDD0FFFF1FB8
:08149400F5FEFFFF13008000CC
:10149C0010B5114C607F002804D0207F002803D0A9
:1014AC00A06910BD002010BD01202077A069002884
:1014BC0007D0FF210C314118012909D800F0C6F9D9
:1014CC00EEE700F073F9002803D40020606160603F
:0C14DC0010BDA06110BDC046D0FFFF1F76
:0C14E800014880697047C046D0FFFF1F1C
:1014F400B0B50D4C607F002814D000F0D7F92068F7
:10150400002808D0012181F31088206800F0FAFA3D
:10151400002181F31088002520222046294607F067
:0C15240067FC6560B0BDC046D0FFFF1F33
:10153000B0B5002920D00246002013781C46303C6C
:10154000E5B20A2D0DD31C46613CE4B2052C01D84E
:10155000573B05E01C46413CE4B2052C09D8373B1B
:101560001C46521C491EE3B20001C0180029E4D1F8
:10157000B0BD0248024981610020B0BDD0FFFF1F0D
:04158000F8FEFFFF73
:10158400F0B58BB0002A2DD015460E4607460196BD
:10159400202D02952C4600DB202403AD00973E4607
:1015A400274602213046FFF7C1FF28707F1EB61C74
:1015B4006D1C002FF5D10C4880690028029D019E06
:1015C400009F0FD103AA01233046214600F00EF8F4
:1015D400002805D460003F18A6192D1BD7D101E0BF
:0C15E400014988610BB0F0BDD0FFFF1F73
:1015F000F0B585B01E46012300939D023B4F7B7CD6
:10160000002B01961FD1049103901446012181F310
:1016100010882E4680363649304600F061FA386030
:10162000002181F31088386800285DD04119796065
:101630000021324607F0DEFBFF2002303882019E97
:101640002246039804993B7C002B07D000233B746F
:101650000346294C2340BB60FE6040E00491BB6818
:10166000E918491E8842029203901FD9304600F0C3
:1016700047F8224800680468002C06D03A68B86829
:1016800029463346A04700282CD40098387438687F
:10169000002631462A4607F0ADFB786831462A46D7
:1016A00007F010FC029A0398049914E02946C41A22
:1016B000386800192E1B04998E4200DB0E46114635
:1016C000324604F045FD78682146324607F0CCFBEF
:1016D0000499029A0398891B92193018019E0029D7
:1016E000B1D1002005B0F0BD0248FBE7540B00204B
:1016F00015970100FFFEFFFF00FCFFFF840C002098
:10170000F0B585B002900120019087020025284E97
:10171000039507202A460240EB087168CB5CD34052
:10172000DB076A1C002B01D015463CE0BA423C4660
:101730000DD02A46541C23460340E6088E5DDE4049
:10174000F30704D1521C7B1E9342F3D13C4603980D
:10175000002809D117480068C06800280199039142
:1017600002D0804701980390631B124800684668C6
:10177000002E04930AD00E498868401909684A1956
:101780001946029BB047049A094E07E0084E30689C
:101790004019FF211A4607F02DFB049A706829466C
:1017A00007F062FB2546BD42B3D305B0F0BDC0468D
:0817B000540B0020840C002002
:1017B800F8B5254F787C00280FD078680126B40248
:1017C800002107220A40CB08C35CD340DA0706D1C0
:1017D800491C8C42F5D100251FE0002532E01B484A
:1017E8000068C068002802D08047002829D4F8681B
:1017F800FFF782FF154800680568002D08D0B86813
:10180800FB683A682146A84700281AD40F480068A0
:10181800C1680029DFD0884705463E74386800262D
:101828003146224607F0E2FA78683146224607F048
:1018380045FB002D06D4054800684069002801D002
:10184800804705462846F8BD540B0020840C00202C
:1018580070B50D4E707C00280CD0306801218C02C8
:1018680000252946224607F0C1FA70682946224613
:1018780007F024FB054800688168002901D08847E3
:1018880070BD002070BDC046540B0020840C0020A1
:1018980080B5044A12689269002A01D0904780BD39
:0818A800002080BD840C00202B
:1018B00010B50E4C607C002816D00D4800680069F9
:1018C000002800D080472068002808D0012181F33B
:1018D0001088206800F018F9002181F3108803486F
:1018E0000021142207F086FA10BDC046540B0020D8
:0418F000840C002044
:1018F40010B584B072B612484178491C4170002476
:1019040010492046FCF7E2FAF7F7E0FE04F01AF873
:10191400F7F782FE022002900320400201900A4958
:101924000091081809490722094B04F005FB0948EE
:101934000121017005F03FFB204604B010BDC046F4
:10194400500E00202143341288F9FF1F9E9301009A
:0819540025E10000490E00200E
:0C195C00014800687047C046880C00205D
:0C196800014800687047C0468C0C00204D
:10197400B0B50C4605461D4804F03AFA002D04D0D3
:10198400286845191A48006802E0194800680546A5
:1019940018490968081818490A682946002A13468C
:1019A40012D08B4203D05B68002BFAD10BE00029E4
:1019B40003D00B6859188142F0D100210C22204633
:1019C40007F016FA0EE00D4600210C22204607F01F
:1019D4000FFA002D06D0256028686060686800282A
:1019E40000D0A060014807F003FCB0BD780B0020D4
:0C19F400880C00208C0C0020900C0020BF
:101A000080B5024804F0F6F980BDC046780B00208E
:101A100080B5024807F0EEFB80BDC046780B002081
:101A2000B0B50D4804F0E6F90C4800680025002820
:101A30002C4608D000210468A14200D30C4640681F
:101A400000282146F7D1044807F0D4FB083C00D217
:101A50002C462046B0BDC046780B0020900C0020DC
:101A6000B0B50446064D284604F0C4F900212046CE
:101A700000F008F80446284607F0BCFB2046B0BD3D
:041A8000780B0020BF
:101A840070B50D460646134804F0B2F912480468CE
:101A94000021002C0BD00F36072296432268B24255
:101AA40007D80DD06268201D002A1446F6D10C46D2
:101AB4000BE0911BA151A11901606068486001E02D
:101AC40061680160266065600834024807F090FB95
:0C1AD400204670BD780B0020900C002014
:101AE00070B50C460546074E304604F083F928468B
:101AF0002146FFF7C7FF0446304607F07BFB204630
:081B000070BDC046780B002007
:101B0800B0B50446054D284604F070F9204607F0A4
:101B18000BFA284607F06AFBB0BDC046780B0020D8
:101B2800B0B50C4605460A4804F060F90720C043E2
:101B38000F340440083D2968A14204D02C602819BC
:101B4800091B00F007F8024807F050FBB0BDC0467B
:041B5800780B0020E6
:101B5C0010B5002206C016490A680838002A23D09E
:101B6C00824201D90B4606E013465268002A01D086
:101B7C008242F9D91B1D426018600868002812D0F7
:101B8C00416800290FD0021D03681C188C4205D136
:101B9C004C6814600968C918016000E00846416887
:101BAC00021D0029F0D110BD0149086010BDC046CE
:041BBC00900C002069
:101BC000B0B50446064D284604F014F9206807F025
:101BD000AFF900202060284607F00CFBB0BDC046DE
:041BE000780B00205E
:101BE400B0B50C460546074804F0CEF807208443F8
:101BF400054804600548056028462146FFF7ACFF08
:101C0400B0BDC046780B00208C0C0020880C00204E
:101C140010B582B0032444430348005D00930123BC
:0C1C240006F086F902B010BDB90C0020DB
:101C3000F0B585B004931546039103210291484302
:101C400013490F5C0A9C002A13D00094384603996C
:101C50002A46049B06F06EF905B0F0BD0122384615
:101C6000214602F007F801460020002EF4D000299A
:101C7000F2D1384602F0AAFB0028E6DC0646002C2A
:101C8000ECD5002E01D13046E6E70298C043E3E7E9
:041C9000B90C00206B
:101C940010B50324444303480019407807F0E2F9DF
:081CA40010BDC046B90C002080
:101CAC0080B5032343430348C018407806F033F94A
:081CBC0080BDC046B90C0020F8
:101CC40080B50321414303484018407802F04AFBA1
:081CD40080BDC046B90C0020E0
:101CDC0080B5032141430248405C02F051FB80BDBA
:041CEC00B90C00200F
:101CF00080B50321414303484018407802F058FB67
:081D000080BDC046B90C0020B3
:101D080070B5044621480178002907D120490022EE
:101D18000A70012101701F4802F0A2FB02F066FB65
:101D28000546182068431C490E182B20FF21315402
:101D38001A48B085A07801210A468240E07881409F
:101D480011433185606802F075FF2F217054104EE1
:101D5800307803214143A078114A505450188570B7
:101D6800E17841700F49284602F01EF8002D03D093
:101D780000200C4902F018F80B480C49002202F028
:101D8800CFF93078411C317070BDC046390E002043
:101D9800380E0020B91E010040040020FFFF00009B
:101DA800B90C0020B91D0100AC0B0020051E010074
:101DB80010B50178012441291AD14178012917D198
:101DC800C178090280780818820B03D07F2040026E
:101DD800014000E081020748007838224243064863
:101DE80080180161002401222046214601F0D6FE18
:0C1DF800204610BDB90C002008F0FF1FB1
:101E0400480708D40448007838214143034840185F
:101E14000121C90201617047B90C002008F0FF1FBD
:101E240080B582B0694600220A8002788A704078C0
:101E3400C870034801900846FFF764FF02B080BDF4
:041E4400A593010061
:101E480080B582B0032141430548401880780121BC
:101E5800009104490022044B01F0F8FA02B080BD59
:0C1E6800B90C0020B4930100306A0100A6
:101E740080B50322424303488018407802F0C4FA34
:081E840080BDC046B90C00202E
:101E8C0080B5032242430348805C012201F0ECFE42
:081E9C0080BDC046B90C002016
:101EA40080B5032242430248805C01F047FF80BDB5
:041EB400B90C002045
:0C1EB8000148002101707047390E002025
:101EC4000349097838224A4302498918086170474E
:081ED400B90C002008F0FF1F0B
:101EDC003022424301488018C160704780090020BD
:101EEC00302242430148801801617047800900206C
:101EFC0010B53024444303480019407807F0B6F875
:081F0C0010BDC0468009002051
:101F140010B582B0302444430348005D009301238C
:0C1F240006F006F802B010BD8009002095
:101F300080B5302141430248405C02F027FA80BD61
:041F400080090020F4
:101F4400F0B585B006464148017800290FD101213A
:101F540001703F4800256022294606F049FFE84306
:101F64003C4908603C4805703C4802F07BFA3C4818
:101F740001F02EFF02F03CFA05463A4901F00EFF4B
:101F84001827384603956843B178012201928A40A4
:101F9400354D28352A522C1881204000A08002207B
:101FA400E0703248A060324802F046FEE07102F070
:101FB4001FFA3278019C2146914004967378264694
:101FC40022469A400A4302904743EA53EC190025FB
:101FD400A560A5800A20E070264802F02DFE224963
:101FE400E071E0200858002809D004680095022117
:101FF400039D28460A460B46A0472C4603E08D71F4
:102004001D488880039C144D287830214143049B4B
:1020140018780F4A50545718587878709978B970CE
:10202400314602F02FFAF004E12149027960B860E8
:102034000298B884BC82163710490A22384604F044
:1020440085F82878411C297005B0F0BD3B0E0020AE
:1020540080090020940C00203A0E00204122010047
:1020640085200100DD200100400400208D210100B5
:10207400A29D0100E2930100020200009E9501006E
:1020840070B50446124D2868002820D4072918D1B9
:10209400302141430F484618204605F0BBFF7060CD
:1020A4002079307260797072A079B072F168002979
:1020B40001D0301D884700200146024601F070FD22
:1020C40002E0002002F016F80020C043286070BD32
:0820D400940C0020800900209B
:1020DC00B0B582B00446007961790902081800F0A5
:1020EC00AFF80125002843D46178203903293FD863
:1020FC007944097949008F44010519291F49086061
:10210C00002535E0302141431B48451869682C46B1
:10211C002634204606F0F0FFA87A2C216854288932
:10212C0068850721002520462A461FE030214143BF
:10213C00114840180169002914D0A27801231340DA
:10214C0001A803709207D20F42700AE0302141437C
:10215C0009484018016A002904D0A078E2781202DC
:10216C0010188847002501222846294601F014FD45
:10217C00284602B0B0BDC04680090020940C002057
:10218C00F8B50C4600F05CF80746052620463146AB
:10219C00009606F0D5FF24252046294606F0D0FFF0
:1021AC000021204606F0CCFF11200101204605F04D
:1021BC003DFF2046314606F0C3FF2046294606F077
:1021CC00BFFF0121204606F0BBFF0321204606F08D
:1021DC00B7FF3020784316490E18715D204606F083
:1021EC00AFFF0421204606F0ABFF2046294606F03F
:1021FC00A7FF0221204606F0A3FF062720463946FA
:10220C0006F09EFF2046009906F09AFF20462946CC
:10221C0006F096FF2046394606F092FF317D2046A7
:10222C0006F08EFF715D204606F08AFFF8BDC046B1
:04223C0080090020F5
:0C22400001480021017070473B0E002097
:10224C00B0B50146084803780022D043002B08D0D3
:10225C00064C143425888D4204D03034521C9A42DA
:10226C00F8D3B0BD1046B0BD3A0E00208009002056
:10227C0080B50848FF210F2206F0B6FDE020064984
:10228C00064A0A500648002202700120887105484F
:10229C00888080BD030E002040040020406A0100AD
:0822AC003C0E0020EF020000CF
:1022B40070B5094C25786D1C2570ECB2032C0AD836
:1022C400049D05266643054C3419641FE170207192
:1022D400A5702270637070BD3C0E0020030E0020B8
:1022E400F8B50C460026184FBD192979814203D050
:1022F400761D0F2EF8D1F8BD0821204606F024FFE4
:102304000B21204606F020FF2979204606F01CFF09
:10231400E978204606F018FFB95D204606F014FF60
:102324006978204606F010FFA978204606F00CFFD5
:10233400287918214143054840182F21415C204643
:1023440006F002FFF8BDC046030E00204004002042
:10235400B0B5417802781202511889B201241C4A9E
:1023640091421ED01B4A914230D11B4DA97802796B
:102374008A422BD18178002928D18079002825D15F
:10238400184800240470184804706878214601F045
:10239400A1FE2878214601F09DFE01222046214617
:1023A40012E00D49897802798A420FD18178002997
:1023B4000CD18079012809D108480078411E0848C9
:1023C400017001210024224601F0EAFB2046B0BD41
:1023D400FEA10000FF210000000D00203F0E0020A0
:0C23E400400E00203E0E00203D0E0020A8
:1023F00070B5417802781202511801240E4A9142B8
:1024000018D101794079000245180C4E307801F05E
:102410006BFA854204D0707801F066FA854209D1E2
:1024200007480078012805D10024012220462146D2
:1024300001F0B8FB204670BD01020000000D002035
:042440003D0E00202D
:1024440010B582B013460A460146044800780024B9
:10245400009405F06DFD02B010BDC046000D0020D3
:1024640080B582B0044800780021009101230A4617
:0C24740005F05EFD02B080BD000D0020F0
:1024800070B504462A480178002929D1012101703C
:10249000284800250322294606F0ACFC0920420109
:1024A0002548294606F0A6FC24482022294606F0A5
:1024B000A1FC23480D22294606F09CFC214840221D
:1024C000294606F097FC20480570204805702048F2
:1024D00005702048057020480560204801F0C4FFC1
:1024E00001F088FF05461E4901F05AFC1D481E49AF
:1024F00001F066FC182068431C490E182B200821A7
:1025000031541B48B085207801210A46824060780A
:10251000814011433185174802F090FB2F21705400
:1025200020786178034A957009020818108070BD00
:10253000430E0020000D0020A4050020CC0A00203E
:10254000120E0020C30D0020400E00203F0E002080
:102550003D0E00203E0E00209C0C00202D3301007B
:1025600055230100B80B0020F12301004004002096
:0825700006500000A8950100CF
:10257800F8B50F490A78482353430E4CE254551CCA
:102588000D70E118009110310346F0CBF0C1F0CB8B
:10259800F0C1F0CBF0C1C16A009C616401680B68AE
:1025A800011D10469847204605F050FCF8BDC0466E
:0825B8003F0E0020A4050020E5
:1025C000F8B500280BD0284800780024800749D5AA
:1025D0007D20800006F0B6FD01F0F4F942E02348CA
:1025E0000678214D2C7801F0CFFF214F3968401A31
:1025F00061B200290AD47D2189000024884231D9A2
:102600002878C1071AD101F009FF2BE01A49884246
:1026100012D348207043174908184121425C297899
:10262000002A19D0890702D54130002101701348D2
:1026300000210160012415E0002413E048217143CA
:102640000C4A5118402201238B54802108432870E2
:1026500001F09AFF386005E04022002484547E2077
:10266000014029702046F8BD410E0020420E002096
:10267000980C0020A4050020E90300009C0C002019
:10268000F0B59DB0044652490878012803D10020D6
:1026900008705049086001F0FBFD0327384002280C
:1026A00000D0C2E04C4E3078002803D0012006F064
:1026B00049FD31E349484078002C05D04849402283
:1026C000642306F0D9FC09E00021CC4344494022B0
:1026D000234606F0D1FC002800D193E0002800D169
:1026E00097E01F2800D085E03E4D3D491F22284637
:1026F00003F02EFD284605F08FFC3B4988427CD133
:102700003A48001D291D0422079203F021FD6C7B2D
:1027100037480078A04200D856E12846083005F036
:102720007BFC01460C20049028560223012200283D
:102730000993184600D410460892002900D1084693
:10274000029048235C43F94806193269EC7B00206B
:102750002E2C0691039300DD90E0112C00DC9DE00F
:1027600021461A39102900D9F8E208230593890077
:1027700001A35B5801469F46C5280100C9280100F6
:102780006F2D01006F2D0100C92801006F2D010080
:102790006F2D01006F2D01006F2D010093280100A6
:1027A0006F2D0100492901006F2D01006F2D0100DF
:1027B000BD2701006F2D0100A52D01003078526862
:1027C0000DAC214690471635284606F0AFFCAEE02A
:1027D000C00C00209C0C00203D0E0020000D0020AD
:1027E000C30D0020CC0A002055534243120E002096
:1027F0003F0E0020002800D558E70120307000F07F
:10280000C5FD89E2DD48407800210A46234606F0EE
:1028100033FCDB480068002800D17DE2002420461C
:10282000FFF7CEFE002800D177E2D64800270770D8
:10283000D5480770BC480078FC43002813D0C54D2C
:1028400041353E462F70A100491909192C390968F4
:10285000C969002903D0F0B28847B34800784835E9
:10286000761C8642EED3C6480068002802D00120BC
:10287000FFF7A6FE0120C54908704EE2A72C1BDC1D
:1028800021464339172945D801228A40C0490A42C6
:1028900040D01635284606F049FC14E0002C37D00D
:1028A000032C0FD0082C00D061E2307852680DACB8
:1028B00021469047E97C3BE0BC2C14DCA82C2DD0B1
:1028C000BB2C28E0E87C0221292C05DD2A2C34D001
:1028D000BE2C32D0A82C02E0082C2ED0282C099136
:1028E00005902AD030E0BD2C00D12DE2BE2C00D0C6
:1028F0003DE2307852680DAC2146904715352846A8
:1029000006F00CFC014613200001A288101810E00C
:102910000146D9E72F2C0146D6D028E230785268FC
:102920000DAC214690471535284605F06AFB014657
:10293000A08848430221012208923122B25C002A79
:1029400000D1104609910590764D2E460836002498
:102950003046214606F0D6FB2C730898002809D093
:1029600006990846099A10436D4D20D186480026E5
:1029700006702AE06A4904980856002800D516E136
:102980008868002800D112E17C4E707801F0B4FB19
:102990007078382460437F4D2818007A002800D1D1
:1029A00017E1012006F0CEFB70786043F4E70029C0
:1029B00001D1022A05D0002900D0B1E1012A00D0BE
:1029C000AEE17148012101700026687B0A96297BDF
:1029D0002A46802529400891482141435D484018F6
:1029E0000990D47B122C1FD0032C79D16A480DA9F1
:1029F0003CC83CC100880880002E00D122E1099D1E
:102A000068780DA98870688888815C4800780024FF
:102A100000940123324605F08DFA0A990A94C0B257
:102A2000461A701E864115E1242E344600D3242414
:102A30003B48123006F07AFB844200D30446002C57
:102A400000D1FDE005943648417C0691067C0DAC32
:102A50000021242720463A4606F0CCF94F490822A7
:102A60002046049203F074FB30200999085C207022
:102A7000F00700D0C1E00698002800D0E5E00DAED8
:102A80003546083520211C22284606F0B3F909985E
:102A9000406C0468204603F053FB0246082800D32C
:102AA000049A2846214603F053FB099D686C44684C
:102AB000204603F045FB0246102800D31022304682
:102AC0001030214603F044FB686C8468204603F014
:102AD00037FB0246042800D3079A20363046A5E08B
:102AE000099D284605F0B6F900285ED06B6B002BD7
:102AF00008D00B490F310AAA284698470646FF28F6
:102B000000D0A7E02E2C00DD16E120461A38102850
:102B100000D95CE106A14000085A40008744C04645
:102B2000CC0A0020120E00203F0E0020A405002039
:102B300051011C009F009F0089019F009F009F0082
:102B40009F0099019F00D3019F009F005A019F00A1
:102B5000FF01C046A40500201148C47C3C40AA687F
:102B6000002A02D028782146904764007C44A4883B
:102B70006400A74417002D0217002D02000D00204D
:102B80009C0C00203D0E00203E0E0020C00C0020BA
:102B900089C0800008F0FF1F70710100A69D010030
:102BA000CC0A00204120012114E201265AE0FD4E0A
:102BB000307801F0A1FA307838246043FA4D2818B3
:102BC000007A002805D0012006F0BCFA3078604376
:102BD000F5E7F648407BF6490978884207D2039921
:102BE0004143F448401820214180052141700120D3
:102BF000FC49087300F0A0FB8EE00698802824D1E1
:102C00000DAE2120F0707570301D202529462A4612
:102C100006F0F0F80998406CC468204603F090FA7A
:102C20000246202800D32A46B01A2430214603F059
:102C30008FFA0DA80122059C2146FFF703FC0A9E8E
:102C4000301B0A900026099D04E0099D6F80052035
:102C500068700126F0B2012804D0002859D100265E
:102C60006E806E70DF4806730A990029DA4F1CD017
:102C7000DC48083006F046FA387801F03DFA08984A
:102C8000002812D1300610D0787801F035FA787823
:102C900038246043D14D2818007A002805D001203F
:102CA00006F050FA78786043F5E7CF4D2878800732
:102CB0000DD4287840071BD42878C00702D0022002
:102CC000C849087300242C7000F036FB25E07878A2
:102CD00001F012FA787838246043C04E3018007A38
:102CE0000028E6D0012006F02DFA78786043F5E759
:102CF000387801F001FA387838246043B74E30183C
:102D0000007A0028D8D0012006F01CFA38786043F9
:102D1000F5E70120B3490873002420461DB0F0BD3B
:102D2000029B022B27D1002A25D1AF480422027032
:102D3000304606F0E7F947E62F2C00D1FCE05A2C8C
:102D40003FD0A82C46D08AE71735284606F0EEF982
:102D50000699814200D9F6E50846F4E5122C06D121
:102D6000E97C0698884200D301460591ECE50020F5
:102D700001460890A8E502201146414043400B431C
:102D80005A425A41002B069B059944D18B4242D9A5
:102D900095480C4604210170191B304606F0B2F923
:102DA000264612E6307852680DAC2146904716351B
:102DB000284606F0BBF90146A08848430121089146
:102DC000BBE50AA9284600F0EDFA064642E7082CC2
:102DD00000D044E70898002800D140E72869069011
:102DE00042687F48C47B28780DA907909047002649
:102DF000A82C00D1FAE0282C00D102E1082C34469E
:102E0000059600D008E1764C2046113006F08EF988
:102E10000590E47C00E108900846591A4B1E0D46C7
:102E20009D4101235A40154300D0C5E06E48002162
:102E3000CBE001266A68002A00D162E16848C17CC3
:102E400031404220285CC00700D058E10846904736
:102E500057E13120285C002800D19FE00A9D002D19
:102E600000D1EFE609990869426808780BAC214661
:102E700090470DAE1021304606F03CF90B99301DFD
:102E800006F038F901277806A1880918304608307D
:102E900006F030F90B9930460C3006F02BF9A1887A
:102EA0003046103006F026F94B480078002100919A
:102EB000142D00D3142531462A463B4605F03AF836
:102EC000C0B2461B28E03120285C002866D00A9D4D
:102ED000002D00D1B6E609990869426808780BAC64
:102EE000214690470B98411E0DAE304606F002F980
:102EF000A188301D06F0FEF83748007800240094C1
:102F0000082D00D30825012331462A4605F012F882
:102F10000A990A94C0B2461A701E864193E6089830
:102F2000002800D09BE63820285C002800D1FFE074
:102F30002720688007208BE6F94C607C00268007FC
:102F400000D487E62869079028780690204611303B
:102F500005F057F805901634204606F0E7F80028EB
:102F600000D177E60346079886680BAA069D284697
:102F7000059C21460393B04706460798C068049015
:102F80000B9A284621463346049CA047002800D1CE
:102F900042E11120099D68806F705AE63A206880EE
:102FA000022055E6000D002008F0FF1FCC0A00208B
:102FB0003F0E0020A4050020069D854200D2234636
:102FC0001A4300D0A7E0D74801210170069E5DE1B9
:102FD00041200021295442E6000D002008F0FF1F87
:102FE000CC0A0020120E00203E0E0020CC4C2046C1
:102FF000113005F006F805901534204605F001F86B
:1030000009E0C74C2046113004F0FBFF0590163450
:10301000204606F08BF804460A98002800D119E6ED
:10302000002C69D00DA9898803F04EF8A04200D386
:103030002046002879D003900D980599814200D34D
:10304000DBE0EC68002C06D0039800900121079883
:103050000A46059BA04709980C3001900021029177
:103060000D460399A9422BD905982C184B1B06989D
:1030700086680BAA07982146B04706460DA8002E81
:103080001CD08088002819D00698C06804900B9A3C
:10309000079821463346049CA04700280ED19F483C
:1030A00000780DA98C880B999F4A009274430023E5
:1030B000224604F03FFF7119A042D1D001200290B6
:1030C00001980468002C06D003980090012100228A
:1030D0000798059BA0470398401B0DA98988414389
:1030E0000A910298002800D1ACE51120099D688062
:1030F0006F70FFF7B7F9ACE500260A96AAE52878C5
:1031000090473020285C052800D1A8E5242068805D
:1031100005206870A6E5029A022A70D1099B012B4E
:103120006DD1804805210170AFE000200A9090E544
:103130002C697B48113004F064FF079005946268A5
:1031400028780DAC069021469047A4880A9D284611
:10315000214602F0B9FF0490A54200D272E507981B
:10316000049909180D98814200D982E0079981429B
:103170007FD20998C468002C06D0049800900021E2
:1031800001220698079BA04709980C300290002660
:1031900035460498A84200D8ADE0431B0598046961
:1031A0000BAA069803950799A04705460DA88488A1
:1031B0006C435A4840780B9922465B4B05F054FF0C
:1031C000A04200D092E003982C1807994118059866
:1031D000406903900B9A06982B46039DA847002848
:1031E0002546D6D0099840780126002803D10999B0
:1031F000481C07704F8025467DE021203BE0012AD6
:103200003BD1099A002A38D14649089808703046BF
:10321000069905F077FF38E0059D404840780DA9F4
:103220004022002305F020FF402820D10B980DA953
:10323000402204F0E1FD002819D10B9840300B909A
:10324000761EEAD1079886680BAA069C2046294676
:10325000039BB04706460798C06804900B9A204627
:1032600029463346049CA0470028D6D091E6012683
:10327000E9E42120099D6880E9E4029A012A08D145
:10328000099A022A05D1274807700026244DFFF726
:103290009CFB0122099B5340029C54401C43634207
:1032A0006341002C0BD1069C0598844207D91D4A26
:1032B00008981070304605F025FF059EE6E7481E89
:1032C00081415340194300D1B0E500260698059985
:1032D000884200D232461343114D01D0FFF775FBEF
:1032E000104801210170069EFFF76FFB039D0998AE
:1032F00047804770012602980468002C06D0049885
:103300000090002106980A46079BA0470498401B9E
:103310000DA9898841430A9195E4C046000D00201B
:0C332000CC0A00203E0E0020B80B00007C
:0C332C000148002101707047430E002092
:10333800B0B582B0104C1149204605F0DFFE0021DF
:103348000F4D28780023C9070AD000930D22214683
:1033580004F0ECFD0D280CD00121401CF1D108E04F
:10336800D94300910D22214604F0E0FD01210028F7
:10337800E7D102B0B0BDC046120E002055534253EB
:04338800000D002014
:10338C0010B5044C207800F0B1FE607800F0AEFE71
:08339C0010BDC046000D002029
:1033A400F0B587B00C46054604AF781C0B263146B1
:1033B40002F0D8FE0820F8703E702348407C3F217C
:1033C40001403F2901D0002934D12168002937D098
:1033D40087093820285CC00104AEB07028782969B8
:1033E4004A6802AD294690470299301D05F080FED7
:1033F400A9880836304605F07BFE25680C2D00D3DD
:103404000C25002F06D004A900200870012F01D13B
:1034140004A9C8710D4800780023009304A92A4622
:1034240004F086FD2168491B2160C0B2401B411E87
:10343400884106E02420688005206870012000E0AF
:10344400002007B0F0BDC046CC0A0020000D0020CB
:10345400F8B51E4600920D46074613480178002928
:103464000CD101210170114800245422214605F099
:10347400BFFC0F4804700F4800F0F4FF0C480178BB
:10348400022910D8069A1C234B43084CE754491CC4
:103494000170E01846608260C560009901611430D3
:1034A400054900F08BFCF8BD450E0020380A0020C9
:0C34B400440E002069370100C134010003
:1034C000F0B58DB004460178602008400126402800
:1034D00027D0002800D03BE16078062800D037E1F3
:1034E000E078032800D033E1A078EE2800D02FE167
:1034F000A679E7790AA801F0B1FB0446994912259B
:103500002A4602F025FE944800782074380281197A
:10351000122900D329460122204600F043FB002651
:1035200016E18D4800786178814200D010E1207961
:1035300061790902081880B2052868D0042800D0F3
:1035400006E1A779E47909A801F088FB0546099A04
:10355000002105F04FFC099A0AAE3046089529462D
:1035600004F065FD7D4D2878182141431031304627
:10357000079105F0F5FD012006900102304604F0A8
:103580005BFD0421304604F057FD2978304605F0F4
:10359000DDFD07250AA80026314605F0D7FD6D1E82
:1035A000F8D12002C01905906C480078002820D07E
:1035B0006B4D1C277743E95D0AAC204605F0C6FD3C
:1035C0000121204605F0C2FDEF19F968204605F0FB
:1035D000B7FC3969204605F0B3FC06240AA800218F
:1035E00005F0B4FD641EF9D1761C5C480078864273
:1035F000DFD30026079905988142069A00D3324608
:10360000814200D30146089800F0CCFAA0E0A078EF
:1036100008900AA800250C22294605F0EBFB4F482C
:1036200000780126002800D192E04D4F089A3978A1
:10363000914204D01C376D1CA842F8D188E0854225
:1036400000D385E07868002800D181E009A801F066
:1036500005FB0146099A0AAD2846029104F0E7FCF1
:103660007E68BF680A98019000212846079105F0FE
:1036700077FD01200102284604F0DEFC05212846E2
:1036800004F0DAFCF9B2284604F0D6FC0397002FC8
:103690004DD03068089070680490B7680696F56859
:1036A0000A9805900AAE0021304605F059FD3046D3
:1036B000089905F055FD02223046049905F06AFC90
:1036C0000898401E052823D8784400794000874494
:1036D000020208161F020AA80322394605F05AFC06
:1036E00016E00AA8294605F03BFD002D10D03978D8
:1036F0000AA805F02BFD7F1C6D1EF8D108E00AAD6D
:103700000421284605F02CFD3968284605F028FDDF
:103710000C98059A80180A99891A05F0F3FC079904
:10372000491C069E1036039807918142B1D10C982E
:10373000019940180A9905F0E5FCA079E1790902A0
:1037400009180A98814200D3014601220298E4E652
:1037500030460DB0F0BDC0464B0E0020440E002098
:08376000380A0020B6950100B3
:0C3768000148002101707047450E002050
:10377400F0B585B00C4606462F490D780020072D7C
:1037840058D8049000A86CC0D8200F58A578A66813
:10379400B8698047010701D5022201E08007C20F02
:1037A4003046294605F074FC0246A17802290546F4
:1037B40000D03546964200D83546FB6C002B03D02A
:1037C40003956078984706E00398C00731D10395C4
:1037D40060787A68904705460498002D2AD0FF2D1A
:1037E40028D0382202995143144846180021304603
:1037F40005F0FEFA03993180A078B0717180A08839
:10380400B0806078C1012943F171002803D1009888
:10381400F06101983062084A1078411C11700F2D34
:1038240008D863786900C918521845218900505492
:1038340000E0049805B0F0BD4004002008F0FF1F2C
:10384400F0B585B014460E4607460A9D03290CD0F0
:10385400022E0CD1D8201049085880690193804762
:10386400019B010705D5022005E0402206E0002265
:1038740004E08007C00F400008490A5A02A98C805E
:103884008E704F700020087004921A462B46FFF782
:103894006FFF05B0F0BDC0464004002092800100D7
:1038A40080B5D8200549085880698047010701D5AB
:1038B400022080BD8007C00F80BDC04640040020A8
:1038C40041060AD00107C90E0006C00F401804497A
:1038D400081845218900405C704700207047C046A5
:0438E400400400207C
:1038E8003821414301484018C079704708F0FF1F4C
:1038F8000248807A8007C00F7047C0464004002005
:10390800F8B5D820094E3558307802280AD3084C23
:1039180038340127A9682046884738347F1C307816
:103928008742F7D3E8688047F8BDC04640040020C6
:0439380008F0FF1F75
:10393C00F8B5592086001A4C0027204639463246E5
:10394C0005F052FA572080000125690221520B2004
:10395C00400114492150280213492150C620134913
:10396C00215225705C3612483946324605F03CFA35
:10397C0000F09EFDF4F77EFCD82026582120C000D4
:10398C002158002901D10B492150706D002800D01D
:10399C008047716900208847054908806572F8BD29
:1039AC0040040020F5930100C57E0100320C00009C
:0839BC0008F0FF1FCB7E0100A3
:1039C400B0B582B0D8200A4D2C5820688047226CAC
:1039D400002A06D06946002008700220904700980B
:1039E40028721020A8722069804702B0B0BDC0467A
:0439F400400400206B
:1039F800F0B58BB0089317460A91382209904243D4
:103A080063498C1800F0B4FD207A0325EE430128A1
:103A180001D1761C1EE05F48807A2840022818D120
:103A28002069002816D11099627E01231A40C80720
:103A380015D00A98002812D1002F10D1606A0028EA
:103A480008D105920496022008400026524A0A929C
:103A58002EE0F61C00F080FD30460BB0F0BD002FC4
:103A680007910496069301D0059201E00120059084
:103A780020461C300A993A4605F0BEFA0646B84276
:103A8800059A05D002200799084010D0002E0DD0C5
:103A9800002ADFD0206A616A401A21888842D9D377
:103AA8000023142103971A461F4615E00799069B21
:103AB800002803D02288BA4201D201E000233A4606
:103AC8004807039203D4971B0A98821904E000223E
:103AD800059800281746BDD0059706930A920791C6
:103AE8002046103023460C33C4212A4A575A7F1CDB
:103AF80057520A990190016000200290D8730698E5
:103B08009873059A62616781207E00280DD120464E
:103B18001830012303700798800600D5029AD82030
:103B28001C4B1858C36A099898470798C00691D43F
:103B380026460A36143400F00FFD32880899002909
:103B480011D0099800F0F2FC0028049E1149039A4C
:103B580014D0079880060ED40021099800F0BEFB07
:103B6800039A0C490AE00998114600F0CDFC049E1E
:103B78000849039A02E00198029B03602068897A49
:103B88002940022901D0F61C66E7161A64E7C046E8
:0C3B980008F0FF1F40040020460E002033
:103BA40080B5074BD8611962012058769A750020B8
:103BB4009882D821034A5158096B884780BDC04672
:083BC40008F0FF1F400400207F
:103BCC00F0B583B00E4604462548807A03210840A0
:103BDC00CD43022808D13820604322490F18387A87
:103BEC00002803D06D1C38E0ED1C36E001920293E6
:103BFC0000F0BCFC797E002909D0C800C0194369CB
:103C0C0082699B18B3421FD0032901D123E03846A7
:103C1C001C3039461931C422114DAB5A5B1CAB52C6
:103C2C002A460660019D45600298B8757B8108782C
:103C3C00401C0870F868002500280CD1D8201058BA
:103C4C00016B2046884706E0183001995118016035
:103C5C000298B875002500F07DFC284603B0F0BD35
:083C6C004004002008F0FF1FD6
:103C740070B51646044638206043184A10180722C7
:103C84008256002A12D40269002A16D042890029D9
:103C940015D0204600F04CFC002814D00125002E3D
:103CA40012D00021204600F01BFB0DE020463246D6
:103CB40000F018F8411E884170BD00250CE0204634
:103CC400114600F023FC00250548807A03210140B9
:103CD400022901D00020C543284670BD08F0FF1F0B
:043CE4004004002078
:103CE800F8B51646044638206043124A1718F86893
:103CF800002802D1787E002819D000253D767A89DF
:103D080000290FD0204600F011FC002810D03846BA
:103D180004F062F90546002E0AD00021204600F082
:103D2800DDFA05E02046114600F0EEFB00E0002534
:083D38002846F8BD08F0FF1F4A
:103D4000F8B50D4604463820604314490F1800F0BA
:103D500013FC787E032812D3002D12D4012038766C
:103D60003E46183600F0FCFB7A892046002D0CD028
:103D7000294600F0DFFB0446401E844109E0002490
:103D800000E0012400F0ECFB05E0114600F0C0FB70
:103D90000024002030702046F8BDC04608F0FF1F08
:103DA0001822424301488018816370474004002074
:103DB0001822424301488018C16370474004002024
:103DC00010B5C022024B9C5898500460416010BD51
:043DD000400400208B
:103DD40010B50549CA7B032A05D89300CB18C8241B
:0C3DE4001851501CC87310BD4004002092
:103DF000F8B50C4605464869002802D0A07E002888
:103E000011D06189284600F06DFB00272761607E94
:103E10000126C00708D1D82004490858816A2846DD
:103E20008847277600E000263046F8BD4004002091
:103E3000F0B583B014460291002853D005463820CF
:103E4000684332490F18FA68002A02D002982146C6
:103E500090473869002824D001953D46143579698A
:103E6000A142264600D82E68002E11D039461031C6
:103E700000910299324602F06BF9009908688019A6
:103E800008602868801B2860029880190290A41B93
:103E9000019D28463946FFF7ABFF002801D00926CF
:103EA00000E00126002C18D038461C30029922462A
:103EB00004F00CF8797EC90702D0398888420CD208
:103EC000387E002809D03C461834D82010490858BC
:103ED000816A28468847002020703846314604F021
:103EE00050F811E00A4EF07B00280DD03746C83755
:103EF00000253A68002A03D0029821469047F07BBB
:103F00003F1D6D1C8542F4D303B0F0BD08F0FF1FC8
:043F10004004002049
:103F1400F0B585B007463820784348490C18607ED0
:103F2400002800D188E026460C36002F03D03168E3
:103F3400002900D080E000210291E175022805D318
:103F4400206A002802D1204604F026F822461932BD
:103F54002546203523461C33D82039490858016D9D
:103F64000029019222D0A08A0490039111781A4664
:103F740004AB38460092039FB84707460498A082D2
:103F8400002F32D4781C30602E68B742039706D9CC
:103F9400204604F001F8BF1B2E68B742F8D8F01B86
:103FA400286000990868C019086028E02A682188F8
:103FB4008A4200D30A460392511C316019681E4696
:103FC400436B3846039A984703982968091A29606D
:103FD400316809183160002804D02188194A8A18E8
:103FE400024205D00298A08209E00120306023E05B
:103FF40002F068F8A18A0818A082012003902046E4
:1040040003F0DDFF2868002816D1019908780228FA
:1040140003D3204603F0C0FF0EE00398002809D024
:10402400A08A002806D0A07D002803D01634029868
:10403400207001E00298087005B0F0BD08F0FF1F81
:0840440040040020FFFF000012
:10404C0070B50446382060431E490D18002C10D062
:10405C00E86802280DDB28460C300021C9430160BA
:10406C00E87D002801D0042100E00621284603F059
:10407C0082FF0020E860687E00280FD02E4619369B
:10408C002046FFF741FF307802281AD8287E0028F6
:10409C0017D06989204600F01FFA70BDD8200A4954
:1040AC000858816B20468847002C08D06989204627
:1040BC0000F012FA4021284603F05DFF70BD00F0BD
:0C40CC0063FA70BD08F0FF1F40040020E4
:1040D80080B538224243044B9A181172D822034BF8
:1040E8009A58126A904780BD08F0FF1F40040020CC
:1040F80080B538214143054A521801211172D8224E
:10410800034B9A58126A904780BDC04608F0FF1FBB
:04411800400400203F
:0C411C00D821014A505070474004002098
:1041280010B5416082604D218900084B5A58002A19
:1041380005D01446844206D02468002CFAD1585081
:104148000260002010BD012010BDC04640040020C0
:104158008B604A603822424302488018426B4163B0
:084168000A60704708F0FF1F18
:1041700010B50D480021C172827A0278022A07D355
:104180000A4B4033012419703833641C9442FAD32B
:10419000417B01220A404273817A10200840083096
:1041A00000F006F810BDC0464004002008F0FF1FD4
:1041B000F0B587B00446D827334EF059B57AA542FA
:1041C0005FD0022123460B402940002B2CD0002930
:1041D0002AD102930391049000950194FFF794FB78
:1041E0003078022810D3294C403401250021217059
:1041F000F059026A28469047284600F013FD3834EB
:104200006D1C30788542F1D30498026C002A019C21
:10421000009D0399029B07D005A90120087000208A
:104220009047029B03990498002B08D1002906D0DF
:10423000026C002A03D005A9002008709047B472D0
:10424000274625436807800F0CD03078022809D311
:1042500001250020C143284600F044F86D1C307849
:104260008542F6D34D2080003458002C09D03D46BD
:104270006268002A02D0A068294690472468002C72
:10428000F6D107B0F0BDC0464004002008F0FF1F83
:0C4290000148807A7047C04640040020BE
:10429C0080B5D8200549085880698047410701D569
:1042AC00022080BD0121084080BDC0464004002092
:1042BC0080B50348817A01200843FFF773FF80BD66
:0442CC00400400208A
:1042D00080B50348817AFE200840FFF769FF80BD62
:0442E0004004002076
:1042E400F8B50D460446D8201C490F5838206043C1
:1042F4001B490E18002D01D500203072002C2BD044
:1043040000F038F907203056002811D439463746D2
:104314001837307E002802D0896A2046884700205A
:10432400387030611027002D0AD57062B06207E042
:10433400B96B2046884700207076F060B082202751
:1043440000F00CF93046394603F019FE002D03D075
:104354007189204600F0C4F8F8BDC046400400202E
:0443640008F0FF1F3F
:104368000649897A03220A40022A05D138214143A5
:1043780003484018406A70470020704740040020F6
:0443880008F0FF1F1B
:10438C0010B5382141430648441800F0EFF8204698
:10439C0003F020FE044600F0DDF8204610BDC046B8
:0443AC0008F0FF1FF7
:1043B00038214143044840180169002901D040696F
:0C43C000704700207047C04608F0FF1F47
:1043CC0010B53821414307484418607E002802D0BC
:1043DC000020C04310BD204603F0EDFDA08A411E15
:0843EC00884110BD08F0FF1F1D
:1043F40004494878182242438A182E23D054421C78
:084404004A70704740040020DB
:10440C003822424301488018C160704708F0FF1FF2
:10441C00B0B500F0ABF8D8200F4D2858806C0028B0
:10442C0000D08047F8202858002800D08047A97A6F
:10443C00E9200840FFF7B6FE2878002808D00024B1
:10444C0001212046FFF748FF641C28788442F7D3EB
:0C445C0000F080F8B0BDC0464004002015
:10446800E421064A5358002B04D0091DF829F9D134
:1044780001207047505000207047C046400400207B
:10448800382242430348801807228256002A00D463
:084498004176704708F0FF1F98
:0C44A000DC21014A50507047400400200D
:1044AC0011210901014A50507047C04640040020B8
:1044BC0070B50025064C074E7319042101222046C5
:1044CC0003F0D4FD18342D1D202DF5D170BDC04640
:0844DC00C4070020EC0A0020D7
:1044E40010B582B00191182141430748441801A92D
:1044F400204601F02DFC002803D0204601F09AFB51
:0C450400F5E702B010BDC046C40700205F
:10451000B0B582B00C46182141430548451801A9A1
:10452000284604F051FE0198A042F8D102B0B0BD77
:04453000C40700209C
:1045340070B582B014460D4618214143064846180A
:1045440001A930462A4601F0B9FB002802D101999D
:0C455400A142F5D102B070BDC4070020E8
:1045600004484178491E41704078002800D07047C7
:0845700062B67047500E0020F6
:1045780072B602484178491C41707047500E0020BD
:0C4588000148006A7047C046500E002039
:10459400B0B50B200B4D2C56002C00D4B0BD7F20A1
:1045A4000440EC72D8202858C16920468847A87A6C
:1045B400002C02D00421084301E0FB210840FFF74E
:0845C400F5FDB0BD400400202C
:1045CC00F0B587B00446C020AE490D58002D07D079
:1045DC00696820468847002800D118E12D68F5E766
:1045EC00D825A84B5E592078602101401AD020298B
:1045FC0049D0402900D008E15878002800D104E1C6
:10460C001D463C3500272968002906D020468847DE
:10461C00002800D1FBE09B48407818357F1C87426E
:10462C00F1D3F2E061780B2940D8490079448988AC
:10463C0049008F440B004200EA004400EA004900A4
:10464C005900EA00B900C100CD00DD00A1780029B5
:10465C0000D0DAE0E178002900D0D6E0A179022977
:10466C0000D0D2E0E179002900D0CEE00F21084043
:10467C00022800D124E2012800D133E2002800D026
:10468C00C3E0597B38E220795978884200D3BCE0EA
:10469C00182141437B484018816B002900D1B4E0BC
:1046AC0020468847002800D0AFE0B0E0302900D188
:1046BC00AFE0312900D1C8E0A7E0002100E00121E2
:1046CC00204600F029FAA2E0A478187A00281D46AA
:1046DC0000D1A2E0F16920468847A87A002C00D1CD
:1046EC00AAE004210843A9E0E078411E0E2900D974
:1046FC00D2E100204900C0467944898849008F44A2
:10470C000E00F200A700CB01CB01C300E500CB01EA
:10471C00CB01CB01CB01CB01CB01CB01F60080202F
:10472C000590FA4D0695FFF7B3FD064601226A7017
:10473C001220287002200190049057208000F1492B
:10474C00085A21210901884200D801460392022E01
:10475C0000DB014604A803F069FC05990498E94BB9
:10476C00884206D21979069A11540498401C049078
:10477C000599884206D25979069A11540498401C1E
:10478C0004900599884206D29979069A1154049896
:10479C00401C04900599884200D3E6E0012E00DD10
:1047AC00DDE0DB490978DBE0FFF7A0F804AB18701B
:1047BC0001210022184680E1A078002833D001287E
:1047CC0023D11C4603F045FCA17A0220084330E0BB
:1047DC00A078002819D1A079012816D1987A062141
:1047EC000140062911D104A800220270012164E1C4
:1047FC00987A06210140062907D1217958788142FF
:10480C0003D8E078002800D17CE0706A804707B0BC
:10481C00F0BDBD4801210170F9E78020044303F08D
:10482C0018FCEC72F3E71C4603F013FCA17AFD2094
:10483C000840FFF7B7FCEAE7FB210840FFF7B2FCA2
:10484C00B048C472007A0128E1D103F002FCDEE723
:10485C00A078042800D9D0E0AE4AC046784400794C
:10486C004000874402D2D7DCEA00A84F0420F8703D
:10487C000921B970032179703870802104AA83C290
:10488C0000E1C04640040020FFF706F89D4B0028CD
:10489C0000D101E1FFF7FCFC9A4B012800DDFBE0A5
:1048AC009A4F0220F8700020B870062179700A2106
:1048BC00397078720120387218793871587978719A
:1048CC009879B87192480078F871E8E0FEF7E4FF47
:1048DC008C4B002800D1DFE0FFF7DAFC894B022873
:1048EC0000DBD9E0012000F0D5F9884FCFE029207A
:1048FC00C0001858002800D1CEE08047814B0746F5
:10490C000120C0E002900391A078019003F0A1FB7C
:10491C007C4A1078022815D3012400262046314603
:10492C001746FFF7D3FB7859C16B002901D02046FD
:10493C008847F1432046FFF7CFFC641C714A10787E
:10494C008442EAD3432080001258002A00D15EE74B
:10495C0002980002019941180398904757E70921E2
:10496C00069A11540498401C0490112005015859C2
:10497C00018804AE30461F4603F058FB0295785967
:10498C004188304603F052FB039D2802385880477B
:10499C000146304603F04AFB05990498884205D23B
:1049AC0006990D540498401C04900599574F2B46BA
:1049BC008842544A06D20699019D0D540498401C15
:1049CC0004900599029D5259D268002A04D088425D
:1049DC000AD20699032203E0884205D206990022E6
:1049EC000A540498401C04900599884257D20699A1
:1049FC000B540498401C049051E0411F9A7B914247
:104A0C0012D288001818026915E0112000011858FC
:104A1C00426810E011200001185882680BE0112048
:104A2C0000011858C26806E0FC21595800290ED024
:104A3C008847344B0246002A09D01078002808D049
:104A4C00501C0026815D761C0029FBD102E000275A
:104A5C0018E000262D4F032078707000801C3870F1
:104A6C0080200590069702200490002E0AD0117821
:104A7C0004A8174603F0DAFA3A467A1C761EF6D1E9
:104A8C00204B224F0020002F06D0002807D0B81C46
:104A9C0004F04CFB014603E05859406AB6E63978FD
:104AAC00A079E27912021018814201D3002200E0B1
:104ABC000122814200D301463846FFF76DF8A6E685
:104ACC002079997A890702D4002800D09DE600F05D
:104ADC00C5F8002800D598E6382141430C48401809
:104AEC00017A09E0987A800700D48EE6587821790B
:104AFC00814200D389E600210448002242700170F3
:104B0C000221DAE740040020470E0020030D0020AC
:084B1C0008F0FF1FC89501001D
:104B240070B582B00C4605460078A978EA7812027E
:104B3400511800281DD18AB2022A1AD1002C18D08B
:104B44006A79002A15D0042A19D8FFF7A5FB002892
:104B540015D0D824304E3059006C00280FD003F003
:104B64007CFA6879694608703059026C04209047D1
:104B74000AE0AA79002A02D1EA79002A06D0D820CC
:104B840025490858406A804702B070BD0F22104082
:104B940002281FD10A041DD1287900F063F80028E7
:104BA400EDD433D005461C4EB07A8007E7D5E1B288
:104BB4002846FFF78FFA002C2AD1D8203058C16B31
:104BC400002901D0284688470020C1432846FFF722
:104BD40087FB1DE0002809D18AB2012A06D10E48BC
:104BE400417B002C0ED0022211430DE0552292008D
:104BF400094B9B58002BC2D089B222469847002803
:104C0400BDD1C1E7FD221140417301E003480472A4
:104C140003F023FAB8E7C0464004002008F0FF1F61
:104C240080B5D821034A5158C96B002900D0884760
:084C340080BDC04640040020D1
:104C3C00064A917B052901D9002005E04B1C937392
:104C4C008B00D2181061481DC0B270474004002080
:0C4C5C008021016000487047030D00201B
:104C6800B0B5014640060FD0094803780022D0436A
:104C7800002B08D0074CE41D25788D4206D0383427
:104C8800521C9A42F8D3B0BD0020B0BD1046B0BD4A
:084C98004004002008F0FF1F9A
:104CA000F0B585B02F4F0025FD70BD7009263E7010
:104CB0000421B971012179710190002801D00720E8
:104CC00000E002207870284C6078387180200390D2
:104CD000217B0143F9710497FFF7E0FA012802DC18
:104CE0002046C63001E02046C730224600783872A0
:104CF0000296607800282ED01446E0201058002834
:104D000003D0426802A92846904718206843221819
:104D1000283202A82946019B00F028F82246A078F4
:104D2000002812D016468C360027311F09788D4294
:104D300007D102A829463246019B00F017F8224607
:104D4000A0781C367F1C8742EFD36D1C50788542BB
:104D5000D3D3029E034FB81C314604F0DBF905B0F3
:0C4D6000F0BDC046030D00204004002000
:104D6C00F0B587B0059315460391074610880021CE
:104D7C00400803D0012202405118F9E705CF083F43
:104D8C00904206D2BA68092313543868401C386024
:104D9C007A68904206D2BA68042313543868401CCF
:104DAC0038607A68904206D2BA68039B135438680C
:104DBC00401C38607A68904206D2BA68AB781354BB
:104DCC003868401C38607A68904205D2BA68115431
:104DDC003868401C38607A68904206D2B968EA7824
:104DEC000A543868401C38607A68904206D2B96818
:104DFC002A790A543868401C38607A68904206D286
:104E0C00B9686A790A543868401C38607A689042EC
:104E1C0005D2B968EA790A543868401C3860AA6827
:104E2C00002A02D0039839469047FEF735FD0090D2
:104E3C00FFF72EFA01904C480078022800D290E03F
:104E4C0001260198301A0290484C3834B002069072
:104E5C0004952888F040C0077CD003CF083F8842D7
:104E6C0006D2B96807220A543868401C3860796841
:104E7C00884206D2B96805220A543868401C38604A
:104E8C007968884206D2B968E2790A543868401CBD
:104E9C0038607968884209D2617A0C220A40A1797B
:104EAC001143BA6811543868401C38606088059901
:104EBC00002904D0A179029A04F0E6F807E00099E1
:104ECC00019A914202DDA17904F0DEF82080069966
:104EDC00884200D3069881B2384603F0A7F8A5881B
:104EEC00FFF7D6F9002801D1E91DCD08002D00D11E
:104EFC000425A179032905D0012905D002280ADB54
:104F0C0000250DE0002808D00020401C29044D0C81
:104F1C00FBD1054604E0012502E0FF2D00D3FF255F
:104F2C0003CF083F884204D2B9680D543868401C3E
:104F3C003860532080000C490A58002A02D02046C1
:104F4C0039469047049DEB68002B03D0E179039818
:104F5C003A469847761C383403480078864200D28B
:104F6C0077E707B0F0BDC0464004002008F0FF1FF3
:104F7C00F8B5FFF7FBFA2948002404700471047299
:104F8C000473274D2C702C712C722C732C742C7573
:104F9C002C762C77234E3470347134723473347411
:104FAC0034753F21C94372186023D454091DFAD1BA
:104FBC001D4AC02111701472147314751746FF2109
:104FCC00297001702972BB202871BF202873DC2046
:104FDC001649095816488847402038701548164914
:104FEC00081816490140164F39602C763868012193
:104FFC0000910A02214603F0F7FE3868000A287770
:10500C0078883074F878307500F0B0FA009828750C
:10501C00102005490872FFF79DFAF8BD10200740D3
:10502C0080200740A02007400021074040040020BA
:10503C00C1530100FF01000000F2FF1F00FEFFFF43
:04504C00A00C002094
:1050500070B5044601252E468E4000F0E5FA00208A
:1050600009490A78002A05D14A78164202D08A787E
:10507000A24205D0401C891D0828F2D1FF2000E083
:0C5080000D70C0B270BDC046C60C002010
:10508C0007214056002801DA152100E019214006BD
:0C509C00C00D014A81547047C02007403D
:1050A80080B50448842101702120C00002490858B5
:0C50B800804780BD1C2007404004002001
:1050C40010B5062141430348441800F0ABFAA08808
:0850D40010BDC046C60C00200F
:0C50DC00014908707047C046982007404A
:1050E80010B50C46FEF7FCFB4006C00D0549425CB6
:1050F800002C02D002231A4301E0FD231A40425437
:0851080010BDC046C0200740A5
:1051100009480068094901408220094A105CC0071B
:10512000000F0818842303608320105CC007000F61
:10513000081803617047C046A00C002000FEFFFF66
:04514000000000204B
:1051440080B500280AD0FEF7CDFB7F2101408820DE
:1051540048430349081884210122425480BDC046B3
:045164000000002027
:10516800B0B500280ED0FEF7BBFB7F210140882098
:105178004843124A10188422002383548522825CF3
:10518800002A00D0B0BD034685338222845C812288
:10519800825C01251D70A301C018094B1B68094DCD
:1051A8001D40E3071B0F0907C90D59184919486025
:1051B8009001054A02430A60B0BDC04600000020C5
:0C51C800A00C002000FEFFFF880040004B
:1051D40080B5FEF787FB7F210140882048430549BD
:1051E40008188121002242548021425485214254CE
:0851F40080BDC0460000002050
:1051FC00034801787F220A40027000207047C046A5
:04520C001C2007401B
:10521000F0B58BB00693099203910446FEF764FB48
:105220007F21014008914801012637023D46E035C3
:105230000540FFF7A1F95B4800685B490840049509
:1052400028180169802211408069400038404018C8
:1052500000210791B84205920ED0802815D0002871
:105260001CD1882008994843504908188321425C82
:105270000792425C724006E08820089948434B49F7
:10528000081883210122425408E0882008994843E5
:105290004649081883210022425407963825654361
:1052A000FFF75EF94248465B09994868B0423446C8
:1052B00000D80446002C39D00968CA0E032A029689
:1052C0000A9407D30A0F022A04D8039A012A3BD072
:1052D000B04239D28820089A5043344A1018079AAD
:1052E000920185182846224600F032FF361B0195B0
:1052F0002BD00398022828D32F19099D0835401E6A
:10530000099068688642344600D3044629683846C6
:10531000224600F01DFF0A9820180A90361B14D070
:105320003F1908350998401EEAD80EE01D4800686C
:105330001D4908400799C907090F049A0A43024307
:1053400010201043002710E001911648006816490C
:1053500008400799C907090F049A0A43024310201D
:10536000104301994160029E0A9F8821089B4B438C
:105370000E4AD218059D535D9B013C04E3180B4374
:105380000360505D012141405155B74203D1069A57
:105390001168491C01E00021069A116038460BB0E3
:1053A000F0BDC046A00C002000FEFFFF0000002062
:0453B00008F0FF1FE3
:0C53B4000148002101707047C40C00206B
:1053C000F0B585B0674D297828790840010733D4B6
:1053D000C4B2E00705D00120287000F0CDF8FEF738
:1053E000C7FEE00603D510202870FEF767FFA00671
:1053F00003D520202870FEF76BFFA00703D50220FD
:105400002870BF202872600701D50420287020066C
:1054100000D4A5E080202870287C0F2800D99FE0C8
:105420005148006851490140524880300860886006
:1054300000200861886193E02A7C4B4800684B4952
:1054400008401409630118185107CE0FF700C0195E
:105450000168120722D404938906090F0391026898
:105460001206FCD488226243414B9D188122AB5C1A
:10547000012102914B40AB542A4681320068002C36
:10548000039901921FD10D291DD10299117080201D
:105490002954B0012818FFF799F82BE01021084390
:1054A00000210160012046408820604330490818EF
:1054B00083214654002C00D080342046FEF702FAA7
:1054C000FEF7C4FD4AE0012914D18001800D03904C
:1054D0002046FEF7F7F9852100226A543146029AE8
:1054E00051408222A954039A002A03D0B1016918BD
:1054F000FEF79EFC1C4800681C49084004990843BC
:10550000074300213960002C06D08422AA5C002ABF
:105510000AD0843529701CE0164878300199097842
:1055200089010143396014E08521029A6A5482217D
:10553000695C8A01AA18C907090F01434A600198EA
:10554000007880010B4A80180860086880220243B6
:105550000A60044D287DDF2101402975082028704C
:1055600005B0F0BD80200740A00C002000FEFFFF2A
:085570000000002008004000CB
:10557800F0B582B0244A1078022101431170234CFF
:1055880083341F20C643002213460196224805682B
:10559800204805401D432A600827284638430260F2
:1055A80010202946009001430A6018210D432A6003
:1055B8001748351820202A54227001980019C277FC
:1055C8004277827788342033361DDFD10E4B187826
:1055D800FD2202401A70104802680E4802400B482B
:1055E80050601743403078600C4810603860009C69
:1055F8001443002020600A4310600D21044A1170F2
:10560800187102B0F0BDC046942007400000002089
:10561800C020074000FEFFFFA00C002088004000CB
:10562800F0B50F480178002919D10E4940228A8027
:1056380003238B70FF2402340C800A31DB430124DE
:10564800254607267602CE520A80CE186F1C2540C2
:10565800B570891D082F3D46F3D101210170F0BDB9
:08566800C40C0020C60C002058
:1056700010B572B6084C6178491C617000210C228B
:1056800003F0B8FB6078401E60706078002800D09E
:0C56900010BD62B610BDC046500E0020D8
:10569C0070B50C46054672B6094E7078401C707099
:1056AC0000210C22284603F09FFB7078401E70707E
:1056BC002C727078002800D070BD62B670BDC046E8
:0456CC00500E00205C
:1056D000B0B5044672B6104D6878401C6870012061
:1056E0006060206800280DD000F008F9204600F026
:1056F0008FF8002804D1207A012801D000206060B2
:1057000000F004F96878401E68706878002800D0BE
:0C571000B0BD62B6B0BDC046500E002017
:10571C0070B5044672B60F4E306A6268002A0AD120
:10572C004518482120462A4600F0BCF8B068C068ED
:10573C0085420CDD72B6207A012801D00020606011
:10574C0071780020002900D070BD62B670BD0120B8
:08575C0070BDC046500E002094
:1057640010B5044672B60068002805D0C06800F081
:105774000DF872B62068F7E703484078002800D097
:0C57840010BD62B610BDC046500E0020E3
:10579000B0B58268002A09D01C49096AC16006CAEE
:1057A000002900D04A60002383601160017C03223D
:1057B0000A40027400D0B0BD144C2169002903D006
:1057C0004B6942699A4206D920612078002810D09E
:1057D0000120607114E08142F7D09A42EBD1034678
:1057E0001B68002B0CD05D69AA4209D18B42F7D10E
:1057F000EAE701202070204601F0EFFB0020207036
:1058000060780028D7D162B6B0BDC046500E0020E7
:1058100070B5044672B60F4D6878401C68702068F9
:10582000002600280CD0C068017C490704D5296AED
:10583000C2688A4200DC0126FFF7AAFF2068F0E771
:105840006878401E68706878002800D162B6F0B2AF
:0858500070BDC046500E00209F
:1058580010B584B001900290094A9368039372B618
:1058680003686C4604600093002B01D068465860BA
:10587800906801746946816000F004F804B010BDB6
:04588800500E00209E
:10588C00B0B5074C25782078401C2070204601F0DC
:10589C009EFB25706078002800D0B0BD62B6B0BD0C
:0458AC00500E00207A
:1058B000B0B584B0019002900F4CA368039372B608
:1058C000A368DA60256A95420FDA02686C460460C4
:1058D0000092002A01D06846506068469860042013
:1058E00001431974FFF7D2FF03E06078002800D16C
:0C58F00062B604B0B0BDC046500E0020EF
:1058FC0002480178491C01707047C046500E0020C8
:10590C0010B50D4C2078401E20706068217800295D
:10591C000FD100280DD072B66068002806D0012087
:10592C002070204601F053FB002020706078002886
:0C593C0000D010BD62B610BD500E00205F
:1059480010B500F07BFB08480121017000F084FBD2
:10595800044603F04FFC021B212A04DB203ACD2128
:0C596800204603F043FA10BD500E002052
:10597400F0B583B08C4C002767700126267072B690
:10598400E06B002804D08047382027546763E7631E
:1059940062B600F063FB0078CD2802D07D2000F0D1
:1059A40061FBA568002D11D0296C00290ED0686810
:1059B4000968002900D088476D6C002D06D029683D
:1059C4000968002900D088476D68F6E73120019006
:1059D400205C002832D03020215CA0683C22815415
:1059E400217900292BD072B62771A06862B60028ED
:1059F40023D00268002A20D04369516999421CD1FE
:105A040011461268002A02D055699D42F8D072B638
:105A14002269824201D0036801E0036823610A46D7
:105A24003C32456A5D622B6041620B680360002B67
:105A340000D0586208605078107062B6A068029670
:105A4400002805D0017C002902D1816B491C8163A7
:105A5400206900282AD072B62569002D27D02E7C13
:105A6400002E24D070070ED5E868216A884204DD30
:105A7400616A884207DA606205E02846FFF786FE1D
:105A8400287C002812D0FB200640102E09D1A868DB
:105A940080684068017C002903D1696940698842B3
:105AA40004D12868206162B672B6D5E772B660790F
:105AB40067710028029E30D0B007216A081860621E
:105AC400E169002901D02046884762B6E56872B6CC
:105AD400002D1ED02069002804D068692169496915
:105AE400884216D3287C40070FD5E868216A88428B
:105AF40007DC2846FFF74AFE72B6287C002808D047
:105B0400E868616A884200DA606262B62D6872B63B
:105B1400DEE7607967710028CED1206900283CD087
:105B24002069007C256900280FD0A8688068456832
:105B34002968686A01602968002900D048622069E0
:105B440040696861284600F031F8A560286B007848
:105B5400CD2803D0782000F085FAA568002D11D057
:105B6400296C00290ED068684968002900D088474C
:105B74006D6C002D06D029684968002900D088473B
:105B84006D68F6E7A0683C21415C019AA15430227B
:105B9400A154416B491C416303E02786A760277029
:0C5BA40062B6014803B0F0BD500E0020B6
:105BB00070B51A4C2178491C2170E16800290BD07E
:105BC00043694D69AB420ED20A460968002905D0E7
:105BD0004D69AB42F8D308E022460C324262002104
:105BE000016010600DE022460C3206463C364262EF
:105BF0000160106048629D4201D1717800E000218F
:105C00003170017C002906D172B6FFF7C1FD6078C2
:105C1000002800D162B6FFF779FE70BD500E00205B
:105C2000034880680021034A126802644164704797
:085C3000500E0020AC0C002016
:105C380010B50446FFF75EFE72B6A068002809D0CA
:105C48000020A06007484078002800D162B62046AE
:105C5800FFF784FD03484078002800D162B6FFF7BB
:085C680051FE10BD500E00209A
:105C700010B5828A036953434468E45C0C70521E79
:105C80005B1C491C002AF7D181688268521E826021
:105C9000C26803695B1C934200D300230361074B76
:105CA0005B78914205D1002B00D162B6FFF75AFD17
:105CB00010BD002B00D010BD62B610BD500E0020EC
:105CC000F8B50C460546104F386A72B6A968002927
:105CD0000DD18618402128463246FFF7E9FDB86805
:105CE000C06886420DDD72B6A8680028F2D0FFF7C2
:105CF00005FE28462146FFF7BBFFFFF707FE002001
:0C5D0000F8BD0120F8BDC046500E002088
:105D0C00B0B58268C3680469A218D31A00D31A46C6
:105D1C00838A5A4344680D78A5545B1E491C521C57
:105D2C00002BF7D18168491C81608168012902D15F
:105D3C00FFF712FDB0BD03484078002800D0B0BD7D
:085D4C0062B6B0BD500E00204C
:105D5400B0B50C460546FFF7CFFD72B6A868E968F2
:105D6400884205D228462146FFF7CEFF002400E0F2
:105D7400012404484078002800D162B6FFF7C4FD2E
:085D84002046B0BD500E0020C6
:105D8C0010B5044609480A4901600021102220463A
:105D9C0003F02AF872B607480168E160046006480F
:105DAC004078002800D010BD62B610BDB00C0020A9
:0C5DBC00C95D0100A40C0020500E002066
:105DC800B0B5044608480568002D0CD0287A00288C
:105DD80007D06868A04204D101202872284600F044
:0C5DE80029F8ED68F0E7B0BDA40C002025
:105DF400B0B50446FFF780FD207A002810D00D4D81
:105E0400A96862688A4209D010212046FFF722FD62
:105E1400207A0028F8D1A86860600020451C03E0BF
:105E240004488068606001252572FFF76DFD2846EF
:085E3400B0BDC046500E002075
:105E3C0070B50446FFF75CFD207A401E2072000608
:105E4C0009D16068002803D041698569A94205D150
:105E5C002046FFF781FCFFF753FD70BD1A49096816
:105E6C00002913D0A1420FD04A6882420CD10A6893
:105E7C00002A09D02B46D5686D699D4200D81D4675
:105E8C001268002A2B46F6D1C968E9E772B6606839
:105E9C0003F08CF90D4E7078002800D162B6606862
:105EAC004561FFF77FFE2568002DD1D072B6E868FA
:105EBC0003F07CF97078002800D162B6E868FFF72F
:105ECC0071FE2D68F0E7C046A40C0020500E002097
:105EDC0010B51548416B00290CD0382101224254D1
:105EEC00427112480468002C03D060688047246813
:105EFC00F9E710BD016A491C826A0023521C8262B8
:105F0C000162C26A5A41C262426A914201DB0121BA
:105F1C0041713021425C002AE3D0521E42541106DA
:105F2C00DFD101210171DCE7500E0020A80C00200C
:105F3C00F0B583B0029315460F4604460021482263
:105F4C00019102F051FF3D200A9921546561A56130
:105F5C0013480078217C01432174099D089E002F71
:105F6C0000D0A762E5622663CD2130462A4602F0B6
:105F7C003BFF701907218843503801210906019A0B
:105F8C000260029AC264074A026441644F21C94309
:105F9C004D31416260602046FFF704FE03B0F0BD56
:085FAC004A0E0020A96F01005C
:105FB40080B508490A78002A03D00A6A8242FCDBC9
:105FC40080BD72B6896804220A74C860FFF75CFC5D
:085FD40080BDC046500E002004
:105FDC0080B50349096A0818FFF7E6FF80BDC04683
:045FEC00500E002033
:105FF000F8B5134D29460CC80CC11CC81CC1C0CD36
:1060000030463946083D00F05FF8044668617D205F
:10601000C500B7422E4607D8284621460E4600F056
:1060200067F800293046F9D12046314600F04CF897
:10603000034CE0612846314600F046F8A061F8BD07
:046040000C0B002025
:10604400EFF3108072B6FF210904034A13680B436F
:0C605400136080F31088704720ED00E01E
:0860600000487047B010002059
:1060680010B50446FFF746FC04480021417062B6AB
:106078000348047001780029FCD110BD500E00209F
:04608800480E00209E
:10608C00CA1751408B1A17D0C1174A4004B4484064
:10609C00411A48081A0000E052008242FCD9002044
:1060AC0000E05208914200D3891A40419A42F8D13B
:0C60BC0004BC5040801A70470020704760
:1060C8000A000FD00300400800E052008242FCD9C9
:1060D800002000E05208934200D39B1A40418A42B4
:0860E800F8D170470020704759
:1060F0000A0010D00300400800E052008242FCD9A0
:10610000002000E05208934200D39B1A40418A428B
:0C611000F8D11900704700207047C0460D
:10611C0010B42024131B07D5A31A91400400DC40B3
:10612C002143904010BC704704009C40210000208B
:04613C0010BC7047DC
:10614000411C02780130002AFBD1401A7047C0463A
:106150008446002A05D00B78037001300131013AE2
:08616000F9D160467047C0460A
:1061680000228446002903D0027001300139FBD196
:0461780060467047C6
:10617C0010B50F2A1BD903000B43541E9B070DD0DF
:10618C00041905E0431C4A1CA34216D01100180048
:10619C0003780A789342F5D0981A10BD03680C68FE
:1061AC00A34204D1043A04300431042AF6D8541E14
:1061BC00012AE5D103780A78EEE743784A78EBE7D1
:1061CC0010B5884209D9002A06D00139441E8B5CCF
:1061DC00A354013A002AFAD110BD8842FCD0002AFF
:1061EC00FAD00023CC5CC45401339342FAD1F3E7C8
:1061FC0010B5002A02D0FFF7BBFF10BD0020FCE752
:10620C00F0B516000F2A30D90400830739D10B02E0
:10621C001D000A0415430B060D431D4333000200F9
:10622C00103B1B091F011032D21925606560A56057
:10623C00E56010349442F8D10F220C2401331B0179
:10624C00C318324034421FD01C00043A9208013269
:10625C009700FF1820C4BC42FCD192009B1803226B
:10626C001640721E002E04D1F0BD0300721E002ECB
:10627C00FAD00132C9B29A18197001339342FBD18A
:0C628C00F2E70300013AF4E71600EFE728
:1062980000000000000000000000000000000000F6
:1062A80000000000FFFFFFFFFFFFFFFFFFFFFFFFF2
:1062B800FFFFFFFFFFFFFFFF0000000000000000DE
:0462C80000000000D2
:0862CC00329701000000000000
:1062D400B3710100C5800100D580010000000000F9
:0C62E400319300000000000000000000EA
:1062F000D19300000594000029950000C5710100AC
:10630000C7710100C9710100D9800100DD80010061
:10631000CB710100CD710100E1800100A595000065
:046320000000000079
:1063240000000000E803000000000000B596000033
:04633400C19600000E
:1063380075980000000000009D9A0000759B000001
:0C634800A19B0000E19B0000419C0000B4
:1063540003777553DB950100000000000000000086
:1063640001777553709401000092010087000000CA
:1063740001777553DE9B0100EA9B01007700000062
:10638400F9A10000E9800100F5A70000D1A50000F3
:10639400E5A7000009A60000F5800100CF71010007
:1063A400929201008C9401000796010096940100DA
:1063B400FFFFFFFFB494010000FFFFFFC69401003C
:1063C400FFFEFFFF99920100FEFEFFFF9E9C01006D
:1063D400FDFEFFFFD4940100FCFEFFFF15960100B3
:1063E400FAFEFFFFAA9C0100F8FEFFFFB69C010025
:1063F400F6FEFFFF22960100F5FEFFFFA8920100C2
:10640400F3FEFFFF2F960100F1FEFFFFE29401006F
:1064140049AC000071AC0000F5A7000091AC00008D
:10642400E5A70000BDAC0000F5800100D1710100BA
:10643400B7920100BE9201003C960100F094010065
:106444007A9C01007E9C0100829C0100869C0100D4
:106454008A9C01008E9C0100929C0100969C010084
:086464009A9C010000000000F9
:10646C00D371010051700100F98001004DAD0000A5
:10647C001181010035810100DD710100EB7101001A
:10648C004D8101001172010023720100C5810100D0
:10649C003D720100DD810100737201007372010015
:1064AC00D371010051700100ED8101004DAD000070
:1064BC007D720100358101009B720100B9720100EF
:1064CC004D8101007372010073720100737201003F
:1064DC007372010073720100737201007372010018
:1064EC000000000031DA000075DC0000D1D20000A1
:1064FC0075D3000065D1000071D20000A5D000005A
:10650C00ADCF0000000000003188010019B200007E
:10651C000DD40000B1D4000000000000F9B300005D
:10652C004D880100000000000000000095B3000041
:10653C00498801000000000000000000897501007E
:04654C000DD7000067
:1065500095C5000075C4000049850100A1850100B2
:10656000F58501005F7301007D7301001D86010048
:0865700039860100AD70010045
:1065780011820100EF720100097301001B73010011
:10658800C5B60000E1B60000EDDE0000158201008E
:106598001182010011B70000518201002D73010022
:1065A800EDE8000081B80000A5B8000011820100E4
:1065B80011820100B982010095B9000041BA0000BA
:1065C8001182010011820100BDBA00001182010090
:1065D800118201001182010025BD00001182010015
:1065E80055BD0000118201001182010011820100D5
:1065F800118201001182010011820100D98201007B
:1066080095BE000051BF0000A1BF000019C90000DD
:106618000DCA00001774010051C00000F18201008A
:106628001F7C0100737C0100117C0100657C010066
:106638002F730100397301004373010011820100B7
:106648001182010011820100118201000183010001
:1066580011820100118201001182010011820100E2
:1066680011820100037C0100577C01000D830100A9
:106678001583010059890100618901001182010017
:1066880089AF00001182010011820100118201000E
:10669800C18601001D8301004D73010091C00000F7
:1066A800A9C0000001C1000011820100118201008F
:1066B8003DC10000118201007DC100003D83010041
:1066C80011820100498301006983010011820100E0
:1066D8001182010011820100118201001182010062
:1066E8001182010011820100118201001182010052
:0C66F8001182010069C200001182010043
:04670400335A6AB8E2
:1067080095C5000075C4000049850100A1850100F8
:10671800F58501005F7301007D7301001D8601008E
:1067280039860100AD7001009B730100F57301000B
:10673800E18401009DC70000000000000000000087
:106748008DCB0000FD8601007B7401000000000075
:04675800000000003D
:10675C004A95010005000000CD870100509501000D
:10676C0005000000D187010018930100060000000D
:10677C00D58701001F93010006000000D987010096
:10678C00EA9C01000B000000DD870100269301004C
:10679C000E000000E1870100F69C010013000000D0
:0467AC00E987010078
:0867B000A5CC000091CD000012
:1067B80000000000010000000300000002000000CB
:0467C80000000000CD
:1067CC0093750100A1750100AF7501006988010086
:1067DC00BD750100CB750100D9750100E77501008D
:1067EC00F5750100F7750100858801005D880100D1
:0C67FC00F975010001D900008D88010032
:106808006F7A0100797A010095E70000617A01004A
:10681800417A010039E7000059E70000E9E6000085
:0868280011E70000058B0100DF
:106830009F7A010057930100BD7A0100369D010047
:08684000DB7A01004A9D010012
:0468480030680100B3
:10684C00F97A0100037B0100218B010061EF00004C
:10685C002D8B0100357001007DEF0000398B01009C
:10686C000D7B010085EF00001F7B0100357B0100D3
:10687C004B7B0100498B0100CD8B0100DD8B0100AE
:10688C0091EF00007DEF00007DEF00007DEF000038
:10689C007DEF00007DEF00007DEF00007DEF00003C
:1068AC00F18B01000D8C0100298C0100617B010032
:1068BC00837B0100458C0100658C0100A57B0100E8
:1068CC00B5EF000049F000006D8C01006D8C0100EB
:1068DC007DEF00007DEF00007DEF00007DEF0000FC
:1068EC007DEF00006D8C01006D8C0100CDF000007F
:1068FC00718C01006D8C01006D8C01006D8C0100A0
:10690C006D8C01007DEF00007DEF00007DEF00003D
:10691C007DEF00007DEF00007DEF0000B37B0100F8
:10692C00C57B01007D8C01008D8C01007DEF00008A
:10693C009D8C0100AD8C0100CD8C0100DD8C010023
:10694C006D8C01006D8C0100CF7B01007DEF000090
:10695C007DEF00007DEF00007DEF00007DEF00007B
:10696C007DEF00007DEF00007DEF00007DEF00006B
:10697C007DEF00007DEF00007DEF00006D8C0100CD
:10698C0015F100007DEF00007DEF00007DEF0000B1
:10699C007DEF00007DEF00007DEF00007DEF00003B
:1069AC00FD8C01007DEF00007DEF00007DEF00000D
:1069BC007DEF00007DEF00007DEF00007DEF00001B
:1069CC007DEF00007DEF00007DEF00007DEF00000B
:1069DC00558D01003D8D0100458D0100358D010067
:0C69EC002D8D01008F7C01004D8D0100FD
:1069F800E9F60000FDF6000011F7000000000000B5
:0C6A080025F70000000000000000000066
:106A140075F50000A9F50000DDF5000001F60000A1
:0C6A240000000000000000000000000066
:106A3000010000008E9D0100BB93010000000000DA
:086A4000B5220100E52201006E
:106A48007D4F0100515001008D5001006D80010003
:106A5800A9500100C5500100AD910100DD500100B1
:106A6800E95001001151010045510100695101002F
:106A7800B1910100000000006F800100D5510100B4
:106A88007180010000000000FD51010000000000BD
:086A980011520100B553010089
:106AA0000D4885460D4C20680434004201D08047D3
:106AB000F9E70B480B49884205D00268043003B45B
:106AC000904703BCF7E700208646EC4600200021F3
:106AD000054A9047FEE70000B0120020B09D01007B
:0C6AE0002A9701002A970100F518010018
:106AEC0016488546F2F7FCFDD4E7FEE7FEE7FEE725
:106AFC00FEE7FEE7FEE7FEE7FEE7FEE7FEE7FEE762
:106B0C00FEE7FEE7FEE7FEE7FEE7FEE7FEE7FEE751
:106B1C00FEE7FEE7FEE7FEE7FEE7FEE7FEE7FEE741
:106B2C00FEE7FEE7FEE7FEE7FEE7FEE7FEE7FEE731
:106B3C00FEE7FEE7FEE7FEE7FEE70000B0120020EE
:106B4C00082148430138FDD57047F0B444464D4602
:106B5C0056465F46F0B46446754630B40A9FB94653
:106B6C000BE0F0B444464D4656465F46F0B46446DE
:106B7C00754630B42C4F3F68B94682468B469446D6
:106B8C001F4680B401246501A60128494B69B34313
:106B9C00984633439E46544620780134A2465C46C0
:106BAC0022780134A346120210430822082F00D584
:106BBC003A46BF1A440802D244464C6106E0082308
:106BCC00C405E40FE340CE5074464C614C460000C3
:106BDC00013CFDD54D604C46013CFDD58D60400817
:106BEC00C046C0460C69A409E4072043013AE1D130
:106BFC00000E644620700134A446002FCBD104BC97
:106C0C00520705D0520F52420832D040013C20703E
:106C1C0044464C6130BCA446AE46F0BCA046A946E6
:106C2C00B246BB46F0BC7047C40B002080F00FF896
:106C3C00F0B5134F402420260823027812060130A9
:106C4C003425520000D204357C51BE63013B7E6377
:106C5C00F6D10139F0D1F0BDF0B5094F80222026D4
:106C6C0008240025BE636D007E633B681B0A00D3BD
:106C7C000135013CF6D1057001300139F0D1F0BD80
:046C8C0090F00F4035
:106C9000012000BD022000BD0A0B9200A358013B59
:106CA000A35002D00A05120EB61AB95B0236CA0604
:106CB000520EA85887460A0552160B0B9B0019590D
:106CC00089181951F1E70A05120F92000B0B9B006E
:106CD000E3580906090F5918A150B95B0236CA06D4
:106CE000520EA858874660B40E0BB600A65901E0B4
:106CF00060B40E0B0B051B0F9B00E5580906490FEE
:106D00008900854808588746AD19E550002D03D104
:106D10000122626460BCC8E70022626460BCC4E710
:106D2000AD1BF2E73540F0E73543EEE77540ECE7A1
:106D3000B540EAE7F540E8E77543E6E70A0B92005D
:106D40000905490EA150B0E70A0B9200B95B023663
:106D5000BB5B02361B040B43A350A6E7626CD20751
:106D600003D5A2E7626CD2079FD509040916490032
:106D700076189AE7626CD207D20F090B890062502D
:106D800093E7CA09530814D2236D9B009A420EDA86
:106D9000E36BF8184906490F8900C918E163390007
:106DA000E36C9A5800F002F820607EE7104702205A
:106DB00000BDE36BF8184906490F8900C918E16363
:106DC0003900BA5B0236D200034B1B689A5800F0B8
:106DD00002F8206069E71047486801008A0603D579
:106DE000E26B043AE263BE50090489154900761843
:106DF0005BE78A0603D5E26B043AE263BE50090BF7
:106E00008900665851E70A05130F9B00E3180A0B27
:106E10009200E06B801A19003B18E0630868186064
:106E200004310433043AF9D13FE70A05130F9B00FC
:106E3000E3180A0B9200E06B39188018EDE7E26B5B
:106E4000D6590432490989005218E2632DE7CA1263
:106E5000D2065216E36BD2188B051B0F9B00490517
:106E600002D5E358D35120E7D259E2501DE720B4B0
:106E70000D052D0FAD00080B8000201803680A06D1
:106E8000120F0B3A626D00D1D20093422DDAFB183B
:106E90004A06520F09061CD5110003D1187860511B
:106EA00020BC02E7012A03D11888605120BCFCE60F
:106EB000022A03D11868605120BCF6E60178490720
:106EC000490F0068C008381800F04AFF605120BC24
:106ED000EBE66059110002D1187020BCE5E6012AEA
:106EE00001D11880F9E71860F7E7022020BDF0B55E
:106EF000A0B0040000AD266C06498022043A8B58ED
:106F0000AB50FBD100F003F8266420B0F0BD00B513
:106F1000A76CCAE6BC0F00203C100020DB207047A5
:106F200038488168002901D108B00ED0EFF30982FA
:106F3000283A0368F8C243464C4655465E4678C236
:106F4000734608C2283A83685A60FEF713FD8168C9
:106F500000291BD04A68143278CAB346AA46A14613
:106F6000984608CA9E46283AF8CA26490B60143249
:106F700082F3098890692449244A884201DB9042BF
:106F800003DB2348034200D162B6704721482249FF
:106F90000968401A80F308882049C161204981614D
:106FA0000621C9438E467047FEF73AFE01BC2046D3
:106FB0001C498E4600BD01F05EF81B481649096861
:106FC000401A20380721884380F3088800210D48A3
:106FD000417062B600F012F8FEE703680CB40021BD
:106FE000417062B61149124A0A60C04672B60CBCC2
:106FF000036070470D490E4A0A6070470B490C4AFE
:107000000A607047500E0020DB6F0100F26F010034
:1070100000FF00009012002020630100000000012A
:10702000E5800100B76F0100B012002004ED00E020
:04703000000000104C
:1070340080B5006800F002F8002080BD08B4024B5F
:0C7044009C4608BC6047C0466D10002050
:10705000B0B50B0B0A05120F0C06640FC90601D45C
:1070600099004358920081588218062C0AD8C046CD
:107070007C4424796400A7440307090B0D0F110019
:10708000C9180CE059430AE0C91A08E0194006E0A3
:10709000194304E0594002E0994000E0D9401160F2
:0A70A0004A424A4142640020B0BD9C
:0270AA0070472D
:1070AC0070B586B004460025059501210491039521
:1070BC00029101AE3046F7F791F830780028284657
:1070CC0030D06D4601212846F7F788F82878001F44
:1070DC00072813D8784400794000874403070B0F26
:1070EC000F0F0F1401A8017805A80FE001A8017873
:1070FC0004A80BE001A8017802A807E001A8007819
:10710C00F7F760F904E001A8017803A8F7F766F82F
:10711C0001AD01212846F7F761F828780028D0D175
:10712C00059D039820632069E1698A6A2946904786
:10713C00FEF7DEFB0120FEF74BFF2069E1694A698F
:10714C00029990470498FEF743FF2069E169C969E9
:10715C0088470446FEF7D4FB204600F062FC06B0DC
:02716C0070BDF4
:02716E00704768
:10717000700000000000000A000000000000000095
:0271800000000D
:02718200704754
:02718400704752
:02718600704750
:0271880070474E
:02718A0070474C
:02718C0070474A
:02718E00704748
:02719000704746
:02719200704744
:02719400704742
:02719600704740
:067198000120C043704716
:0A719E0080B55221F2F72DF880BDF4
:0A71A80080B5D721F2F728F880BD6A
:1071B20010B50446DB0008462146FFF7D7FC002045
:0271C20010BDFE
:0271C400704712
:0271C600704710
:0271C80070470E
:0271CA0070470C
:0271CC0070470A
:0271CE00704708
:0271D000704706
:0A71D200016C891E01640120704762
:0E71DC000A0B92000905490E815000207047F1
:1071EA0010B5C26B0B0B9B00D41AC463846CA21833
:1071FA0089093C240C400019594208C85350091DFA
:06720A00FBD1002010BDC5
:107210000A0B92008358090549165918815000201D
:027220007047B5
:107222000A0B920083585B1E835004D0026C09093A
:0A723200C9B2511A01640020704730
:10723C0010B5012292020A400B093C241C40031990
:10724C00090449160324A143C46B6118806C4018CF
:10725C00002A194600D00146002A00D018460068C2
:06726C000860002010BDC7
:0A727200016C891E016402207047C0
:10727C0010B58A0605D5C26B121FC263036C846CF1
:0E728C00A3500913890041580164002010BD71
:10729A0010B5026C131D0364836C9C5A9A185288A9
:0E72AA0012041219090B89004250002010BD79
:1072B80010B5C26B0B0B9B00D418C463846CA21866
:1072C80089093C240C400019594208CA08C0091D04
:0672D800FBD1002010BDF7
:0272DE007047F7
:0272E0007047F5
:0A72E20072B60020F6F7C7FEFAE7C7
:0272EC007047E9
:1072EE00B0B5F6F71AFE04467025284601F0EDFB00
:0A72FE0020462946F6F78DFFB0BDCB
:1073080080B501F025FB0220FEF764FE01F024FBA6
:0273180080BD36
:10731A0080B501F024FB0220FEF75BFE01F023FB9F
:02732A0080BD24
:02732C007047A8
:0A732E0080B5CD20F4F7DDFF80BD2F
:0A73380080B5CE20F4F7D8FF80BD29
:0A73420080B5CF20F4F7D3FF80BD23
:10734C0080B501200002F7F73DF8002001F0B4FBF6
:02735C0080BDF2
:10735E00B0B504460069E16989698847054600F0C1
:0E736E005FFB681E414241413C202154B0BDEE
:10737C00B0B504460069E169C9698847054600F063
:0E738C0050FB681E414241413C202154B0BDDF
:10739A00B0B582B0044601A80421F6F720FF019D8A
:1073AA00FAF739FB854201D2019801E0FAF733FB7B
:1073BA000190052814D3FAF74EFB054601980023DD
:1073CA000093291D001F82B22046F5F786F928602E
:1073DA00011D2846F6F71FFF2846FAF790FB02E040
:0A73EA00002000F01FFB02B0B0BD50
:1073F400B0B582B0044601AD01212846F6F7F2FE8D
:1074040020692978E269D26B904700F00EFB02B044
:02741400B0BD09
:1074160010B584B003A801242146F6F7E2FE02A8BF
:107426002146F6F7DEFE0220F6F7CFFF00280CD144
:1074360002A8007803A909780902081801A9F7F734
:0E744600F6FE01990022F5F704FA04B010BD1D
:10745400B0B5044685683F2085430BD02069616838
:1074640008182946F6F786FF206940192061A068AC
:06747400401BA060B0BD4A
:10747A00F0B587B0074606AE02213046F6F7AFFEF2
:10748A00307871788900091D41431F304009059001
:10749A000818FAF7E0FA0446307881000122D54349
:1074AA00002C29D00395651872785043800028185B
:1074BA0004902046F6F793FE06AE70783178414381
:1074CA0089002846F6F78BFE3869F9698F6D31789D
:1074DA0072780091019221462A46049D2B46B847AC
:1074EA00002814D4012000F08FFA2846059901F0EB
:1074FA00DAFA01F0F6FA13E00846F6F764FF06A88E
:10750A004178007848438000F6F75DFF01E0039D6B
:10751A006D1C284600F078FA01F0E3FA002C02D03C
:0A752A002046FAF7ECFA07B0F0BDB6
:10753400B0B50D460446F9F7F5FC002021680A7839
:0E754400AA4202D1491C2160B0BDC043B0BDB7
:10755200F8B5164604460068876C204601F047F9E4
:107562000121CD4300280BD420687B6903213246D8
:107572009847002805D12068B96A8847002500E0AD
:067582006D1C2846F8BD57
:0A75880080B50068F6F79AF980BD9F
:0E75920080B5032008401146F8F779F980BD56
:0E75A00080B5042008431146F8F772F980BD4B
:0E75AE0080B5032008401146F8F76BF980BD48
:0E75BC0080B5032008401146F8F7EEF880BDB8
:0E75CA0080B5042008431146F8F7E7F880BDAD
:0E75D80010B50446F8F7BEF80020606110BD43
:0E75E60010B50446F8F7C9F80020606110BD2A
:0275F4007047DE
:0275F6007047DC
:1075F800F0B58FB00B93002A00D1A5E015460C46D4
:1076080042688168069115990591149E01214B07DE
:107618000C93B14002910321891B039100210A9127
:10762800C9430491089007960699A143F140491C63
:107638008D422B4600D30B460C990A4200D02B46AC
:107648000D93022E099413DB022221460746059B5F
:1076580001F018F9002879D43A680B980D9C214656
:10766800F8F72EFA214600282046079E55D06DE0EF
:1076780021463246059B01F005F9002804984BD4B1
:1076880001F068FB0028049846D10D9802280B9F4A
:10769800099A24D3461E0B9F099A144607200EA95F
:1076A800F8F7F2F8002833D122462046039908401B
:1076B800C0000E99C1400E9139700798002804D077
:1076C8000E98000A7870BF1C00E07F1C089840687C
:1076D8000C99084201D102981218761EDDD1019248
:1076E80003200EA9F8F7D0F800280498079E13D1B4
:1076F800039801990140C8000E99C1400E91397054
:10770800002E0D9808D00E98000A78700D9803E0A6
:10771800F8F732F80498079E0D99002817D40A9AAA
:1077280082180A928842099C12D1B140089842688E
:107738000C9B1A4200D164180D9BED1A0B9B5B1829
:107748000B93002D04D06FE7002000E004980A9006
:067758000A980FB0F0BD1D
:0E775E0080B52C300021202201F045FB80BDBB
:10776C00F0B58FB005464E20285C002800D1A6E06D
:10777C0028464C30002405908470A968002900D15B
:10778C009EE028688847002800D199E06A680026A6
:10779C00F443002A06D0286829461831904700285F
:1077AC0000D58DE02969002904D028688847002875
:1077BC0000D585E001960394A869012800DA84E0DD
:1077CC00284618300A9000210C918800281803468E
:1077DC00007F801E022802D85C7F1F2C06D10C99DA
:1077EC00491C0A9800688142EEDB6EE0D87F059A4E
:1077FC005178401A099011780126A14201D80796B8
:10780C0003E0081B32468240079218461D30029056
:10781C00099886401E330B9300200D900798012881
:10782C0043DB03988840C04308900D9A0998824026
:10783C000494201801210E9181400691002408988F
:10784C00024009981F280DD0002017180721394035
:10785C00FF08EF192C23FB5CCB40D9070AD1401C45
:10786C00B042F2DB06981218641C07988442E6D1E9
:10787C00049C1AE00B9801781F29049C15D0002455
:10788C00EF68002F0AD028680C9900910A990D9A7C
:10789C002346B847002816D40B9801780E988840D8
:1078AC00641C8442ECDB029804780120A0400D9902
:1078BC00491C0D91814292DA05980178AEE70024BB
:1078CC0020460FB0F0BD039CFAE769690029039CC0
:0E78DC0003D0286888470028F2D4019CF0E70A
:1078EA0010B50446806BC168002900D010BD002184
:1078FA00102201F07AFAE069026E002A13D0206998
:10790A0000219047A16B08602069E1690A6E012194
:10791A009047A16B48602069E1690A6E022190478D
:0E792A00A16B886000E0A16B0120C86010BD59
:02793800704796
:10793A00F0B590B00F240325EE43254601272F40CA
:10794A007F421F406D087D40761CF7D3A6006F4624
:10795A00BD51651E002C2C46EDD1037853401A0701
:10796A00920E6C46A2581B0953401A07920EA4584D
:10797A001A096240491E401C0029EED1104610B077
:02798A00F0BD4E
:0A798C0080B5F0F761FD002080BD1A
:1079960010B5FF2912D8002810D0002A0ED053188F
:1079A60001242402A34209D83F23DB02CB18611A23
:0E79B600914200D80A461946FEF7C7FB10BDE5
:1079C40070B5C0B002460024E043002A11D0012360
:1079D4001D02A9420DD16E46304611462A46FEF7D5
:1079E400B5FB3F20C00231462A462346F0F79CFCF3
:0679F400204640B070BD0A
:0279FA007047D4
:1079FC00B0B5002806D00446002508222946FEF71B
:067A0C00FFFB2560B0BD88
:107A120080B582B0019001A8042101F048F802B0BB
:027A220080BD25
:0A7A240080B50021F6F782FC80BD5A
:107A2E0080B582B0019001A80421F6F7F2FB02B0F6
:027A3E0080BD09
:107A400080B5FFF7A8FB1420FEF7C8FAFFF7A2FBEA
:027A500080BDF7
:0E7A520080B50020FFF79CFBF0F7CDFD80BD56
:0E7A600080B50A4601460020FAF720F980BDE5
:0A7A6E0080B50020FAF73DF980BD55
:0A7A780080B50020FAF72EF980BD5A
:0A7A820080B50020FAF71DF980BD61
:107A8C0080B5FCF7FFFB03210140891E48424841A9
:027A9C0080BDAB
:107A9E0010B50268406843180121002410462246A2
:0E7AAE00F7F779FC012800D0E443204610BD14
:107ABC0010B5026840684318022100241046224683
:0E7ACC00F7F76AFC022800D0E443204610BD04
:107ADA0010B5026840684318042100241046224663
:0E7AEA00F7F75BFC042800D0E443204610BDF3
:0A7AF80080B500F09EF8002080BD6C
:0A7B020080B500F068F8002080BD97
:107B0C0080B503684268C8181146F6F783FB00205D
:027B1C0080BD2A
:107B1E0080B50068002802D000F096F801E000F071
:067B2E0069F8002080BD93
:107B340080B50068002802D000F099F801E000F058
:067B44006CF8002080BD7A
:107B4A0080B50068002802D000F087F801E000F054
:067B5A005AF8002080BD76
:107B600010B582B0002401940068012101AB2246C7
:107B7000F7F718FC002801DAE04300E0019802B0B2
:027B800010BD36
:107B820010B582B0002401940068022101AB2246A4
:107B9200F7F707FC002801DAE04300E0019802B0A1
:027BA20010BD14
:0E7BA40080B5F7F79FFC401E411E884180BD52
:107BB20010B50068002421462246F8F772F82046E4
:027BC20010BDF4
:0A7BC40080B5F8F769F9002080BDD4
:0A7BCE00C068411E4842484170475C
:0E7BD80080B50620F7F762FDFFF763FA80BD67
:0E7BE60080B50020F7F75BFDFFF7C8FA80BD01
:0E7BF40080B50320F7F754FDF0F76EFD80BD5D
:0E7C020080B50320F7F74DFDF0F747FD80BD7C
:0E7C100080B50120F7F746FDFFF7B7FA80BDFB
:0E7C1E0080B50220F7F73FFDF0F719FD80BD9D
:0E7C2C0080B50020F7F738FDFFF7A8FA80BDFD
:0E7C3A0080B50620F7F731FDFFF794FA80BD04
:0E7C480080B50020F7F72AFDFFF798FA80BDFF
:0E7C560080B50320F7F723FDF0F72DFD80BD6C
:0E7C640080B50120F7F71CFDFFF78EFA80BDFA
:0E7C720080B50220F7F715FDF0F7FFFC80BD8E
:0E7C800080B50020F7F70EFDFFF77DFA80BDFE
:0A7C8E0080B500F00AFAC0B280BD14
:107C9800F0B583B00D46436881681C46CE1A01D5FD
:107CA80001698E19964200DB1646002E20D007691E
:107CB8000290006801962146C019401A864234464F
:107CC80000DB0446284622460F46FEF73DFA3A19DD
:107CD800029807690068C3199A42014600D0114604
:107CE800361B2D19002EE7D10298C1604160019E14
:067CF800304603B0F0BDB0
:107CFE0010B50446F8F7F7F92822002120460B4666
:067D0E00F8F75DFA10BD5C
:107D14000021425C002A09D01346613BDBB2192BD7
:0E7D240001D8203A4254491C0B29F2D1704775
:107D32005621C9430246303A0A2A01D2273103E0CA
:107D42000246613A062A01D2081870470246413AB1
:0E7D5200062A02D3563108467047373870476C
:107D600007220A40C90840188107C90E8A18032152
:107D700088430168002A06D0D14020239A1A40681F
:0A7D80009040084370470846704722
:0E7D8A0002680B0A53701170911C0160704763
:107D980002680B0ED3700B0C93700B0A53701170A2
:067DA800111D016070478F
:0A7DAE000178407800024018704789
:107DB8000178427812025118827812048918C07822
:067DC800000608187047D8
:107DCE0010B50A781346413B1A2B00D220320378A5
:107DDE001C46413C1A2C00D22033002B03D0491CE8
:0A7DEE00401C9342EDD0981A10BD1E
:107DF800B0B503460020012A08DB0C781D78A5429F
:107E080005D1521E5B1C491C002AF6D1B0BD0120C9
:027E1800B0BDFB
:0A7E1A0080B5002200F0F1FF80BDEA
:107E240080B5002803D4002200F0EAFF80BD404260
:0A7E3400002200F0E5FF404280BD8F
:107E3E00012806DB01461F20401E49000029FBDCFD
:067E4E0070471F20704781
:107E5400B0B504464020205C25463135002804D0C6
:107E6400012000020F21685202E0287C002807D07C
:107E74003A20608002206070002129700846B0BD5D
:107E840020782169896988470121012809D0C2B273
:107E9400002A0ED12A78002A0BD13A2161800221CE
:107EA40005E02A78002A04D1282161800621617026
:067EB40000212870E2E746
:0A7EBA0080B50020FAF7DFFB80BD61
:067EC400012000027047DE
:027ECA007047FF
:107ECC00F8B5164645688368EA1A002E21D00F468D
:107EDC000092C2689B185A1B00D3134604469A1989
:107EEC00AA4200D81546ED1AB54200D33546206893
:107EFC00C01839462A46FEF725F9A0682B18A3604E
:107F0C00009A521B761B04D000927F19656820469C
:067F1C00DFE71046F8BD8E
:107F220080B582B0102300930023FBF764FD02B0FA
:027F320080BD10
:107F3400F8B5054606980090002811D428460F4647
:107F440016461C46FBF740FE011D0DD1284600993C
:107F5400FBF7F4FE0028324623463946EED00CE007
:107F64002846FBF731FEF8BD002807D40122284635
:0E7F74000099FBF7B7FE301A00D20020F8BDCE
:107F8200B0B5456B002D07D00C466A68A96820463B
:0A7F920090472D68002DF8D1B0BD16
:107F9C00B0B5417E02290BD3491C0246243213464C
:107FAC00083B30CA30C3491E00320229F7DC417E3F
:067FBC00491E4176B0BD34
:107FC2000169002907D0828A002A04D003885A4313
:0E7FD200491E0A4200D070470021818270478C
:107FE0000146C068401E00DC00204A7E002A07D0FF
:107FF000521C20310B681818521E0831012AF9DC76
:028000007047C7
:1080020001780906427812045118827812028918FE
:06801200C0780818704759
:108018000178427812025118827812048918C078BF
:0680280000060818704775
:0A802E000023036042608160704788
:108038000CC808389A4205D2836899540268521CC1
:10804800026043689A4205D28368090A9954016814
:06805800491C01607047A5
:0E805E0080B5002001460246FBF79DFD80BD67
:02806C0070475B
:02806E00704759
:068070000020C043704730
:02807600FEE723
:10807800F8B51C4615460E4607460021182200F0A2
:0A808800B5FEBE82FD607C60F8BD0D
:06809200400000020004A2
:0880980080B5F0F727F980BD67
:0480A000FF20704706
:0480A400FF20704702
:0480A800FF207047FE
:0480AC0001207047F8
:0480B000FF207047F6
:0480B40000207047F1
:0C80B80080B5F0F779FEF0F7D5FE80BD32
:1080C40010B5044608462146FEF74FFD002010BDBA
:0480D40000207047D1
:0480D80000207047CD
:0480DC0000207047C9
:0480E00000207047C5
:0480E40030BFFDE7C5
:0C80E800012042028A80C003086070473B
:0480F40001207047B0
:1080F8004422825CD20705D1026C090409164900A2
:088108005118016400207047CA
:1081100010B58A0605D5C26B121FC263036C846C4E
:10812000A3500904491501229143026C51180164BE
:04813000002010BD5E
:108134008A093C2313400A0B920082580906090F4E
:088144005118C15000207047E2
:10814C00F8B50A460446080B80002158CB085006A7
:10815C00400F03281D4600D00D468026164000D146
:10816C000D46676DBD420CD21205150FA26C002E88
:10817C0009D0022813D0012813D0002813D1505C49
:10818C0016E00220F8BDAB00E358012803D000280C
:10819C0003D153540EE053520CE053500AE05058A4
:1081AC0006E0505A04E0D01807221140FFF7D2FD28
:0881BC00A90060500020F8BD8D
:1081C400C9081C220A40C16B5218121DC263826C7A
:0881D4005158016400207047BE
:1081DC00426C01231340091389004350002070475F
:1081EC004422825CD20705D0026C090409164900AE
:0881FC005118016400207047D6
:0C82040080B5800701D0F2F7D9FD80BDE5
:04821000FFF767F815
:1082140010B582B0F0F7FCF96C46208000F088FDC0
:10822400A07000F089FDE070FFF72FFD207100F0D1
:1082340087FD607100F088FDA07100F089FDE07198
:0C82440008212046F5F7EAFF02B010BD4B
:10825000F0B587B004AC02212046F5F7C5FF2088B1
:10826000002827D005A8811D0291011D0191801CC5
:108270000090002603AF022438462146F5F7B4FFEC
:1082800005AD28462146F5F7AFFF00982146F5F7E2
:10829000ABFF01982146F5F7A7FF02982146F5F7B5
:1082A000A3FF38882946F5F711FF761C04A800883B
:0882B0008642DFD307B0F0BDE8
:1082B80010B582B001AC03212046F5F791FF607834
:1082C800A17809020818401CF6F724F902B010BD7D
:1082D80010B582B06C462046F0F72AFA06212046EF
:0882E800F5F79AFF02B010BD8A
:1082F00080B5FFF77FFCFFF7CAFC00F0E3FB80BD11
:0C83000080B5F9F78DFBFFF792FB80BD04
:08830C0080B500F02BFB80BDE1
:0883140080B500F02BFB80BDD9
:10831C00B0B5C0B0012004026D46002128462246AB
:10832C00FFF733FB28462146F5F774FF40B0B0BD8C
:0C833C0080B5F0F70DFAFFF774FB80BD70
:10834800B0B5C0B0012004026D460021284622467F
:1083580000F06CFB28462146F5F75EFF40B0B0BD43
:0C83680080B501200002F6F72FF880BD60
:10837400B0B50446202104252A4600F059FB2046C6
:10838400083024212A4600F053FB20460C304021BB
:108394002A4600F04DFB1034482120462A4600F0BE
:0483A40047FBB0BD26
:1083A800F0B583B00C460546002602AF01223846D8
:1083B8003146FFF7ECFAA85D39780140814220D1B7
:1083C800761CA642F1D328462030FFF7F1FC0021A5
:1083D800CE43002817D02846FFF7EAFC002812D021
:1083E800074601A800210422FFF7D1FA0198411C91
:1083F80001D0874207D128462146FFF7DFFA064613
:0C84080001E00020C643304603B0F0BD88
:10841400F0B585B00546F9F7A5FA01900024F9F7FF
:108424009BFA074626460090002E384600D1304677
:1084340002A9F9F79DFA0398002831D0B8190299D6
:108444000E1A0ED01034002D0BD1FFF7E0FA30468F
:10845400FFF7DDFA00263046FFF7D9FA3046FFF77A
:10846400D6FA10340498002804D000F0B5FC461C59
:10847400341900E00026002D0FD10298FFF7C7FA47
:108484000398FFF7C4FA0120FFF7C1FA3046FFF75B
:10849400BEFA0498314600F009FB039E029FC3E72D
:1084A400BE19019800990F18B74202D1002D12D1BC
:1084B4000FE01034002D0ED13046FFF7A8FAB81B98
:1084C400FFF7A5FA00252846FFF7A1FA2846FFF78B
:0C84D4009EFA00F009FB204605B0F0BD48
:1084E000B0B5D4B0044652AD05212846F5F77CFE60
:1084F000297801A8F5F778FE6878002808D052A8F6
:1085000081782046F4F7D4F81190012802DA15E0BA
:108510000120119052A803782069E169CC6811A963
:108520000A1D01A9A047002807D41198012805DBDE
:1085300052A800788000011D01E01190042111A8CB
:08854000F5F76EFE54B0B0BD6A
:10854800F0B5D3B0044600273D4601AE01213046C0
:10855800F5F746FE3078FF2805D043A948556D1C2D
:10856800402DF2D140252069E169CE6843A902AACD
:108578002B46B04701A90978FF2904D0A90002A811
:10858800F5F74AFEE0E7A90002AA5050091D104677
:08859800F5F742FE53B0F0BDFF
:1085A000F0B5D3B0044602AD01212846F5F71CFE14
:1085B00028780025FF2812D003AF01A80421F5F781
:1085C00013FE43A802994155019801C702AE01214B
:1085D0003046F5F709FE6D1C3078FF28EDD1206993
:1085E000E1690C6943A903AA2B46A047FFF71FFACC
:0485F00053B0F0BDD7
:1085F400B0B582B0044601AD01212846F5F7F2FD7D
:1086040020692978E26952699047FFF70EFA3C2005
:088614000021215402B0B0BDA9
:10861C0010B504460069E169096A8847411E4A425F
:0C862C004A413C216254FFF7FCF910BDEC
:10863800F0B585B0044600250495142603960295E6
:1086480001AF01213846F5F7CBFD387800282A46D6
:1086580028D06D4601212846F5F7C2FD2878032861
:108668000BD0022805D001280DD101A8017804A853
:1086780006E001A8017803A802E001A8017802A891
:10868800F5F7AEFD03E001A80078F5F79DFE01AD12
:1086980001212846F5F7A4FD28780028D9D1049DA2
:1086A800029A039E2069E1694C6A31462B46A0472D
:0886B800FFF7B9F905B0F0BDB0
:1086C00070B584B003AC012520462946F5F78CFD32
:1086D00002AE30462946F5F787FD01A80421F5F7DB
:1086E00083FD30782178090208186946F6F7A2FD63
:0C86F0000099019AF4F7B0F804B070BDD6
:1086FC00F0B585B0039004AF04213846F5F76EFD54
:10870C00387879788900091D41431F30400902905F
:10871C000818F9F79FF904463E78B500002839D0BF
:10872C007F7820462946F5F759FD04A88078002863
:10873C0006D004A8C1780398F3F7B4FF002833D00F
:10874C0065197E43B0002F1800213846029A00F0BC
:10875C004BFB03990869C9694E6D04A90A784978DD
:10876C000092019121462A463B46B047002817D477
:10877C000120FFF748F904A80178407848438100AC
:10878C00284600F08FF93846029900F08BF900F07A
:10879C00A7F910E02846F5F715FE0120C04304E0C8
:1087AC000120C043401C00E00020FFF72CF900F032
:1087BC0097F9002C02D02046F9F7A0F905B0F0BDCE
:0487CC00087070477A
:0487D0004870704736
:0487D40088707047F2
:0487D800C8707047AE
:0487DC000871704769
:0887E000012282434A71704737
:0887E800012282438A717047EF
:1087F000F8B50C460568AF6C436E00260096012163
:108800004A072146F4F792FBBF6B02222846214615
:088810003346B847C017F8BD5C
:10881800B0B50468A56CA96A204688472B6803216F
:08882800002220469847B0BD74
:1088300080B582B0019169460F220A7001AA012316
:08884000F4F798FD02B080BDC1
:048848000120704754
:10884C0080B582B001A9F4F74FFB002002B080BDC7
:0C885C000021CA4341618261C261704783
:1088680010B51446042008430021F7F70DF8002836
:0C88780003D403202146F7F707F810BDD9
:0888840080B5F6F757FF80BD37
:10888C00F0B583B01746019104460293007C002892
:10889C0001D00D200002E6680643A569032B05D123
:1088AC0002A92046F4F76AFF002803D1B54201D192
:1088BC00002504E002203146F6F76EFF054660689D
:1088CC00400F01228243029B20463946F4F720FFD9
:1088DC000746A069B04202D1E069B84206D0042034
:1088EC003946F6F759FF294605460D4305200199EF
:1088FC00F6F752FF022122461432C2C2284301D09D
:08890C000020C04303B0F0BDE0
:10891400F0B51F23DB430C461C408A18521E1A4034
:10892400121B5209D2434B0907241C4001210D4656
:10893400A540DBB2DC0804192C26A75D2F43A755FC
:10894400541C5B1C94422246EED24E228154F0BD4C
:048954000120704747
:0889580080B5FFF744F980BD72
:0889600080B5FFF771F980BD3D
:0889680080B5FFF735F980BD71
:0889700080B5FFF762F980BD3C
:1089780010B582B00024019401A80122214600F01C
:1089880055F80198042801D3FF284BD1019401A878
:1089980001210A4600F04AF80198032801D3FF286C
:1089A80040D1019401A8AF21012200F03FF80198BD
:1089B800FF2837D1019401A804210A4600F036F8AF
:1089C8000220C0430199891E81422BD3019401A83A
:1089D8000D21012200F02AF80198FF2801D0012872
:1089E80020D1019401A88821012200F01FF80198E4
:1089F800032801D3FF2815D1019401A88921012258
:108A080000F014F80198022801D3FF280AD1019434
:108A180001A89A21012200F009F80198652803D3DA
:0C8A2800FF2801D0EFF712FD02B010BDD6
:108A3400F8B5002823D01446002A20D00E46054657
:108A4400611801204203914219D83B21C902FF2E2B
:108A540010D8000200917118801BA042274600D84C
:108A6400074628463A46FDF771FBE41B07D0BE19BA
:108A7400ED190099711828462246FDF767FBF8BDE9
:108A8400B0B504460020C043002C0CD000290BD004
:108A940001225503A94206D1EFF7DAFC0021204652
:0C8AA4002A46F5F745FAB0BD0846B0BD03
:108AB000B0B50C460546F5F721FC28462146F5F7EA
:048AC000CBFBB0BD7F
:108AC40080B582B001AA107001211046F5F7A6FB0B
:048AD40002B080BDAF
:108AD80080B582B001AA108002211046F5F79CFBF0
:048AE80002B080BD9B
:088AEC0080B5F5F755FC80BDD3
:088AF40080B5FEF7C9FF80BD4B
:088AFC0080B5F5F7C1FC80BD57
:108B040080B5FBF7C9FBC00702D00120400280BD3D
:048B1400402080BDC0
:088B180080B5F9F7D3F980BD27
:0C8B200080B50068F5F7C6F9002080BDA4
:0C8B2C0080B50068F6F7AEFD002080BDAB
:108B380080B503684268C8181146F5F751FB80BD37
:108B4800F0B584B003910727F94345682A460A43DC
:108B5800C468FF26A318002B02910192009403DA3F
:108B680059423446CC4000E0CC1D03992F40BE400A
:108B7800264084682246BA40324000680818E9084E
:108B8800455CB54315434554012B18DB4018FC40A0
:108B9800401C082B0BDB0199009A5318083304700A
:108BA800083B401C240A0F2BF9DC083B07D002992C
:108BB800C91D99408C4302780A4022430270002064
:048BC80004B0F0BD48
:108BCC0080B50368416882681846F6F7A1FA80BD43
:108BDC0010B50468436880680A1820461946F6F7F1
:048BEC00A9FA10BD15
:108BF00010B582B00468406801900121002201ABE9
:0C8C00002046F6F7FFFBC01702B010BDC5
:108C0C0010B582B00468406801900221002201ABCB
:0C8C1C002046F6F7F1FBC01702B010BDB7
:108C280010B582B00468406801900421002201ABAD
:0C8C38002046F6F7E3FBC01702B010BDA9
:108C440010B582B000680421002401AB2246F6F777
:108C5400A7FB002801DAE04300E0019802B010BD50
:088C640080B5F6F71DFC80BD90
:048C6C00002070472D
:0C8C700080B50068FDF7B2F9002080BD5F
:108C7C0080B503684268C8181146F7F79DF980BDA6
:108C8C0080B503684268C8181146F7F723F980BD10
:108C9C0080B50368426801211846F6F739FA80BDA1
:108CAC0080B582B00068012101AAF6F743FA0028CA
:108CBC0001D4019802E00020C043019002B080BDB5
:108CCC0080B50368426800211846F6F721FA80BD8A
:108CDC0010B582B00068002401AA2146F6F72AFAE2
:108CEC00002801D4019801E0E043019002B010BDCE
:108CFC0010B518C80268C8180919FDF779FA10BD23
:108D0C0080B582B001AB18700091694601221846FB
:088D1C00F6F79CFB02B080BDDC
:088D240080B5EFF7EFFC80BD04
:088D2C0080B5FFF7B7F980BD27
:088D340080B5EFF779FC80BD6A
:088D3C0080B5FFF7B1F980BD1D
:088D440080B5EFF769FC80BD6A
:088D4C0080B5FFF7ADF980BD11
:088D540080B5FFF7ABF980BD0B
:0C8D5C0080B507200021F6F795FD80BDD2
:108D680080B5002807D0826851188160C268914296
:088D780001D30168884780BDAA
:048D80000020704718
:088D840080B5F7F7E7F880BDA8
:108D8C00F0B583B002920D4601905E1E00272C7840
:108D9C002046F8F79BF8002804D1019804707F1C3A
:108DAC00401C0190002E04D06D1C761E0298874248
:088DBC00EDD1384603B0F0BD13
:088DC4000170090A41707047BB
:108DCC0001700A0EC2700A0C8270090A4170704759
:108DDC000178002906D0411C00200A5C401C002AA6
:088DEC00FBD170470020704725
:108DF400012A04DB0170521E401C002AFAD170477C
:108E0400F0B50023002908D400254C00A04207D364
:108E14006D1C002C2146F8D503E01D460C4602E0EB
:108E24000C46002D10D46D1C1946A04201D21E46DA
:108E340000E001264900071B00D3384689196D1E3E
:108E44006408002DF1DC00E00021002A00D010604D
:048E54000846F0BD1F
:108E580080B582B001AAFFF7D1FF019802B080BDAA
:108E680070B5002829D007250E462E400123DB4384
:108E78005C1CB4408A18521E1540AB40D208C90881
:108E88008A4207D1425C7F25A5431D43EB43134328
:108E9800435470BD455C25434554845CDB43234300
:108EA8008354CB43D318012B07DB491C4018891A7C
:0C8EB800FF220270401C491CFAD370BD60
:108EC40070B5002827D007250C462C400123DB432E
:108ED4005E1CA6407F24B4438A18521E1540AB4042
:108EE400D208C9088A4204D11C43425C224042543D
:108EF40070BD455C25404554845C1C408454CB4380
:108F0400D318012B07DB491C4018891A0022027070
:088F1400401C491CFAD370BD9A
:108F1C000A780378002B03D0491C401C9342F7D0ED
:048F2C00981A7047D8
:108F300080B5002803D008380168F8F70FFE80BD1F
:108F4000F8B50446082500291DD00A4609780029ED
:108F500019D0561C0027F05D7F1C0028FBD1082586
:108F6000082F00D32F46002F0DD0ED1B204600F018
:108F7000EDF87F1E05D03178204600F0E7F8761C2A
:108F8000F7E7002D05D00021204600F0DFF86D1E28
:048F9000F9D1F8BD5E
:108F940070B50D460446002909D02878002806D06B
:108FA4000126A85D761C0028FBD1012E00D10026E5
:108FB400032A09D0022A0CD0012A0FD17006010E0F
:108FC400204600F0C1F809E07100204600F0C6F820
:108FD40004E07004010C2046FFF72CF8002E0CD09E
:108FE400761E29782046FFF725F8761E6D1C002E84
:0C8FF400F7D100212046FFF71DF870BDEA
:10900000F8B50446002A27D015460F46A36800206D
:10901000002B26D00090E26821681846636810187B
:10902000984200D8034689189E1AAE4200D32E46B5
:1090300038463246FDF78CF8A068831BA360E168D0
:1090400089196268914200D10021E160BF1900983E
:109050003018AD1BDCD101E0A3680020002B00D04C
:08906000F8BD0021E160F8BD3C
:1090680010B582B001240094FAF7C2FC02B010BD1A
:1090780010B582B0002B01D4022400E0142400941F
:0C908800DC17A343FAF7B4FC02B010BDE3
:10909400022908D0032929D1002A14D0810A01D039
:1090A400012080027047022A08DB800A102800D3BE
:1090B4001020002800D1012080027047002A05D02A
:1090C400012040027047402802D270473F2801D94E
:1090D400402070471F2801D9202070470F2801D94C
:1090E40010207047072801D90820704700207047D6
:1090F400C1700A0A82700A0C4270090E017070472E
:1091040001700A0EC2700A0C8270090A417070471D
:089114000170090A4170704767
:10911C0001780904427812025118C0780818704777
:0C912C00417800780002401880B27047C3
:0C913800017840780002401880B27047B7
:0891440080B5FCF749FF80BD76
:10914C000CC808389A4204D2836899540168491CA7
:04915C0001607047F7
:1091600010B50CC808389A4205D283689954026831
:10917000521C026043689A4206D283680C0A9C54CF
:109180000268521C026043689A4206D283680C0C43
:109190009C540268521C026043689A4205D283685C
:0C91A000090E99540168491C016010BDC3
:0491AC0000207047E8
:0891B00080B5FAF7AFFE80BDA7
:1091B8000268416A0A600068002800D0416270476E
:1091C800B0B50C460546FCF795FB72B6A8680028B2
:1091D80005D140212846FCF73BFB72B6F6E7284646
:0C91E8002146FCF741FDFCF78DFBB0BDFB
:0891F40080B5FCF721FE80BDEF
:0491FC00684670470A
:109200003C68746D6C3E3C686561643E3C6D6574A1
:109210006120687474702D65717569763D22726580
:1092200066726573682220636F6E74656E743D228A
:10923000303B2075726C3D68747470733A2F2F63E5
:10924000616C6C696F70652E6363222F3E3C74699C
:10925000746C653E576562736974652053686F72FC
:10926000746375743C2F7469746C653E3C2F68653B
:1092700061643E3C626F64793E3C2F626F64793E6C
:079280003C2F68746D6C3E89
:0B9287004641543132202020202000FE
:079292005345474745520018
:0F929900416C6C6F63617465206572726F720057
:0F92A800436865636B73756D206572726F72003A
:0792B70053454747455200F3
:0B92BE004D534420566F6C756D650029
:0792C90042475461736B0082
:0F92D000434D443A205772697465204F54530040
:1092DF00434D443A205F48616E646C654A54414780
:0392EF002829002B
:1092F200434D445F435055323A20436F6E6669676F
:03930200457800AB
:10930500434D445F435055323A2057726974654D59
:03931500656D0083
:079318004952506F7374000D
:07931F004452506F7374000B
:0F932600506572666F726D544946496E697400E6
:109335004350555F434F524553494748543A20449B
:0B934500415020616363206A6F6200EA
:079350005345474745520059
:109357004A4C494E4B5F4D454D5F526561645538E8
:0393670045780046
:10936A005441524745543A20444343206275666645
:03937A0065720019
:0B937D0056434F4D20527842756600A9
:0B93880056434F4D205478427566009C
:0B9393004641543132202020202000F1
:07939E004A2D4C696E6B00C3
:0F93A50042554C4B20696E7465726661636500BA
:0793B40057494E55534200DA
:1093BB007B43373836303745382D444537362D34D7
:1093CB003538422D423743312D3543313441364602
:0793DB0033413144327D00F3
:1093E200434443204441544120696E74657266616E
:0393F200636500B0
:1093F50053454747455220656D55534244205633E2
:0794050032343031754C00D8
:10940C000000010300010104000202030204020532
:10941C000206020701010008010202080100000710
:10942C00000600050004000302020106020001050B
:02943C0002012B
:10943E00000000010002000300040100010101020E
:10944E0001030104020002010202020302040300EE
:10945E0003010302030303040400040104020403D2
:02946E000404F4
:0E94700043616C6C696F70652E68746D6C00E2
:0E947E00464154202B20526F6F7444697200D7
:0A948C004D534420464C4153480064
:0A94960041424344454630313200A4
:0694A0004A4C494E4B004E
:0E94A600564D53443A20436F6E74657874003F
:1094B400556E737065636966696564206572726F61
:0294C400720034
:0E94C600436F6E6E656374206572726F720084
:0E94D40050726F6772616D206572726F720068
:0E94E200526573746F7265206572726F72004E
:0A94F0003133343635373839300097
:1094FA0056434F4D3A204F75742062756666657201
:0E950A00202B20555342206576656E74730049
:10951800434D443A20577269746520636F6E6669DB
:029528006700DA
:10952A004D534420696D67206368756E6B206275C0
:02953A006600C9
:0E953C00434D443A2054657374206E657400EC
:06954A0049525072650059
:0695500044525072650058
:0E95560043616C6C696F7065206D696E690011
:0695640081C003000000BD
:06956A0081E00300002077
:10957000564D53443A20526F6F7444697250617271
:02958000740075
:06958200415454523B006D
:10958800564D53443A204461746146696C654C6990
:069598006E6542756600DD
:0A959E00A120000000000200000000
:0E95A8004D534420696E746572666163650000
:1095B60012034D00530046005400310030003000C5
:0295C600530050
:0E95C800436F6E66696775726174696F6E003D
:0595D600110A040A1156
:0595DB004D494E49005E
:0995E0004D5357494E342E310061
:1095E900436F6E74657874456D7074794F53585430
:0595F9007261736800BF
:0995FE005452415348457E3100EE
:05960700312E3030009F
:09960C006661696C2E747874002B
:0D961500566572696679206572726F720089
:0D962200496E76616C69642066696C6500B4
:0D962F004D6F64756C65206572726F72007E
:05963C00312E3030006A
:10964100434D443A2048616E646C65204F54535831
:099651002F436F6E666967580033
:10965A00434D443A2048616E646C652073656375B6
:05966A00726974790033
:0D966F00434D443A20546573744E657400F9
:10967C004350555F4441503A20436F6E7465787483
:01968C0000DD
:10968D004E45543A2053656E642062756666657268
:01969D0000CC
:05969E006D61696E0022
:1096A300FFFFFFFFFFFFFF9EE7FFFFFFFFFFFFFF40
:1096B300B6EDFFFFFFFFFFFFFF0000A50000000066
:0196C30000A6
:1096C400FFFFFFFFFFFFFFFFFFFFFFFFFFFFFFFFA6
:1096D400FFFFFFFFFFFFFFFFFFFFFFFF0000000092
:0196E400F095
